:020000040800F2
:1040000000500020357D0008097C00080D7C000868
:10401000117C0008157C0008197C000800000000D5
:10402000000000000000000000000000217C0008EB
:104030001D7C000800000000257C0008DDA20008AF
:10404000297C00082D7C0008317C0008357C0008A4
:10405000397C00083D7C0008417C0008457C000854
:1040600000000000497C00084D7C000800000000B2
:104070000000000000000000000000000000000040
:1040800000000000000000006D7C0008717C00084A
:10409000817C0008917C0008AD7C0008FD4500088B
:1040A000BD7C0008054A0008000000000000000078
:1040B0000947000839460008DD460008C17C0008B1
:1040C000C57C0008C97C0008CD7C0008D17C0008B4
:1040D000D57C0008D97C0008DD7C000881450008FB
:1040E000E57C0008E97C0008ED7C00080000000089
:1040F00000000000000000000000000000000000C0
:0C41000000000000000000005FF800005C
:10410C0030BF704720BF704740BF7047BFF36F8F01
:10411C007047BFF34F8F7047BFF35F8F704701DF5E
:10412C007047EFF31480704780F31488BFF36F8FE0
:10413C007047EFF30980704780F309887047EFF3FD
:10414C000880704780F30888704772B6704762B673
:10415C00704771B6704761B6704780F3118870472D
:10416C00EFF31280704740BA704700BA70470000F6
:10417C00054A0649064B1160064A1360064A13604D
:10418C00064A1360704700BFC40400201591000854
:10419C00CD8F0008A00400206403002098040020A8
:1041AC00064A074B1A60074A074B1A60074A084B26
:1041BC001A60084A084B1A60704700BF39B20008F1
:1041CC006403002045B40008C404002039B400087E
:1041DC009804002035B20008A004002030B597B038
:1041EC0003F0B6FA03F0D4FA09F0F0FF6A4B00259D
:1041FC004FF480301D700AF009F80AF06DF90128AF
:10420C00044627D110200AF093FC02200AF078FC17
:10421C0028460AF04BF828460AF05CF84FF4806008
:10422C000AF04EF84FF480304FF4E0110AF01AF80F
:10423C0020460AF023F839200AF038F90028FAD081
:10424C0002200AF021F80AF029F80828FBD1524B79
:10425C0001221A70012001460AF0DEF84FF00060CE
:10426C004FF480410AF03AFA4FF440700AF098F992
:10427C004A4B1B78552B0ED1494B1B78532B0AD12B
:10428C00484B1B78422B06D1FFF772FF464B01229D
:10429C001A70013A05E0FFF783FF434B00221A70B6
:1042AC000132424B424C1A7005F068F905F0A0F946
:1042BC0007F0DAFA03F0F0FE20463E4905F058FB11
:1042CC0006F046F805F06EF93B4B1B78012B05D137
:1042DC00207804F083FCE07804F0ECFB324B1B7884
:1042EC00012B25D1354C0DF1100C25460FCDACE82A
:1042FC000F00AE46BEE80F00ACE80F009EE80F00C2
:10430C0030340DF1400E8CE80F000FCCAEE80F00EE
:10431C0094E8030005248EE80300009404AC019497
:10432C00042010AC264902221C23029404F0B0FF96
:10433C001E4B1B78012B05D11D4B1A6958799968B6
:10434C0007F080F800F046F800F03CF800F056FD5D
:10435C0001F05EF903F0E8F940F2127006F088FA09
:10436C0040F2167006F026FA03F04AFB03F0B8FA96
:10437C0000F046F820B902F0DBFE00F095FC04E0FA
:10438C00012002F0D5FE00F0B7FD03F0CFF906F0E6
:10439C0047FA00F09FFBE9E7B0040020FC3F00085F
:1043AC00FD3F0008FE3F00081800002051000020CF
:1043BC00C8040020D00300204E00002074FF000829
:1043CC0000080140024B00225A601A70704700BF6F
:1043DC0094010020084A094B12680021D20283F88C
:1043EC002C109A629A605A611A62DA609A615A6267
:1043FC001A61DA61704700BF14000020940100209C
:10440C00014B93F82C00704794010020014B186B62
:10441C00704700BF94010020014B586B704700BFE0
:10442C0094010020014B1868704700BF2809002038
:10443C00014B986B704700BF9401002008B5024BEC
:10444C0018680BF06BFD08BD60090020014BD86BA0
:10445C00704700BF94010020014B1868704700BFE3
:10446C007C090020014B1868704700BF3009002000
:10447C00014B1868704700BF38090020034B93F8B4
:10448C00462022EA000283F846207047D003002021
:10449C00034B93F8463018420CBF002001207047A4
:1044AC00D0030020034B93F85D2040EA020283F80E
:1044BC005D207047D0030020034B93F85D2022EA67
:1044CC00000283F85D207047D0030020034B93F863
:1044DC005D3018420CBF002001207047D003002033
:1044EC00014B1868704700BF4C090020014B18683D
:1044FC00704700BF14090020014B5868704700BF7B
:10450C0014090020014B1868704700BF6409002093
:10451C00014B5868704700BF6409002008B50120A2
:10452C00FFF7D4FF48B1054B00220420DA63FFF7F4
:10453C00CDFF10B10120FFF7BFFF08BD9401002093
:10454C0008B506F083FB08BD08B506F0E7F908BD11
:10455C0008B54FF4803004F0E5FF08BD08B5044BF6
:10456C0093F86C301BB94FF4003004F0DBFF08BD3E
:10457C00D003002008B5034B1B78012B01D104F0AC
:10458C00D1FA08BD4F00002008B50220FFF780FFCC
:10459C0038B1044BB3F8440006F05EFB0220FFF781
:1045AC006DFF08BDD003002008B50120FFF770FF98
:1045BC00C0B106F05BFB0C4991F825300A6C5B0826
:1045CC00B2FBF3F3B0FBF3F202FB1303074A21F83F
:1045DC00443F126802F14400022205F035F8012034
:1045EC00FFF74CFF08BD00BFD003002004000020E3
:1045FC0008B54FF480700AF00DFB88B14FF4807051
:10460C000AF016FB074B1B78012B03D0064B1B78CB
:10461C00012B05D1FFF7C8FFFFF7B6FFFFF77EFFB1
:10462C0008BD00BF4C0000203B02002008B5044B25
:10463C001978012903D1034B186809F06BFA08BDEE
:10464C004C0000204800002038B51D4C0221206889
:10465C0009F05AFA012827D10221206809F05AFAE8
:10466C00002003F0CFF9174C0546014694F84000A2
:10467C0006F01CF9144B84F8405093F8212080B2BA
:10468C00062A11D1E26B01B28A18E26360B193F889
:10469C006D304BB10D4B9A6812F0200F02D02022D6
:1046AC005A6101E020221A61054C0121206809F0B1
:1046BC002BFA0128014602D1206809F02BFA38BDEB
:1046CC004000002094010020D00300200010014085
:1046DC0008B5074B1978012903D1064B186809F066
:1046EC0019FA054B1B78012B01D1FFF7ADFF08BD63
:1046FC003B020020480000204400002008B5074B76
:10470C001978012903D1064B186809F003FA054BF7
:10471C001B78012B01D1FFF797FF08BD3A0200204F
:10472C00480000203902002038B5244B93F8212092
:10473C00072A25D0082A39D0062A3DD1204A01283B
:10474C00D36B1F4D08BF536401286A6C1D4C6B64FE
:10475C0002D1AB6C23602FE09B1A184A206892F8A8
:10476C0025104EF66022534349080622514322324B
:10477C0093FBF1F107F0C0F920602368AB641BE0F8
:10478C0001280F4A0F4C02D1D36C23600AE00E496A
:10479C000868196C4EF66023434393FBF1F32360D6
:1047AC002368D364084B00221A6005E0074B186895
:1047BC000BF0B4FB034B186038BD00BFD0030020D6
:1047CC0094010020300900207809002060090020A5
:1047DC0010B504464FF4804004F0A4FE034B0120B6
:1047EC00DC639C63FFF7A0FF10BD00BF94010020A9
:1047FC00B0F5007F10B5044610D003DCB0F5807F17
:10480C0037D121E0B0F5806F03D0B0F5006F30D117
:10481C000DE004F07FFE4FF4807019E004F07AFE96
:10482C004FF4807004F07EFE4FF4806014E004F0CE
:10483C0071FE4FF4807004F075FE4FF4806004F04C
:10484C0071FE4FF400700BE004F064FE4FF48060D6
:10485C0004F068FE4FF4007004F064FE4FF4006046
:10486C0004F060FE4FF4804004F05CFE024BA3F8B1
:10487C006E40024B1C6010BDD00300203409002098
:10488C0010B504464FF4803004F054FE012808D0D3
:10489C00044B4FF400601C60FFF7AAFF024B002290
:1048AC001A6010BD3C0900206009002038B505468F
:1048BC004FF4803004F03EFE01281CD00E4B4FF418
:1048CC0080601C680D4B9D63FFF792FF4FF4804096
:1048DC0004F028FEB4F5007F04D1094B1A68094B8B
:1048EC001A6008E0B4F5006F05D1074B18680BF09F
:1048FC00FBF8044B186038BD3409002094010020EB
:10490C0060090020F80800203009002008B5034B8E
:10491C00DB6BC018FFF7CAFF08BD00BF9401002075
:10492C0038B505464FF4803004F004FE01281AD047
:10493C000D4B4FF400701C680C4B1D60FFF758FFBB
:10494C00B4F5006F05D10A4B18680BF0CDF8094B84
:10495C001860094B9B6813F4004F04D104F004FE5B
:10496C0008B902F085FF38BD340900207C0900200D
:10497C0030090020600900200010014008B54FF4F8
:10498C008070FFF735FF08BD38B5174B186809F074
:10499C00B3F8164B0422196C91FBF2F290420ADA2E
:1049AC004FF0030C0CFB02FC114B1B6D634502DD3D
:1049BC00CB1A1B180DE003235343984206DD0C4B16
:1049CC001B6D934202DAC31A5B1A02E0084B1B6D93
:1049DC00C31A074A0749D46B0D68E41AEB1A0B602B
:1049EC001065D46338BD00BF48000020D003002000
:1049FC009401002078090020224A08B51288224B25
:104A0C0012F0100F2ED121495A6D08680132013075
:104A1C00086019785A65012903D11D4B4FF40051D8
:104A2C0019611C4B93F82130072B0AD1132A05D995
:104A3C00154A002318465365FFF776FE0120FFF751
:104A4C00A3FF144B93F82130062B01D0082B13D164
:104A5C000D4B5A6D132A0FD9002210465A65FFF7D9
:104A6C0063FE09E01978012906D1094B4FF4005275
:104A7C0009485A610AF04CFD0248012109F04AF834
:104A8C0008BD00BF002C014094010020100900203B
:104A9C0000100140D00300200024014008B502F0B2
:104AAC00F7FEA0B904F060FD88B900F5005004F0E1
:104ABC0041FD60B900F5807004F03CFD38B9044B41
:104ACC004FF461729A861A879A8702F0D1FE08BD5C
:104ADC00002C014010B505F035FC204CA36DC31A19
:104AEC00002BB8BF5B42B3F57A7F36DD1C4B9B685D
:104AFC0013F4006F2AD102F0CBFE60B1012004F058
:104B0C0009FD402004F006FD94F85C300A2B02D815
:104B1C00013384F85C304FF4807004F00BFD20B945
:104B2C00FFF7FEFE0F4B00221A6002F0B1FE80B1BF
:104B3C000A4B93F85C300A2B0BD8094B4FF480626C
:104B4C001A6140205A6104F0EDFC02E0002384F865
:104B5C005C3005F0F7FB014B986510BD940100200B
:104B6C00001001406009002010B505F0EBFB194C5A
:104B7C00236EC31A002BB8BF5B42642B28DD164B87
:104B8C00186803F0F9F8154B206393F82F30012BBC
:104B9C000AD103F55A63984206DD02F071FE042037
:104BAC0004F0B8FCFFF7EAFE0A4B1B6BB3F57A7FF7
:104BBC0002DC022004F0AEFC064B1B6BB3F57A7FD3
:104BCC0002DD022004F0AEFC05F0BCFB014B1866C4
:104BDC0010BD00BF9401002038000020D00300203D
:104BEC0010B505F0AFFB264C636EC31A002BB8BF93
:104BFC005B42B3F57A7F42DD224B186803F0BCF8B8
:104C0C006063082004F096FCB8B9636B40F6B322DD
:104C1C00934209DD083004F07DFC02F063FE02F0E3
:104C2C002FFEFFF7ABFE26E0B3F5156F0ADC08206C
:104C3C0004F078FC02F05CFE09E0626B40F60B239A
:104C4C009A4218DC082004F06DFC02F057FE0E4B63
:104C5C009B6813F4004F0ED104F086FC58B900F594
:104C6C00005004F067FC30B900F5807004F062FC71
:104C7C0008B902F0FDFD05F065FB014B586610BD4F
:104C8C00940100203C0000200010014008B5054AAA
:104C9C000346022093FBF0F080B282F8253005F039
:104CAC0097FF08BDD00300202DE9F0413A4B93F853
:104CBC002C201446002A6DD15A68254601325A60C0
:104CCC00012D05D0022DDFF8DC8008D0334B07E036
:104CDC00334B186803F050F8324B1F6805E0324B29
:104CEC00186803F049F8D8F8007047432F4B1A594D
:104CFC00974201D901321A512D4B1A59974201D2C0
:104D0C00013A1A512A4B03F10C021E59125918334D
:104D1C00B6181B5976089E4201D95E1C01E038BFBB
:104D2C005E1E012D09D0022DDFF878800CD0D8F84A
:104D3C0000101A4BB6FBF1F10BE01A4B1968184B2B
:104D4C00B6FBF1F1186805E0D8F80010164BB6FB6D
:104D5C00F1F1186803F018F8154B16491A590E5151
:104D6C00BA4201D201321A51104B1A59BA4201D926
:104D7C00013A1A5101350434032DA1D1094B4FF4DA
:104D8C007A711A68044B4A435968914202DB01223A
:104D9C0083F82C20BDE8F08194010020340200201F
:104DAC00300000201400002034000020A801002056
:104DBC009C010020B401002010B50C4C23789BB949
:104DCC000B4B4FF40061186802F0DEFF094B4FF4F7
:104DDC000061186802F0D8FF074B4FF400611868A7
:104DEC0002F0D2FF0123237010BD00BF94010020FC
:104DFC0034020020300000203400002010B502F0F6
:104E0C004FFD012002F0F8FF2B4C2C4803F036FE2E
:104E1C002B4803F033FE05F05DFB94F82130062B94
:104E2C000FD14FF4004004F075FB802004F07AFBA6
:104E3C00012005F0EBFD94F82500400805F0ACFDD1
:104E4C0001E005F0C3FD1C4C94F82130072B21D157
:104E5C004FF4004004F066FB802004F063FB94F8F0
:104E6C002E30012B02D1002005F0D0FD124C206C0D
:104E7C0094F8301005F050FF94F82510206C490878
:104E8C0005F0B2FE05F0C0FE03F07CFA012005F03F
:104E9C00C1FE01E005F00AFF0A4C4FF4007301203B
:104EAC00236102F0AFFF4FF480432361FFF7F6FD5F
:104EBC00FFF782FF10BD00BFD003002014090020B3
:104ECC00640900200010014038B5094C094D94F8D4
:104EDC00682095F821309A4208D0FFF78FFF012007
:104EEC00FFF722FC95F8213084F8683038BD00BFFC
:104EFC0094010020D00300202DE9F04190B005F082
:104F0C0021FA554C0646E36EC31A002BB8BF5B4220
:104F1C00B3F57A7F0DDB0025206F04F02FFA606F5C
:104F2C00256704F031FAA06F656704F033FAE66682
:104F3C00A5674A4A484B1168494A186F12690029FB
:104F4C00B8BF49420130002AB8BF5242914218679B
:104F5C0003DC102004F0DEFA02E0102004F0E2FA88
:104F6C00FFF7B2FF3E4DFFF7FFFDFFF739FE3D4B5C
:104F7C00AA6919689142C0F0B680374C0021A26F23
:104F8C004FF4004001321960A26704F0D3FA0128F3
:104F9C0034D14FF4806004F0CDFA01282ED1A16BEE
:104FAC00314BE26B284603F049FD304B186004F09E
:104FBC0031FA60B104F09CFA022808D1A26BE36BC1
:104FCC000E920F930EAB93E8030004F03FFA224AC3
:104FDC00234B906BD16BDA68411A0029B8BF494258
:104FEC0091420BDC1D4A9B681268002AB8BF5242E2
:104FFC009A4203DC4FF4804004F08CFA184C94F87D
:10500C002030012B38D14FF4806004F093FA012842
:10501C000DD1114A1649D36B956B144A2046126870
:10502C00009503F015F90AF05FFD124B18604FF470
:10503C00007004F07FFA012829D10E4C20680AF088
:10504C006DFF0A4B01461A68054803F0CBF80AF0CD
:10505C004BFD20601BE000BF9401002030090020B4
:10506C00D0030020800900204C0900207C0900207E
:10507C00F808002060090020924B216818680A4645
:10508C00494206F019FD0AF02FFD8F4B18604FF4C2
:10509C00007004F04FFA012805D04FF4806004F042
:1050AC0049FA01281FD1884D884C28680AF036FF30
:1050BC0026680146864B3246864803F073FC864BC5
:1050CC00186004F0A7F970B104F012FA01280AD1A3
:1050DC0028680AF023FF23680E900F930EAB93E819
:1050EC00030004F0B3F97D4E7A4B3168DA699142D2
:1050FC00C0F060817A4F9A8D7B6F4FF0000EC6F82E
:10510C0000E003F1010C3E26C7F874C00AAC00960F
:10511C00744D06F5D276C8214B23204601964FF4E8
:10512C000266029602F004FF94E8070085E8070087
:10513C004FF4806004F0FEF901280BD04FF400709E
:10514C0004F0F8F9012805D04FF4006004F0F2F9EE
:10515C00012840D15D4B624DD3F80080614A594B18
:10516C0005F17C0E6F4607CAD3F800C087E807002C
:10517C00CDF810E0DFF888E1574ECDF814E0DFF8F9
:10518C0048E1534B53485849584A594CCDF818E00C
:10519C00CDF81CC0CDF82080039603F039F9B5F991
:1051AC007C20B5F97E103368524D89182068102286
:1051BC002B6006F0A1FC206004F02CF958B104F02F
:1051CC0097F940B923682A680F930E920EAB93E8B7
:1051DC00030004F03BF9464B3E4D1868294605F098
:1051EC008BFA05F0C3FA2B6E984228D905F0AAF871
:1051FC003B4CD4F88030C31A002BB8BF5B42B3F5DC
:10520C007A7F1CDB05F070FA4FF4003004F082F961
:10521C0095F86C3063B9384B29461868012201F8AF
:10522C006C2F6C3004F010FA05F08CF8C4F8840084
:10523C0005F0AEFA05F086F8294BC3F8800005F0AE
:10524C0081F8274B2349D3F884204B6E821A002A0D
:10525C00B8BF52429A420BD391F86C20012A07D165
:10526C00254B1868002301F86C3F6C3004F0ECF906
:10527C00184B93F86C30012B03D14FF4003004F031
:10528C0049F94FF4003004F055F9012808D11048C1
:10529C0003F0F4FB194803F0F1FB0020FFF7F0FAE0
:1052AC0002F01EFE124B1A680A4B002A5B68B8BF4C
:1052BC0052429A4226DD012004F02CF902F02CFB1C
:1052CC0025E000BF7C090020600900203009002087
:1052DC0014090020D00300203C09002010090020F4
:1052EC00940100204009002064090020FC080020E3
:1052FC003809002028090020040000204C09002057
:10530C00F8080020012004F00DF902F00DFB2B4BE6
:10531C0093F8222012F0010F22D0294A1268002A99
:10532C001EDD93F8233013F0010F03D0002002F0A0
:10533C0013FB40B9214B93F8230010F001000FD15F
:10534C0002F00AFB60B90220FFF7C0F810B11D4B48
:10535C000022DA630020FFF7E3FA1B4B00221A60ED
:10536C00164B93F8222012F0020F23D0144A126825
:10537C00002A1FDA93F8233013F0020F03D0012018
:10538C0002F0EAFA48B90D4B93F8233013F0020FF0
:10539C0010D1012002F0E0FA60B90220FFF796F874
:1053AC0010B1084B0022DA630020FFF7B9FA064B64
:1053BC0000221A6010B0BDE8F08100BFD0030020BD
:1053CC003009002094010020600900200A4938B5FA
:1053DC00CC6B00238C630949094D0B6009490022F1
:1053EC000A602A60084A094D01202B601360FFF700
:1053FC009BF9FFF703FD38BD940100207C090020C8
:10540C0060090020F8080020280900203C09002031
:10541C0010B5104B5B788BB90F4A012091780F4A6D
:10542C0014680F4A10700F4A11700133E21812F809
:10543C00011C0C4A082B9954F7D10AE0012B08D116
:10544C00094B05221A710132DA7158329A71022213
:10545C005A7110BD58030020C804002024000020FD
:10546C00C0030020C4030020B8040020044B5A6879
:10547C0040F2D2439A4202D1024B01221A70704779
:10548C00580300208409002010B51C4A1C4B1168DD
:10549C0001EA03031B498B422ED152681A4B9A42E4
:1054AC002AD102F0EDF9194B1B78012B10D103F026
:1054BC009FFE04F047FF044601E002F011FA04F0ED
:1054CC0041FF001B0028B8BF4042B0F57A7FF4DBE7
:1054DC0004F056F809F032F8002008F0B7FC00216F
:1054EC000B4809F04BFC0A4809F0A8FB09480AF0E4
:1054FC004FF9002004F04EF810BD00BF58030020F7
:10550C0000FFFF0000819200D6C5B4A31800002054
:10551C00080002400024014010B5164B9A78012A6D
:10552C0008D003D3022A144C0FD109E0587802F0AA
:10553C0013FA02E0587802F07BFA0F4B586006E041
:10554C00587802F019FA606001E0042323700B4BC9
:10555C001B786BB1084B0A495A680A4B0A601AB996
:10556C001A6842F0080202E01A6822F008021A6077
:10557C0010BD00BF58030020B80400209C0400207C
:10558C00BC0300206003002008B5104B9A78012A58
:10559C0002D0022A16D10CE05A7842B9586810B9D8
:1055AC0003F0F0FF11E0104603F0F0FF0DE00322D2
:1055BC0009E05A68587812B902F0BEF905E002F019
:1055CC00C3F902E00422024B1A7008BD58030020F4
:1055DC00B804002008B50B4B9A78022A0ED15B78E0
:1055EC00372B09D89B00084903F5E260C9180A302B
:1055FC00023204F005F804E0032200E00422034B1D
:10560C001A7008BD58030020F4040020B8040020D0
:10561C00144A00231360144A10B51360134A136024
:10562C00134A1360134A1370134A00219950043320
:10563C00B3F5806FF8D1114B1B7E63B940F21A742D
:10564C000F4920460919042203F0DAFF043440F212
:10565C00FA739C42F4D1094A0A4B527D02B10122E1
:10566C001A7010BD64040020BC030020F00400205C
:10567C006003002054030020F4040020C804002020
:10568C00DAFDFF1FA404002008B50B4B9A78022A00
:10569C000ED15B78372B09D89B00084903F5E260E3
:1056AC00C9180A30023203F0CFFF04E0032200E0F5
:1056BC000422034B1A7008BD58030020F404002088
:1056CC00B804002008B5604B9A781AB1022A40F051
:1056DC00A68099E05B78502B69D020D8452B51D00F
:1056EC000ED8422B44D005D8402B38D0412B40F05B
:1056FC0089803BE0432B3FD0442B40F083803EE03D
:10570C00492B48D004D8462B3FD0472B7AD13FE0C9
:10571C004C2B46D04D2B47D04B2B73D13EE0812BDD
:10572C0059D00ED8532B4BD004D8512B42D0522BDE
:10573C0068D142E05A2B49D0802B4AD0552B61D1ED
:10574C0041E0842B52D004D8822B4BD0832B59D1DF
:10575C004AE0FE2B4DD04FD8F02B53D149E03B4BB8
:10576C00186803F0EFFF3A4B58605BE0394B41E0AF
:10577C00384B5A78364B4EE0364B1A79FAE7354BA4
:10578C00DA69F7E7334B5A79F4E7324BDA68F1E729
:10579C00304B9A68EEE72F4BDA7D2FE02D4BDA7801
:1057AC00E8E72C4B9A78E5E72A4B5A7DE2E7294B40
:1057BC009A7DDFE7274B1A7DDCE7264B1A6AD9E77F
:1057CC00244B1A69D6E7234B1A7ED3E7214B5A6A2E
:1057DC00D0E7214B0EE0204B1A78042A14BF00228C
:1057EC000122C7E71D4B02E01D4B00E01D4B1A6860
:1057FC00C0E71D4B1A78BDE71C4B1A78003A18BF4E
:10580C000122B7E703220BE05A78114B372A04D850
:10581C00174951F822205A6004E0032201E00422C7
:10582C000B4B1A70134B1B786BB1094B12495A680E
:10583C00124B0A601AB91A6842F0080202E01A68A0
:10584C0022F008021A6008BD580300200C0000204A
:10585C00B8040020C8040020A40400206404002024
:10586C008C09002088090020B0040020940400203A
:10587C00F40400209C040020BC03002060030020E2
:10588C0010B5884B9A781AB1022A40F01D81FEE0BF
:10589C005A784C2A00F09C801ED8442A5ED00CD832
:1058AC00412A42D003D8402A40F0F98039E0422AFC
:1058BC0044D0432A40F0F38048E0472A66D005D80C
:1058CC00452A53D0462A40F0EA8057E0492A65D051
:1058DC004B2A40F0E4806EE0532A00F0AD800ED8E5
:1058EC00502A00F0858003D84D2A40F0D88077E00C
:1058FC00512A00F08580522A40F0D18094E0832A0E
:10590C0000F0B98006D8552A00F09E805A2A40F043
:10591C00C680A5E0842A00F0B280FF2A40F0BF8048
:10592C00B2E01979604B186805E0604A1B79106881
:10593C005F4A1946137003F01DFFC8E05B4A1B79E0
:10594C0010685B4A013019465370F4E7574A1B79CB
:10595C001068574A043019461371ECE7534A5B68D8
:10596C00106853491C3041F81C3F80E04F4A1B79AA
:10597C0010684F4A053019465371DCE74B4A5B6897
:10598C0010684B490C3041F80C3F70E0474A5B689B
:10599C0010684749083041F8083F68E01A79444BD1
:1059AC0012B1444901224A60DA75404B1868404BE9
:1059BC001730D97DBFE73D4A1B7910683C4C03304A
:1059CC001946E37003F0D6FEE07803F073F87EE03E
:1059DC00364A1B791068364A023019469370AAE78A
:1059EC00324A1B791068324A153019465375A2E7B2
:1059FC002E4A1B7910682E4A1630194693759AE771
:105A0C002B4A127D12F0010F05D01B7913F0010FF8
:105A1C0001D103F067FF254A224B10681B79244AF9
:105A2C0014301946137586E7204A5B6810682049C4
:105A3C00203041F8203F1AE01C4A5B6810681C4972
:105A4C00103041F8103F12E05A68012A3CD8174A2E
:105A5C001B7910681649183001F8183F012207E02D
:105A6C00124A5B6810681249243041F8243F042222
:105A7C0003F0EAFD2BE00F4B5A680F4B02E00D4B85
:105A8C005A680E4B1A6022E01A790D4B1EE05A78B8
:105A9C00372A04D859680B4B43F8221017E003221D
:105AAC0013E000BF580300200C00002090010020E0
:105ABC00C8040020B80400208C09002088090020AC
:105ACC0094040020F40400200422014B1A7010BD31
:105ADC00B804002008B50020FEF722FF08BD00BF67
:105AEC0008B5024B5868FEF71BFF08BD5803002091
:105AFC0008B5034B58684042FEF712FF08BD00BFC3
:105B0C005803002008B5AF4B9A78002A41F00F815A
:105B1C005A78AD2A00F02E856FD81E2A00F0C38269
:105B2C0030D8092A00F0B38113D8032A00F01E8163
:105B3C0005D8012A00F0EF8000F2FB80DDE0062A98
:105B4C0000F04C81072A00F07681042A41F0ED80A8
:105B5C0012E1192A00F0248208D80B2A00F0EE81F9
:105B6C00C0F0C0810D2A41F0E08013E21B2A00F046
:105B7C005E82C0F038821C2A00F05F821D2A41F040
:105B8C00D48089E29C2A00F059831CD8922A00F018
:105B9C00FA8209D8852A00F0A082862A00F0C882F1
:105BAC001F2A41F0C28091E2972A00F0218303D88A
:105BBC00962A41F0BA8015E3982A00F01F839B2A9D
:105BCC0041F0B38020E3A32A00F0EC8308D8A12A8B
:105BDC0000F06B8300F29E839F2A41F0A68033E392
:105BEC00A52A00F04184C0F01184A62A00F06A8432
:105BFC00AC2A41F09A8000F093BCE22A00F0FA85BE
:105C0C003BD8C42A00F09A851BD8BF2A00F05085D7
:105C1C000AD8B22A00F01585BE2A00F03B85B12ABD
:105C2C0041F0838000F0CDBCC12A00F05D85C0F04E
:105C3C004D85C22A00F06685C32A41F0768000F0BB
:105C4C006FBDC82A00F0B28506D8C62A00F092852E
:105C5C0000F29E8500F080BDD22A00F0B58504D8F4
:105C6C00C92A41F0628000F0A8BDD32A00F0B385A8
:105C7C00D42A41F05A8000F0B5BDF12A00F0CE864E
:105C8C001FD8EA2A00F0F3850AD8E52A00F0C0856F
:105C9C00E62A00F0C485E42A41F0478000F0B1BD4B
:105CAC00EE2A00F0438604D8EB2A41F03E8000F047
:105CBC0015BEEF2A00F06286F02A41F0368000F023
:105CCC0085BEFA2A00F068870AD8F52A00F0FC860F
:105CDC00F92A00F03787F42A41F0278000F0C9BE7A
:105CEC00FC2A00F0A787C0F07F87FD2A00F0CB8745
:105CFC00FE2A41F01A8000F0EFBF052805D1314B88
:105D0C005868FEF7D3FD01F029B8062841F026802B
:105D1C00FEF78EFB26E0052805D12A4B5868FEF7C6
:105D2C0057FD01F01BB8062841F01880FEF78EFBDA
:105D3C0018E0052811D1234B234A586800F542334B
:105D4C0003F5A863934203D8FEF7EAFD01F006B809
:105D5C001E4B04221A7001F001B8062840F0FE8791
:105D6C00FEF77AFB194B586000F0E6BF062840F0AE
:105D7C00F587FEF777FBF5E705280AD1114B144997
:105D8C005B688B4295BF134A104B13601A7000F07E
:105D9C00E5BF062802D10F4B1A686BE2072806D123
:105DAC000D4B0C49186803F04FFC00F0D7BF0828C6
:105DBC0040F0D487084B0749186803F021FC00F029
:105DCC00CDBF00BF58030020801A0600B804002085
:105DDC00400D0300D00300200400002005280ED144
:105DEC009A4B44F620625B68934203D8984A5360FE
:105DFC0000F0B4BF974B04221A7000F0AFBF062816
:105E0C0002D1934B5A6835E2072808D1924B0422F1
:105E1C0018689249801803F017FC00F09FBF0828FF
:105E2C0040F09C878C4B042218688C49801803F036
:105E3C00E7FB00F093BF05280DD1844B884A5B68C3
:105E4C00934203D8824A936000F088BF814B0422AE
:105E5C001A7000F083BF062802D17D4B9A6809E2C4
:105E6C00072808D17C4B7F4918680422083003F0BE
:105E7C00EBFB00F073BF082840F07087764B794934
:105E8C0018680422083003F0BBFB00F067BF05283C
:105E9C000CD15B68724A934203D86D4A136100F0CF
:105EAC005DBF6C4B04221A7000F058BF062802D15B
:105EBC00674B1A69DEE1072808D1674B6A491868F5
:105ECC000422103003F0C0FB00F048BF082840F05B
:105EDC004587614B644918680422103003F090FB2D
:105EEC0000F03CBF05280DD1584B604A5B689342CB
:105EFC0003D8574AD36000F031BF564B04221A70B6
:105F0C0000F02CBF062802D1514BDA68B2E1072809
:105F1C0008D1514B5649186804220C3003F094FBFD
:105F2C0000F01CBF082840F019874B4B50491868EB
:105F3C0004220C3003F064FB00F010BF05280DD1D7
:105F4C00424B4A4A5B68934203D8414A536100F082
:105F5C0005BF404B04221A7000F000BF062802D186
:105F6C003B4B5A6986E1072808D13B4B41491868DD
:105F7C000422143003F068FB00F0F0BE082840F057
:105F8C00ED86354B3B4918680422143003F038FB7E
:105F9C0000F0E4BE062840F0E186FEF74FFAE1E699
:105FAC00052804D15A682A4B5A6600F0D7BE062839
:105FBC0002D1274B5A6E5DE1072808D1264B2E499A
:105FCC0018680422643003F03FFB00F0C7BE0828B9
:105FDC0040F0C486204B284918680422643003F032
:105FEC000FFB00F0BBBE052805D1184B5A68184BA7
:105FFC001A6600F0B3BE062802D1154B1A6E39E1B1
:10600C00072808D1144B1D4918680422603003F08E
:10601C001BFB00F0A3BE082840F0A0860E4B1749CE
:10602C0018680422603003F0EBFA00F097BE0628E3
:10603C0040F0948604F09AFB94E6052820D1034B9B
:10604C00586804F09FFB00F089BE00BF5803002085
:10605C00D0030020B804002004000020D40300204A
:10606C00400D0300D8030020E0030020A0860100AF
:10607C00DC030020E4030020340400203004002062
:10608C00062802D104F078FB6CE6072840F06686FF
:10609C0004F07EFB00F062BE052840F04B86FEF754
:1060AC005DFA00F05BBE052804D1586804F09AFB39
:1060BC0000F054BE062802D104F08EFB52E60728ED
:1060CC0040F04C8604F094FB00F048BE052840F0EC
:1060DC003186FFF77BF900F041BE05280CD1A24BAD
:1060EC005B680A2B03D8A14A936100F037BEA04B22
:1060FC0004221A7000F032BE062802D19B4B9A691A
:10610C00B8E0072808D19B4B9B491868042218302B
:10611C0003F09AFA00F022BE082840F01F86954B37
:10612C00954918680422183003F06AFA00F016BE7C
:10613C0005280CD18C4B5B680A2B03D88B4AD36196
:10614C0000F00CBE8A4B04221A7000F007BE062821
:10615C0002D1864BDA698DE0072808D1854B874937
:10616C00186804221C3003F06FFA00F0F7BD082801
:10617C0040F0F4857F4B8149186804221C3003F0F1
:10618C003FFA00F0EBBD05280ED15B68012B06D859
:10619C00754B1A79754B83F8202000F0DFBD744BDA
:1061AC0004221A7000F0DABD062804D16F4B93F864
:1061BC00202000F0A1BD072808D16E4B704918684B
:1061CC000122203003F040FA00F0C8BD082840F04E
:1061DC00C585684B6A4918680122203003F010FA13
:1061EC0000F0BCBD062840F0B985FEF741F9B9E5D1
:1061FC00062840F0B385FEF709F9B3E5062840F010
:10620C00AD85FEF709F9ADE5052811D1564B49F6D8
:10621C004042586800F59C432033934203D8FEF764
:10622C002FFB00F09BBD524B04221A7000F096BD60
:10623C00062840F09385FEF7F5F893E5062840F024
:10624C008D8503F087F98DE505280ED1464B5B68EB
:10625C009A1F022A04D8454A82F8213000F07EBDEC
:10626C00434B04221A7000F079BD062806D13F4B2F
:10627C0093F821203E4B5A6000F05EBD072808D1F0
:10628C003C4B404918680122213003F0DDF900F045
:10629C0065BD082840F06285364B3A4918680122E2
:1062AC00213003F0ADF900F059BD052813D12E4A69
:1062BC002E4B52683AB193F85D2042F0010283F8FC
:1062CC005D2000F04BBD93F85D2022F0010283F8B5
:1062DC005D2000F043BD062805D1244B93F85D20CA
:1062EC0002F00102C6E7072808D1224B264918689C
:1062FC0001225D3003F0A8F900F030BD082840F011
:10630C002D851C4B2049186801225D3003F078F96B
:10631C0000F024BD052813D1134A144B52683AB12E
:10632C0093F85D2042F0020283F85D2000F016BD68
:10633C0093F85D2022F0020283F85D2000F00EBD80
:10634C00062805D1094B93F85D20C2F3400291E772
:10635C0007281BD1074B0C49186801225D3003F04C
:10636C0073F900F0FBBC00BF58030020D0030020E1
:10637C00B804002004000020E8030020EC030020F7
:10638C00F0030020F10300202D040020082840F029
:10639C00E5849B4B9B49186801225D3003F030F972
:1063AC0000F0DCBC052812D15A68974B3AB193F82F
:1063BC005D2042F0040283F85D2000F0CFBC93F81E
:1063CC005D2022F0040283F85D2000F0C7BC062893
:1063DC0005D18D4B93F85D20C2F380024AE7072864
:1063EC0008D1874B8749186801225D3003F02CF9DE
:1063FC0000F0B4BC082840F0B184814B8149186886
:10640C0001225D3003F0FCF800F0A8BC05280ED189
:10641C007E4B5A68032A05D81A797B4B83F82220C5
:10642C0000F09CBC7A4B04221A7000F097BC062832
:10643C0003D1754B93F822201CE7072808D1704B29
:10644C00744918680122223003F0FEF800F086BC73
:10645C00082840F083846A4B6E4918680122223068
:10646C0003F0CEF800F07ABC05280ED1674B5B68C0
:10647C00B3F5803F04D2644AA2F8443000F06EBCFD
:10648C00634B04221A7000F069BC062803D15E4BE2
:10649C00B3F84420EEE6072808D1594B5E4918683A
:1064AC000222443003F0D0F800F058BC082840F029
:1064BC005584534B584918680222443003F0A0F815
:1064CC0000F04CBC05280ED1504B5A68032A05D855
:1064DC001A794D4B83F8232000F040BC4C4B04221E
:1064EC001A7000F03BBC062803D1474B93F82320CD
:1064FC00C0E6072808D1424B4849186801222330CE
:10650C0003F0A2F800F02ABC082840F027843C4B8A
:10651C00424918680122233003F072F800F01EBCC7
:10652C0005280DD1394B5B68B3F5803F03D2364A51
:10653C00536300F013BC364B04221A7000F00EBCEF
:10654C00062802D1304B5A6B94E6072807D12C4B06
:10655C00334918680422343003F076F8FEE3082837
:10656C0040F0FC83264B2E4918680422343003F08B
:10657C0047F8F3E305280AD15B68B3F5803F02D2F4
:10658C00214A9363EAE3224B04221A70E6E30628BD
:10659C0002D11D4B9A6B6DE6072807D1184B214988
:1065AC0018680422383003F04FF8D7E3082840F07D
:1065BC00D583134B1B4918680422383003F020F89C
:1065CC00CCE305280CD1114B44F620625B68934256
:1065DC0002D80D4AD363C1E30D4B04221A70BDE3FC
:1065EC00062802D1084BDA6B44E607281ED1044B6F
:1065FC000D49186804223C3003F026F8AEE300BFC6
:10660C00040000202D040020D0030020580300209B
:10661C00B8040020F203002014040020F30300202F
:10662C0004040020080400200C040020082840F07A
:10663C009583A24BA249186804223C3002F0E0FF7B
:10664C008CE305280BD19F4B5B68012B03D89E4A2A
:10665C0082F86D3082E39D4B04221A707EE306288B
:10666C0003D1994B93F86D2004E6072807D1934B7F
:10667C009749186801226D3002F0E6FF6EE3082896
:10668C0040F06C838D4B9249186801226D3002F0FA
:10669C00B7FF63E3052804D18C4B586802F06EFEFB
:1066AC005CE3062840F05A8302F02CFEFFF75ABB3D
:1066BC00052804D1854B586802F066FE4EE3062887
:1066CC0040F04C8302F024FEFFF74CBB052804D1AC
:1066DC007E4B586802F05EFE40E3062840F03E8395
:1066EC0002F01CFEFFF73EBB052804D1774B58681F
:1066FC0002F056FE32E3062840F0308302F014FE1E
:10670C00FFF730BB052804D1704B586802F04EFEE1
:10671C0024E3062840F0228302F00CFEFFF722BB94
:10672C00052804D1694B586802F046FE16E306288A
:10673C0040F0148302F004FEFFF714BB052804D1CB
:10674C00624B586802F03EFE08E3062840F00683D0
:10675C0002F0FCFDFFF706BB052804D15B4B586823
:10676C0002F036FEFAE2062840F0F88202F0F4FD60
:10677C00FFF7F8BA052804D1544B586802F02EFEE6
:10678C00ECE2062840F0EA8202F0ECFDFFF7EABAF0
:10679C00052804D14D4B586802F026FEDEE206288F
:1067AC0040F0DC8202F0E4FDFFF7DCBA062840F092
:1067BC00D582FDF7A7FEFFF7D5BA062840F0CE82AA
:1067CC00FDF7A6FEFFF7CEBA062840F0C782FDF70C
:1067DC00BBFEFFF7C7BA062840F0C082FDF7B0FE3B
:1067EC00FFF7C0BA062840F0B98201F0D3FD00B221
:1067FC00FFF7B8BA062840F0B182FDF771FEFFF73B
:10680C00B1BA062840F0AA82FDF770FEFFF7AABACB
:10681C00062840F0A382FDF76FFEFFF7A3BA052808
:10682C000BD1284B5B68B3F5803F02D2264A136527
:10683C0094E2264B04221A7090E2062802D1224BD5
:10684C001A6D17E5072807D11C4B2249186804223A
:10685C00503002F0F9FE81E2082840F07F82174B9D
:10686C001C4918680422503002F0CAFE76E2052852
:10687C000AD15B68B3F5803F02D2134A53656DE2CF
:10688C00124B04221A7069E2062802D10E4B5A6D83
:10689C00F0E4072807D1094B0F491868042254303B
:1068AC0002F0D2FE5AE2082840F05882034B0A4903
:1068BC0018680422543002F0A3FE4FE204000020BA
:1068CC000C04002058030020D0030020B804002042
:1068DC003D040020200400202404002005280BD1B6
:1068EC008C4B5B68B3F5803F02D28B4A936535E2E3
:1068FC008A4B04221A7031E2062802D1864B9A6D1B
:10690C00B8E4072807D1864B86491868042258300A
:10691C0002F09AFE22E2082840F02082804B814946
:10692C0018680422583002F06BFE17E205280BD1D0
:10693C00784B5B68B3F5803F02D2774A93620DE2E5
:10694C00764B04221A7009E2062802D1724B9A6A1D
:10695C0090E4072807D1724B734918680422283039
:10696C0002F072FEFAE1082840F0F8816C4B6E4997
:10697C0018680422283002F043FEEFE105280BD101
:10698C00644B5B68B3F5803F02D2634A9364E5E1E4
:10699C00624B04221A70E1E1062802D15E4B9A6C1C
:1069AC0068E4072807D15E4B604918680422483018
:1069BC0002F04AFED2E1082840F0D081584B5B49E6
:1069CC0018680422483002F01BFEC7E105280BD1E1
:1069DC00504B5B68B3F5803F02D24F4AD364BDE1A4
:1069EC004E4B04221A70B9E1062802D14A4BDA6CDC
:1069FC0040E4072807D14A4B4D49186804224C3013
:106A0C0002F022FEAAE1082840F0A881444B484934
:106A1C00186804224C3002F0F3FD9FE105280ED1DA
:106A2C005A68444902F5423303F5A8638B4202D8F5
:106A3C00394B9A6692E1394B04221A708EE1062882
:106A4C0002D1354B9A6E15E4072807D1344B3A49DD
:106A5C0018680422683002F0F7FD7FE1082840F046
:106A6C007D812F4B344918680422683002F0C8FD30
:106A7C0074E105280CD1274B42F210725B689342EB
:106A8C0002D8254AD38469E1244B04221A7065E1AB
:106A9C00062804D1204BB3F92620FFF7EBBB0728BF
:106AAC0007D11F4B254918680222263002F0CCFD75
:106ABC0054E1082840F05281194B204918680222F1
:106ACC00263002F09DFD49E1052808D1114B5A688A
:106ADC00114B003A18BF012283F82F203EE1062803
:106AEC0003D10D4B93F82F2006E1072807D10C4B4F
:106AFC001349186801222F3002F0A6FD2EE1082858
:106B0C0040F02C81064B0E49186801222F3002F000
:106B1C0077FD23E158030020D0030020B8040020A7
:106B2C000400002028040020F80300201804002092
:106B3C001C040020801A060038040020F6030020F4
:106B4C00FF03002005280BD1854B5B68022B03D873
:106B5C00844A82F82E3001E1834B04221A70FDE046
:106B6C00062804D17F4B93F82E20FFF783BB072810
:106B7C0007D17E4B7E49186801222E3002F064FD4D
:106B8C00ECE0082840F0EA80784B7949186801223B
:106B9C002E3002F035FDE1E005280AD15B68B3F533
:106BAC00803F02D26F4A1364D8E06F4B04221A70F4
:106BBC00D4E0062803D16B4B1A6CFFF75BBB07289C
:106BCC0007D16A4B6B4918680422403002F03CFD37
:106BDC00C4E0082840F0C280644B6649186804225F
:106BEC00403002F00DFDB9E0052808D15C4B5A6825
:106BFC005C4B003A18BF012283F83020AEE0062827
:106C0C0003D1584B93F8302076E0072807D1574B27
:106C1C00594918680122303002F016FD9EE0082810
:106C2C0040F09C80514B544918680122303002F0DE
:106C3C00E7FC93E005280BD1494B5B68012B03D88B
:106C4C00484A82F8313089E0474B04221A7085E0BB
:106C5C00062804D1434B93F83120FFF70BBB0728D0
:106C6C0007D1424B454918680122313002F0ECFC47
:106C7C0074E0082872D13D4B40491868012231302C
:106C8C0002F0BEFC6AE005280BD1354B5868831E18
:106C9C00FC2B02D8FDF7FAFF60E0334B04221A708C
:106CAC005CE0062804D12F4B93F82520FFF7E2BABD
:106CBC00072807D12D4B324918680122253002F0E4
:106CCC00C3FC4BE0082849D1284B2D4918680122F8
:106CDC00253002F095FC41E0052808D1204B5A687C
:106CEC00204B003A18BF012283F8242036E00628F6
:106CFC0007D11C4B93F82420003A18BF0122FFF750
:106D0C00B9BA072807D1194B1E491868012224303B
:106D1C0002F09AFC22E0082820D1144B194918687B
:106D2C000122243002F06CFC18E0032200E0042263
:106D3C000D4B1A70062811D1134B1B7873B10A4BEB
:106D4C0012495A68124B0A6022B91A6842F00802BA
:106D5C001A6003E01A6822F008021A6008BD00BF2E
:106D6C0058030020D0030020B804002004000020A9
:106D7C00FE03002010040020000400200104002069
:106D8C00F5030020F40300209C040020BC03002029
:106D9C006003002008B5204B997811B15B78032B68
:106DAC0036D11D4B5B780A2B30D8DFE803F006098F
:106DBC000C0F14171A1D22252A0002F06FFB22E07B
:106DCC0002F068FB1FE002F06DFB1CE0124B5868F0
:106DDC0002F06AFB17E002F00DFB1CE002F012FB64
:106DEC0019E002F017FB0EE00B4B586802F070FB39
:106DFC0011E002F07DFB06E0074B586802F07EFBC9
:106E0C0009E002F081FB054B586004E0032200E02E
:106E1C000422024B1A7008BD58030020B80400204D
:106E2C0008B50B4B9A7872B95A7812B1012A08D16D
:106E3C0003E05868FDF73AFD08E05868FDF766FD79
:106E4C0004E0032200E00422024B1A7008BD00BFCC
:106E5C0058030020B804002010B5A94AA94B10789B
:106E6C0051686422232859601A70587000F0F6801B
:106E7C0053D8132800F0CB8028D8082811D805281F
:106E8C0080F0B080022800F0A48003D8012840F0E4
:106E9C0049819BE0032800F09F80042840F0428148
:106EAC009DE00B2800F0A78006D8092800F09D80F3
:106EBC000A2840F037819BE00E2800F0A2800F28B2
:106ECC0000F0A2800C2840F02D8197E01B2800F0E8
:106EDC00B08011D8162800F0A38006D8142800F032
:106EEC009980152840F01E8197E0172800F09B80B0
:106EFC00182840F0178199E01F2800F0A38006D8CD
:106F0C001C2800F099801E2840F00C8197E0212865
:106F1C0000F09E8000F29F8097E0822800F0C580F0
:106F2C0029D8432800F0AC8011D8402800F09F806D
:106F3C0006D8242800F09580272840F0F38093E0B1
:106F4C00412800F09780422840F0EC8095E04628DC
:106F5C0000F09F8006D8442800F09580452840F02A
:106F6C00E18093E0802800F09A8000F29B80472813
:106F7C0040F0D88090E0882800F0B68011D88528A1
:106F8C0000F0A48006D8832800F09280842840F07A
:106F9C00C98090E0862800F0A180872840F0C2804C
:106FAC00A5E08D2800F0B28006D8892800F0A280D8
:106FBC008C2840F0B780A0E0F22800F0AD80FF28CC
:106FCC0000F0AD808E2840F0AD80A2E0FEF788FD89
:106FDC00ABE0FEF78DFDA8E0FEF77CFDA5E0FFF72A
:106FEC001FFFA2E0FEF78EFD9FE0FEF749FC9CE040
:106FFC00FEF768FB99E0FEF747FB96E0FEF7EAFA2E
:10700C0093E0FEF7C1FA90E0FEF786FA8DE002F00D
:10701C00D5FD8AE002F0B0FE87E002F03BFF84E091
:10702C0002F02EFF81E002F08FFF7EE002F0A4FF61
:10703C007BE003F01BF878E002F0B0FF75E002F0A3
:10704C00B3FF72E002F0C8FF6FE002F0F5FF6CE0F6
:10705C0002F008FE69E003F02DF966E003F01EF97A
:10706C0063E002F05DFE60E002F002FD5DE000F026
:10707C005FFB5AE000F05EFB57E000F05DFB54E074
:10708C0000F05CFB51E000F05BFB4EE000F05AFBC3
:10709C004BE000F059FB48E000F058FB45E002F0F3
:1070AC0037FD42E002F0FEFC3FE002F00DFD3CE05B
:1070BC0002F010FD39E000F0E3FB134B1C7D02F0F5
:1070CC0049FA0146204602F083FE2EE002F09CFEB7
:1070DC0000F0CEFB0020FDF7D3FB26E00A4B197D18
:1070EC00987803F079F820E0FEF792F91DE002F0B1
:1070FC0091FE1AE003F0B6F817E003F041F814E043
:10710C0058030020B8040020C804002002F006FD3B
:10711C000BE0FFF73FFE08E0FEF7B6F905E0FEF7DF
:10712C00A5F902E0014B02221A7010BDB804002030
:10713C002DE9F04F764B8BB01B78044663B1754B41
:10714C001B78062B08D00A2B06D00F2B04D01F2B34
:10715C0002D0714B00221A70704B1B78012B48D156
:10716C006D4B1A78511EC9B2012942D858786C4916
:10717C006C4BCD681B78012A0CBF4FF0070C4FF0FD
:10718C00080C002201958DF800C08DF801008DF8D7
:10719C000220D3B9644A8E681578117992F801E00F
:1071AC0092F807C0907952798DF808608DF80950E3
:1071BC008DF80AE08DF80BC08DF80C008DF80D20C1
:1071CC008DF80E108DF80F300DE0012B09D1574BB7
:1071DC000132D15C0AA88318082A03F8211CF6D1C5
:1071EC0001E0022B05D0684604F07EF8002800F080
:1071FC003F824F4B1B78012B4CD1474A1278032A04
:10720C0020D1484B1B7893B9454E474DB0787778D1
:10721C002A786B78C719BF18EA79FF18AB79BF18B1
:10722C006A79FF182B79BF18FF18FFB218E0012BF1
:10723C0030D100253D4BE85C013501F04BFC092DAC
:10724C00F8D127E0042A25D1354E374DB27877781E
:10725C001046D719013700222B706A60FFB26A7092
:10726C0001F038FC707801F035FC287801F032FC24
:10727C00687801F02FFCE87901F02CFCA87901F07A
:10728C0029FC687901F026FC287901F023FC3846AA
:10729C0001F020FC274B1B78012B73D11E4A12786E
:1072AC00072A49D11F4B1B782BBB1D4A1E4B557807
:1072BC00967893F800E093F801C0AF19D879774429
:1072CC00997967445A79C7191B79CF19D719DF19DE
:1072DC008DF818708DF810608DF811508DF812E043
:1072EC008DF813C08DF814008DF815108DF816203C
:1072FC008DF8173009E0012B07D1013B0B4A995C43
:10730C0004AAD1540133092BF8D104A8092137E080
:10731C00940400205803002020020020510000207B
:10732C00C8040020C0030020B8040020C4030020BF
:10733C004E00002018000020082A23D19B499C4AAB
:10734C0091F801C091F802E000250EEB0C06013615
:10735C0004A8092155608DF812308DF813502F4672
:10736C008DF814508DF815508DF816508DF8175067
:10737C008DF81860557013708DF810E08DF811C0F1
:10738C0001F020FE8B4B8C491A7800230B708B4933
:10739C000B7012B1012002F0FDF8894B1D78012D04
:1073AC003CD1684603F020FF002837D09DF8001030
:1073BC00844B9DF808A09DF809809DF80A709DF8F3
:1073CC000B609DF80CC09DF80D009DF80E907B4A4B
:1073DC009DF801B0072983F8049083F800A083F886
:1073EC0001809F70DE7183F806C0587182F801B07D
:1073FC0001D1157001E002231370734B1B785A1ED8
:10740C00D2B2012A05D9052B03D0704B01251D7072
:10741C0005E06E4B00221A70012500E000256C4B34
:10742C001B78012B59D10DF1270001F02DFB002801
:10743C0053D001F045FB10B1604B00229A705F4BAA
:10744C009DF8270099784A1CD2B2C918092A0871EC
:10745C009A7041D1554A18795178002288429A7015
:10746C003AD11346554D291D895C01325B18082A07
:10747C00DBB2F7D12A7B9A422CD1524B697AAA7A89
:10748C00EE7A6F7995F806E095F807C0287A1E71A8
:10749C0099715A711F7083F801E083F802C0D8719A
:1074AC0002F050FF484B4B4E1B783060591E4A4837
:1074BC000022C9B2AA700270033201292A7005D9C0
:1074CC00052B03D0414B01251D7006E03F4B0022DC
:1074DC001A7001E004232B700125404B1B78012B03
:1074EC0049D107A801F056FD002844D02F4B9DF838
:1074FC001C205B789A4276D10022134607A9C95CFE
:10750C0001335218082BD2B2F8D19DF824102B4C11
:10751C0091422ED12B4B9DF821109DF822209DF8E5
:10752C001D609DF81EE09DF81FC09DF820009DF881
:10753C00235099715A711E701D7183F801E083F804
:10754C0002C0D87102F0FEFE1F4B22491B78086066
:10755C005A1E21490020D2B208700721012A21703D
:10756C0003D9052B01D0012200E00022174B1A7021
:10757C0039E0237037E0002D35D113490B78013BEE
:10758C00DBB2012B2FD8012C2DD1154B1A68B2F57B
:10759C00006F27D8104601321A600A4902F026FA09
:1075AC00064B09221A70094B1C701CE0C804002001
:1075BC00B804002084090020C00300202002002011
:1075CC005100002058030020A40400209C0400203B
:1075DC004E000020B4040020C0040020180000203D
:1075EC00640400200D70244B1B78042B04D1234B16
:1075FC0093F90030002B2EDA214B1B783BB1042B76
:10760C0005D0082B03D0062B01D0FFF725FC1C4B13
:10761C001B78092B05D1184A1178022901D10331A5
:10762C001170184A12681AB3092B21D1124B1B780E
:10763C00012B1DD11449013B096809E0134850F88E
:10764C0023000133814203D10B4B05221A700FE04A
:10765C009342F3D30CE0FDF791F9094B1B783BB146
:10766C00042B05D0082B03D0062B01D002F05EFDB5
:10767C000BB0BDE8F08F00BFA4040020580300201D
:10768C0020020020A80400206404002068040020CC
:10769C0073B5204B024640781F4D18709078002629
:1076AC005870D078EC46987010790C46D871507997
:1076BC00987192F806E095E8030083F805E0D2791A
:1076CC008CE803001A71154B1E70FFF7C5FB144BA9
:1076DC001B7873B9637023702B78A3706B78E3708D
:1076EC00EB792371AB7963716B79A3712B79E371AE
:1076FC0008E0012B06D10B4B9B195B78A355013687
:10770C00082EF8D1044B6A4692E8030083E8030084
:10771C007CBD00BF58030020B80400209C0400204E
:10772C00C0030020C4030020704700BF704700BF97
:10773C00704700BF704700BF704700BF704700BF65
:10774C00704700BF704700BF704700BF704700BF55
:10775C000E4B10B50022012002214FF4FA744FF0A9
:10776C00080C5C6283F805C09860D9601A621A70C4
:10777C0058709970DA701A719A711A611A755A7573
:10778C009A75DA751A76DA6110BD00BFC80400204C
:10779C002F4B4FF4FA7CC3F808C04FF4FA6CC3F8C3
:1077AC0014C04FF0020CC3F81CC00CF1040CF0B563
:1077BC0083F821C00CF1020C83F825C00CF1C00C2D
:1077CC004FF47A64C3F868C040F2DC5C00220120FC
:1077DC0005274FF416764FF44875C3F83CC01C646B
:1077EC001C605C60ACF5966C4FF47A741146DA64EC
:1077FC0083F8222083F8232083F824209A629A8528
:10780C0083F83020A3F8442083F846209A641F6143
:10781C009E63C3F850C09D6583F85C00DF6098617F
:10782C0083F82000DC8483F82E0083F82F005E633D
:10783C005D6583F85D2083F83120064A83F86C106F
:10784C001A6643F290325A6683F86D10F0BD00BF91
:10785C00D003002000390300014B10225A617047FD
:10786C0000080140014B10221A61704700080140CA
:10787C00024B4FF400421A61704700BF00100140E8
:10788C00024B4FF400425A61704700BF0010014098
:10789C00024B986800F40040704700BF0010014094
:1078AC00024B4FF480521A61704700BF0010014028
:1078BC00024B4FF480525A61704700BF00100140D8
:1078CC00704700BF704700BF704700BF704700BFD4
:1078DC00704700BF704700BF704700BF704700BFC4
:1078EC00704700BF014B04221A6170470008014029
:1078FC00014B04225A61704700080140054B9A68FD
:10790C0012F0040F02D004225A6101E004221A6121
:10791C00704700BF00080140024B4FF400721A611F
:10792C00704700BF000C0140024B4FF400725A61CB
:10793C00704700BF000C014010B9024B20225A6165
:10794C00704700BF0010014010B9024B20221A6191
:10795C00704700BF0010014018B1012803D000206F
:10796C0005E0034B00E0034B9868C0F380007047C0
:10797C0000140140000C014008B1002003E0024B50
:10798C009868C0F34010704700100140064B1B78FC
:10799C00012B04D1054B4FF480521A6102E0044BC9
:1079AC0001221A70704700BF18000020000C014023
:1079BC0030020020064B1B78012B04D1054B4FF4F1
:1079CC0080525A6102E0044B00221A70704700BFCB
:1079DC0018000020000C014030020020054B1B78E1
:1079EC00012B03D1044B0020DB6801E0034B18781A
:1079FC00704700BF18000020000C0140300200202E
:107A0C00704700BF094B10B59C68C4F382140CB1CD
:107A1C00072C05D1012803D11F3001F07BFD02E0BA
:107A2C00202001F07FFD204610BD00BF000C01405E
:107A3C0008B518B1012804D0002006E0034B5868A3
:107A4C0001E0024B986800F097F908BD180000207F
:107A5C0037B501AD002429464FF01F030848ADF897
:107A6C0004308DF8074006F017FF4FF0030329464A
:107A7C0004488DF80740ADF8043006F00DFF3EBD0C
:107A8C0000100140000C01402DE9F347584E01ADA8
:107A9C0004200121032406F0BFFC102730464FF0D0
:107AAC00BE032946ADF804308DF806408DF80770FA
:107ABC0006F0F2FEAE234FF00408DFF83CA130468E
:107ACC003761294673614FF04103ADF804308DF8EE
:107ADC0006408DF8078006F0DFFE0820012106F035
:107AEC009BFC41F2386350462946ADF804304FF008
:107AFC0020098DF806408DF8077006F0CDFE41F296
:107B0C00182350462946CAF81090CAF8143040F68B
:107B1C00C71306F50066ADF804308DF806408DF8F5
:107B2C00078006F0B9FE3846012106F075FC304698
:107B3C004FF220432946ADF804308DF807708DF8CC
:107B4C00064006F0A9FE4FF4E043336103F5A15360
:107B5C003046736129464FF43C63ADF804308DF820
:107B6C0006408DF8078006F097FE4FF01F03304655
:107B7C0029460026ADF804308DF806408DF80760D4
:107B8C0006F08AFE4846012106F046FC4FF4004000
:107B9C00314606F011FF4823164829468DF8073068
:107BAC00ADF804808DF8064006F076FE304633467C
:107BBC0011494FF480644C610A468968013611F40E
:107BCC00006F4FF480611161926808BF013312F4A9
:107BDC00006F18BF01300A2EEAD10A2B01D0002009
:107BEC0003E00A2814BF00200120BDE8FC8700BF79
:107BFC000008014000140140000C0140704700BF18
:107C0C00FEE700BFFEE700BFFEE700BFFEE700BFD8
:107C1C00704700BF704700BF704700BF704700BF80
:107C2C00704700BF704700BF704700BF704700BF70
:107C3C00704700BF704700BF704700BF704700BF60
:107C4C00704700BF704700BF704700BF704700BF50
:107C5C00704700BF704700BF704700BF704700BF40
:107C6C00704700BF08B5024B1B68984708BD00BFA2
:107C7C006403002008B5024B1B68984708BD00BF81
:107C8C00C4040020684620F00701044B8D4601B562
:107C9C001B689847BDE80140854670479804002052
:107CAC0008B5024B1B68984708BD00BFA004002014
:107CBC00704700BF704700BF704700BF704700BFE0
:107CCC00704700BF704700BF704700BF704700BFD0
:107CDC00704700BF704700BF704700BF704700BFC0
:107CEC00704700BF704700BF704700BF704700BFB0
:107CFC00704700BF704700BF704700BF704700BFA0
:107D0C00704700BF704700BF704700BF704700BF8F
:107D1C00704700BF704700BF704700BF704700BF7F
:107D2C00704700BF704700BF684620F007018D46C2
:107D3C0001B5002303E00B495958995004330A4A02
:107D4C000A4998188842F6D3094B02E0002243F8FE
:107D5C00042B084A9342F9D3FCF740FABDE80140E2
:107D6C0085467047EC0301080000002090010020BC
:107D7C0090010020EC1C0020024B33F8100080B264
:107D8C00704700BF40020020024B03EB40031982F6
:107D9C00704700BF40020020024B03EB4003188ADF
:107DAC00704700BF4002002010B50A4C24781CB963
:107DBC00002914BF0A461A4650214843064B424339
:107DCC0002991878039B002808BF0B4692FBF3F02E
:107DDC0010BD00BF9009002092090020A523434349
:107DEC00044AA3F5A52310684FF48052584390FB26
:107DFC00F2F0704754000020014B1870704700BF20
:107E0C0092090020014B1870704700BF90090020A8
:107E1C00074B10B51B68074C34F8130080B2FFF702
:107E2C00DDFF20220146206A03F066FE206210BDB1
:107E3C003400002040020020F8B5114B114E1B6895
:107E4C00044636F8130080B2FFF7C8FF0E4B054608
:107E5C001B6836F8130080B2FFF7C0FF064605FB1F
:107E6C0005F006FB060077197F4207FB070003F0BD
:107E7C00A9FDA680A060678025802046F8BD00BFC4
:107E8C00340200204002002034000020F8B5114BD1
:107E9C00114E1B68044636F8130080B2FFF79EFFA4
:107EAC000E4B05461B6836F8130080B2FFF796FFA1
:107EBC00064605FB05F006FB060077197F4207FB1B
:107ECC00070003F07FFDA780A06066802580204618
:107EDC00F8BD00BF3402002040020020300000201A
:107EEC0038B5104C257885B1012D1AD10E4B5B6A33
:107EFC00002BB8BF5B42B3F5E16F12DDFFF7D8FC86
:107F0C0000232370094B1D700BE0074B5B6AC733D2
:107F1C00B3F5C77F05D8FFF7C3FC044A01231370E0
:107F2C00237038BD920900204002002091090020E6
:107F3C002DE9F74F534C0025074665625248884699
:107F4C0092469946DDF834B005F0C6FDC8F5E168F7
:107F5C00404501D307241EE04C4B626A1B68002A83
:107F6C0034F8130004EB43010B8A80B2B8BF5242C1
:107F7C00C01A80EAE073A3EBE07393420E9BC8BF78
:107F8C00606251460193CDF800B04A460C9BFFF756
:107F9C000BFF062405463C4805F0A2FD404501D3E5
:107FAC00002621E03A4A374B1268596A33F812001E
:107FBC0003EB4206328A80B2801A81EAE172A2EBAC
:107FCC00E17280EAE071A1EBE0719142C8BF5862A6
:107FDC000E9BCDF800B0019351464A460C9BFFF71F
:107FEC00E3FE24F002040646274805F07DFD4045DB
:107FFC0002D34FF0000822E0264A224B1268596A3D
:10800C0033F8120003EB420CBCF8102080B2801A3B
:10801C0081EAE172A2EBE17280EAE071A1EBE0711E
:10802C009142C8BF58620E9BCDF800B001935146E7
:10803C004A460C9BFFF7B8FE24F004048046022C41
:10804C0007D0042C09D0012C0BD108EB06056D428E
:10805C0007E008EB0506764203E006EB0508C8F1DD
:10806C00000805FB05F006FB060008FB080003F002
:10807C00A9FCA7F80480B8607E803D803846BDE836
:10808C00FE8F00BF40020020002C01403402002073
:10809C00300000203400002070B590B0FFF7D8FC01
:1080AC000120014606F0AAF901214FF4007006F0F8
:1080BC00B3F9414806F0C2FD404B00240093404BFD
:1080CC000726019380230593DB18069303F5407371
:1080DC000793A3F5787338486946089303F5FF5363
:1080EC0009930294039604940A9406F017FE012156
:1080FC00314806F043FE01254FF4602331480BA9AB
:10810C000D930B948DF830508DF831400E948DF802
:10811C003C6007F09BF92C4B2A4819782A4603231C
:10812C0007F016FA294B022219782648032307F088
:10813C000FFA274B032219782248134607F008FA46
:10814C00244B042219781F48032307F001FA224B11
:10815C00052219781B48032307F0FAF91F4B062256
:10816C0019781848032307F0F3F91D4B3246197898
:10817C001448032307F0ECF9224612484FF4FC6133
:10818C0007F0A8F90F48294607F09AF90D48294637
:10819C0007F08CF90B4807F0A7F90A4807F0AAF981
:1081AC000028FAD1074807F0A9F9064807F0ACF9FE
:1081BC000028FAD110B070BD080002404C240140D8
:1081CC00400200200024014028000020290000204B
:1081DC002A0000202B0000202C0000202D00002065
:1081EC002E000020F0B54469856903466543881A62
:1081FC004FF47A7C002895FBFCF6B8BF4042B042A5
:10820C00B8BF0CFB00F5104E4FF47A7C30682D187B
:10821C0095FBFCF00CFB105737600CB9114611E0C4
:10822C00914205DA1B6841189942A8BF194609E02A
:10823C0008DD064A1B6895FBF2F569185B4299420A
:10824C00B8BF19460846F0BD6802002018FCFFFFB5
:10825C002DE9F047044690F821000D4606281646F5
:10826C009846DDF820A027681ED10868014607F063
:10827C008FFC3E4907F08CFC814694F825004008A1
:10828C0007F032FC0146484607F082FC63698146E0
:10829C007820584307F028FC0146484607F02CFD8F
:1082AC0007F03CFE034611E0072801D000230DE047
:1082BC000868014607F06CFC2D4907F01DFD07F01E
:1082CC002DFE236C6269434393FBF2F3C245C8EB6A
:1082DC000A08B8BF7F42B8F1000FB8BFC8F1000858
:1082EC004FF480409845D8BF002701F023F90128AE
:1082FC0003D1304607F0F8FB31E0384607F0F4FBC9
:10830C002E6880464146304607F0E0FD70B1A0690A
:10831C00636937B90B225043584307F0E1FB154909
:10832C0017E0584307F0DCFB134912E04146304696
:10833C0007F0EAFDA0B1A069636937B90B2250437D
:10834C00584307F0CDFB0D4903E0584307F0C8FB39
:10835C000B4907F0D1FC0146304607F011FB2860B1
:10836C00286807F0DBFDBDE8F08700BF0000C040C7
:10837C000000F04200401C4600007A4400401CC63D
:10838C0000007AC4024B00229A601A605A6070474F
:10839C006C020020014BB3F90C0070476C020020FA
:1083AC0070B54668044615460846324671421E466C
:1083BC0003F082FB636B00B2B3607368A16B451B67
:1083CC00E818F1603560706011B1104B93FBF1F15E
:1083DC000A46494203F070FB0346F068B168326804
:1083EC0058434A434FF4803190FBF1F0A1F57F41A3
:1083FC0092FBF1F2801830617360A1F5014147F6F0
:10840C00FF7203F059FB00B270BD00BF0000FF7F8C
:10841C002DE9F04F87B0A44DBDF84040BDF842C0E7
:10842C002C82A5F812C0044628699B46DDF84C80C6
:10843C008A469146149E02F08DFEC0F30F43ADF8B0
:10844C001230ADF81000049BB8F800706B6194F812
:10845C002130072B25D0082B00F0FD81062B40F096
:10846C00588202F087FA94F8313085B2012B0AD188
:10847C0094F8251018984908E26902F055FA02F0B0
:10848C000FFA4519ADB294F82430012B03D105F540
:10849C00FE45FF35ADB22DB2284602F039FA002068
:1084AC00ADE102F0BDFB012840F0C3814FF4007038
:1084BC0001F040F8012801D1179B5BB94FF4006023
:1084CC0001F038F8012840F0B181D8F80030002BC9
:1084DC0000F0AC8194F82E00012800F0468104D302
:1084EC000228714D40F08F815DE06F4B42F21071AC
:1084FC005A6801328A425A6025D8E56BB4F86E305E
:10850C005543B3F5007FB5FBF1F5ADB202D0B3F531
:10851C00806F02D12BB2C8F80030002002F0F8F9BD
:10852C00002002F08DFB0021604802F0B7FD02A98B
:10853C00C0F30F43ADF8080004223046ADF80A3002
:10854C0007F050F9FCE100225A60104602F070FB73
:10855C0094F82E302BB994F8463043F0010384F88C
:10856C00463094F82E30022B05D194F8463043F067
:10857C00020384F846304C4B4FF0000159831983A9
:10858C00584600F07BFA504600F078FA159A169986
:10859C000023002013600B6002F03CFB4FF4004002
:1085AC0000F0B8FFB3E12B68032B00F2B081DFE8D9
:1085BC0003F00241B5B56B6842F210729342DFF8DA
:1085CC00E8B02AD8E56B01335D43CBF804300020CA
:1085DC00B5FBF2F502F09CF9002002F031FB002112
:1085EC000BF1140002F05AFD0422C0F30F43ADF856
:1085FC00080002A93046ADF80A3007F0F3F8B4F8D9
:10860C006E30ADB2B3F5007F03D0B3F5806F40F0A0
:10861C0097812BB2C8F8003092E1002002F008FBE1
:10862C0094F8463043F0020384F846300123CBF82B
:10863C0000306CE1AD6894F8252085EAE5705208AD
:10864C00A0EBE570C2EB02418842174B63DAA16ED6
:10865C00E769C1EBC1314F435743B4F86E2014485E
:10866C00B2F5007F97FBF0F702D0B2F5806F11D115
:10867C00169B0021D3F800B0584607F045FC08B112
:10868C00ED1B05E05846002107F020FCA8B17D1930
:10869C00054B11E0B2F5006F0FD1D8F80020002A7D
:1086AC0008DDED1B08E000BF6C02002080020020FA
:1086BC00C027090001D07D199D609F4F0020A58F18
:1086CC0002F026F9B86802F0BBFAB7F9081007F106
:1086DC00140002F0E3FC0422C0F30F43ADF80800D1
:1086EC0002A93046ADF80A3007F07CF8B4F86E30C9
:1086FC00B3F5007F02D0B3F5806F02D12BB2C8F86E
:10870C00003094F8467017F0020740F019818A4B3C
:10871C0002221A6015E103221A60F8E04FF0000102
:10872C0029836983584600F0A9F9504600F0A6F950
:10873C00159900232A680B601699022A0B6005D143
:10874C00002002F067FA4FF4004000E080207A4DE0
:10875C0000F0E0FE002002F0DBF8A86802F070FAEE
:10876C00B5F9081005F11400D6E0FFF74BF9724D7E
:10877C0001468046287F02F099F885F81C801FFA84
:10878C0080F802F0F7F805B2284602F0C1F818F4A8
:10879C00004F03D005F5D445AA3507E0B8F1000F1A
:1087AC0000F0F68005F5144505F5AA75B4F94000FE
:1087BC0094F8253045435B0895FBF3F04FF6FF73B7
:1087CC0090FBF3F080B202F047FA02F057FA5A4BE2
:1087DC004FF000025A831A830546584600F04EF9B2
:1087EC00504600F04BF9002002F014FA4FF4004010
:1087FC0000F090FE05F5004501352DB2284602F03B
:10880C001FFA294675E005F11400002102F046FC20
:10881C000027C0F30F43ADF8080002A9304604222C
:10882C00ADF80A303D4606F0DDFF8AE000214348F2
:10883C0072E002F023FA94F82E3000F50045013571
:10884C00012BADB203D102F095F800B200E000208C
:10885C0002F05EF8D1E7E269169994F825304FEAF8
:10886C000238086803FB08F807F058FB0028B8BF6B
:10887C00404200FB08F82B6A40F2DC5298FBF2F8FD
:10888C009844642398FBF3F203FB1283169A2B6231
:10889C00D2F800B0002158464FF0000507F034FB29
:1088AC0008B14FF00105EDB225B1234B6FF0630118
:1088BC009A8907E05846002107F008FB38B11E4B97
:1088CC0064219A8998FBF1F89044A3F80C801A4B18
:1088DC00B3F80C8015B108F5804806E05846002125
:1088EC0007F0F4FA18B1A8F580481FFA88F80FFAC7
:1088FC0088F1124802F0D2FB02A9C0F30F43ADF885
:10890C00080004223046ADF80A3006F06BFF002553
:10891C0017E005F11400002102F0C0FB0025C0F3A4
:10892C000F43ADF8080002A930460422ADF80A3016
:10893C002F4606F057FF04E06C0200208002002056
:10894C00002739B25346B6F900202046FFF728FD20
:10895C00134F4B46388329B2B6F902202046FFF755
:10896C001FFD788307F1180002F0F4FA07F11800E4
:10897C0002F016FBC0F30F43ADF80000ADF8023067
:10898C00009B18467B6201F0F9FC07B0BDE8F08F44
:10899C0001F0F0FF00F5FE40FF3085B22AE700BF82
:1089AC006C020020F8B506680446154608463246A7
:1089BC0071421E4603F080F8636D451BB360A36DD6
:1089CC001D49F3600746356028464FF6FF7203F0E9
:1089DC0073F803467068F16818183360706019B149
:1089EC0063681B0493FBF1F10A46494203F064F8F7
:1089FC000346F068B168326858434A434FF48031FB
:108A0C0090FBF1F0A1F57F4192FBF1F280183061FF
:108A1C00736094F82130082B08D1002F01DDE06B36
:108A2C0009E016BFE06B3846404204E061680A4634
:108A3C00494203F041F8F8BD0100FFFF70B5066D27
:108A4C001D4604469E60881A0023EB6028600A4984
:108A5C004FF6FF7203F030F80346A8684FF48072AB
:108A6C00584390FBF2F028612B6021680A4649427A
:108A7C0003F022F870BD00BF0100FFFF002303616B
:108A8C0003604360704700BF094B19685A689142F4
:108A9C0001D100200BE01A68D118097A013201705B
:108AAC001A601A68202A01D100221A60012070472E
:108ABC0094020020014B9862704700BF9402002082
:108ACC00034B1A78104612B100221A70012070471D
:108ADC009409002038B50B4B8446DC6A1A6B0134C0
:108AEC00202C08BF002494420AD0DD6A0648ED18F9
:108AFC0085F834C040F227710122DC6204F026FABA
:108B0C0038BD00BF940200200048004038B505462F
:108B1C00002401E0FFF7DEFF2B5D01341846002B2B
:108B2C00F8D138BD70B5294C238813F0200F1AD01A
:108B3C00FEF754FF08B1A38815E0254B5A68196855
:108B4C000132202A08BF00228A4205D05968A08829
:108B5C00C918C0B208725A601E4B0A221A601C4B0C
:108B6C009A6A1D4B1A60194E338813F0800F1BD074
:108B7C00194B1C68C4B9164DEA6A2B6B9A420DD07E
:108B8C00FEF704FF2B6B5A1992F834200133B28094
:108B9C002B632B6B202B07D12C6305E03046224630
:108BAC0040F2277104F0D2F90848038813F0400F03
:108BBC000AD040F2266104F0C1FA054B1A6BDB6A4D
:108BCC009A4201D1FEF7F6FE70BD00BF004800408E
:108BDC0094020020980900209C09002030B505461D
:108BEC0087B0544804F0FAFA4FF48020012105F0C4
:108BFC0021FC0820012105F00FFC0820002105F0C4
:108C0C0027FC4D48002105F0D7FE06AC4FF48063DD
:108C1C0024F8043D0323494821468DF816301533BA
:108C2C008DF8173005F038FE042344488DF81730C2
:108C3C0021464FF40063ADF8143005F02DFE684664
:108C4C0004F04EF90B2D25D8DFE805F02406090CAD
:108C5C000F1215181B1E20224FF461531CE04FF409
:108C6C00964319E04FF4E14316E04FF4164313E03A
:108C7C004FF4614310E04FF496330DE04FF4E133C1
:108C8C000AE04FF4613307E02D4B05E02D4B03E078
:108C9C002D4B01E04FF4165369462648009304F01F
:108CAC0055FA27230024012504A88DF8103005233C
:108CBC008DF811308DF812408DF8135005F07AFCB8
:108CCC001C4840F2FF3104F015FA282122461948BD
:108CDC0004F03CF92A46174840F2277104F036F9A3
:108CEC002A46144840F2266104F030F92A4611480D
:108CFC0040F2255104F02AF922460E4840F2244154
:108D0C0004F024F922460B4840F6460104F01EF903
:108D1C002246084840F66A1104F018F960212246F0
:108D2C00044804F013F92946024804F001F907B08D
:108D3C0030BD00BF0048004010001400000C014082
:108D4C0090D0030020A1070040420F00014B0322EA
:108D5C001A607047E8020020044A054B927A0AB167
:108D6C00052200E001221A60704700BFB009002004
:108D7C00E8020020704700BF014B00225A60704788
:108D8C00E802002008B5074B1A6892B242F00802BC
:108D9C001A601A6892B242F004021A60FFF7D6FF0A
:108DAC0008BD00BF405C004010B5064C4FF6FB738D
:108DBC00226802EA03032360FFF7CEFF4FF4064359
:108DCC00236010BD405C0040072818BF1F4B10B536
:108DDC001E4C18BF18702378052B33D8DFE803F02E
:108DEC0003060A0E1621FFF7DFFF2BE0FFF7DCFF6F
:108DFC00042328E002236370013324E06378013BF1
:108E0C00DBB263706378FBB9042218E0104B1A686C
:108E1C0092B242F010021A6005232370DB186370C3
:108E2C0012E06378013BDBB26370637863B9084A84
:108E3C004FF6EF73116801EA030313600622034B2C
:108E4C001A7001E00623237010BD00BF140A002025
:108E5C00405C0040034B9B7A13B1034B05221A6014
:108E6C00704700BFB0090020E8020020014B04222B
:108E7C001A607047E8020020034B1A7A202A01D1AD
:108E8C0000221A72704700BFE8020020704700BF32
:108E9C00212808B508D1124B1B681B7803F07F03FF
:108EAC00212B1AD10F4B0EE0202816D10C4B0E4A59
:108EBC001B681B7810720D4A03F07F03212B0CBF2B
:108ECC00134600234BB1064A4FF0000112680020F4
:108EDC00518293619847002000E0022008BD00BF3A
:108EEC00100A0020318F0008E80200204D8F000886
:108EFC00074B1B681B7803F07F03212B05D102283D
:108F0C0001D0222801D1002000E00220704700BFD0
:108F1C00100A002019B9012801D8084600E00220E7
:108F2C00704700BF28B9044B4FF008021B681A8227
:108F3C0000E00248704700BF100A002058000020D3
:108F4C0028B9044B4FF008021B681A8200E0024853
:108F5C00704700BF100A0020580000200B4B10B5C2
:108F6C00DA6882B11B68052B01D000220BE00023CC
:108F7C0003E00749595CC15401330449CC68A3424E
:108F8C00F7D30023CB60104610BD00BFE8020020D1
:108F9C001C0A0020084BDB68082B01D800200AE0D3
:108FAC000023064A9A5CC2540133092BF9D1024BB7
:108FBC000022DA6001207047E80200201C0A002021
:108FCC00704700BF10B5074C0B468AB2C0216360D6
:108FDC0003F0F0F90120A18803F018F8012002F049
:108FEC00E3FE10BDE802002008B5064B1B68DB78D9
:108FFC00042B01D9002004E0034901EBC30103F069
:10900C0039FC08BD100A00206000002008B5024998
:10901C0003F030FC08BD00BF8000002008B50249F9
:10902C0003F028FC08BD00BF88000020334B10B5AE
:10903C001B686FF03F0200245A72DC729C7220464F
:10904C0002F02AFE20464FF4007102F043FE10217C
:10905C00204602F055FE4021204602F0ABFF802155
:10906C00204602F097FF204602F0D4FE244B204607
:10907C0093F8641002F0ECFF204602F0A3FE0120EE
:10908C00214602F027FE0120C02102F083FF0120BF
:10909C00202102F035FE0120214602F049FE02207B
:1090AC004FF4C06102F016FE02204FF4807102F002
:1090BC0071FF0220214602F03BFE0220202102F02B
:1090CC001FFE0320214602F005FE03204FF4887199
:1090DC0002F070FF0320402102F0BAFF03204FF48E
:1090EC00405102F025FE2146032002F009FE2046E5
:1090FC0003F0CEFB034B01221A6010BD100A0020B6
:10910C0058000020E802002008B5174B174A1968D0
:10911C0089B2118016491288098801EA020212F4F8
:10912C00806F05D04FF6FF321A60124BDB6B9847FD
:10913C000E4B1A880E4B1B8803EA020212F4007FB6
:10914C0008D009490C4A4FF6FF500860117C0131D8
:10915C00C9B21174054A1288134013F4004F01D0A0
:10916C0003F094F908BD00BF445C0040A209002044
:10917C005C0A002058000020E802002010B50320F3
:10918C0002F096FF064C034602464FF488710548E0
:10919C00E36003F027F9032002F014FE10BD00BFBA
:1091AC00E80200201C0A002008B5064A064B20B134
:1091BC001068198805F0D8FB03E01068198805F0D1
:1091CC00D1FB08BDAC090020A809002038B5064D1C
:1091DC0001232B60054B002420461C60FFF7E4FFA5
:1091EC0003232B60204638BD405C0040445C0040AB
:1091FC0008B5FFF7EBFF08BD08B50120FFF7D4FF5A
:10920C00064B0121196006494FF4E0520A800549CA
:10921C000020186008601A6008BD00BF405C004068
:10922C005C0A0020445C0040084B10B51B6800240D
:10923C009C72FFF7E1FF064A4FF406431460043AB0
:10924C001360044A1460044A138010BD100A0020F5
:10925C00445C0040E80200205C0A002007B51422A0
:10926C0000238DF8042001A801228DF806308DF81A
:10927C0007208DF8053005F09DF90EBD002008B5CE
:10928C0005F040F84FF40000012105F0D3F808BDBB
:10929C00F7B5184C184E194F194D9DF820C0316078
:1092AC002A8038600999302204F17E0084F87230EB
:1092BC0084F873C006F096FA0A99182204F1B200E9
:1092CC0006F090FAFFF7DAFFFFF7C8FF03F0A2F9F8
:1092DC003868012105F0A0F803232D888DF806309D
:1092EC0030680D3301A9ADF804508DF8073005F046
:1092FC00D3FAFEBD58000020AC090020180A00204B
:10930C00A8090020014B1868704700BF241A0020E0
:10931C00014B1868704700BF1C1A0020014B1868DD
:10932C00704700BF181A0020014B1868704700BF27
:10933C00101A0020014B1868704700BF201A00203B
:10934C00014B1868704700BF041A0020014B1868C5
:10935C00704700BF0C1A0020014B1868704700BF03
:10936C00081A0020014B1868704700BF141A00201F
:10937C00014B1868704700BF600A0020014B186051
:10938C00704700BF241A0020014B1860704700BFC3
:10939C001C1A0020014B1860704700BF181A0020DF
:1093AC00014B1860704700BF101A0020014B186069
:1093BC00704700BF201A0020014B1860704700BF97
:1093CC00041A0020014B1860704700BF0C1A0020D3
:1093DC00014B1860704700BF081A0020014B186041
:1093EC00704700BF141A0020014B1860704700BF73
:1093FC00600A0020024B00225A6001321A7070473A
:10940C00FC020020024B00225A601A70704700BF09
:10941C00FC020020014B1878704700BFFC020020B2
:10942C00014B5868704700BFFC02002008B5064B82
:10943C0000215A6899600132B2F5FA7F5A6001D165
:10944C00FFF7E0FF08BD00BFFC02002013B50E4B78
:10945C006A4682E803000D499A680C680132A24200
:10946C0001469A6001980DDB1A785AB15B68B3F526
:10947C00FA7F07DA064A02EBC304606042F8331045
:10948C00FFF7D4FF1CBD00BFFC02002088010020A8
:10949C00640A00204FF4FA70704700BF4FF47A60F2
:1094AC00704700BF02207047B0F5FA7F0CDA11B19B
:1094BC00012909D103E0054B53F8300005E0034BBB
:1094CC0003EBC000406800E000207047640A0020F5
:1094DC00012804D0022802D0044B18B900E0034B39
:1094EC00D86001E00022DA60704700BFFC02002067
:1094FC00014BD868704700BFFC020020014B18607C
:10950C00704700BF88010020014B1868704700BFEE
:10951C0088010020024B1A6840EA02021A60704768
:10952C000C030020024B1A6822EA00021A607047F2
:10953C000C030020034B1B6818420CBF00200120B9
:10954C00704700BF0C03002008B56D20FFF7EAFF41
:10955C0008BD00BF034B10B51C68FFF7F5FF204694
:10956C0010BD00BF0C030020034B10B51C68FFF7A7
:10957C00EBFF04F06F0010BD0C03002062B67047C7
:10958C0072B6704708B5FEF77BF908BD08B5FEF753
:10959C006FF908BD08B510B105F0AAF801E005F0A7
:1095AC00AFF808BD07B5104B1B78E3B1FEF798F97F
:1095BC00FEF798F9FEF7B8F9002301E0019B01339F
:1095CC000193019A094B9A42F8D9FEF791F9FEF7EB
:1095DC00A3F9002301E0019B01330193019A034B92
:1095EC009A42E3D8F7E70EBDC10300203F0D0300FC
:1095FC0008B5FEF749FA014B187008BDC1030020ED
:10960C0070B5044600200E4615460321024602F0B2
:10961C00CDF80020C4F30721024602F0C7F8002061
:10962C00E1B2024602F0C2F8002407E0944214BFF3
:10963C000022012202F0BAF83055013400206A1ED3
:10964C00AC420146F2D370BD2DE9F04104460F4601
:10965C00164600200621012202F0A8F80020052160
:10966C00024602F0A3F800200122014602F09EF807
:10967C0010F0020FF2D000200221024602F096F800
:10968C000020C4F30721024602F090F80020E1B25A
:10969C00024602F08BF8002543E0013414F03F0839
:1096AC00795D01D1012204E0721E954214BF0022A3
:1096BC000122002002F07AF8B8F1000F30D1731EAD
:1096CC009D422DD200200521024602F06FF80020A9
:1096DC000122014602F06AF810F00100F2D10621D5
:1096EC00012202F063F800200521024602F05EF828
:1096FC0000200122014602F059F810F0020FF2D0BE
:10970C0000200221024602F051F80020C4F3072188
:10971C00024602F04BF80020E1B2024602F046F895
:10972C000135B542B9D300200521024602F03EF8BE
:10973C0000200122014602F039F810F0010FF2D19D
:10974C00BDE8F08110B5044600200321024602F06A
:10975C002DF80020C4F30721024602F027F8002060
:10976C00E1B2024602F022F800200146012202F08A
:10977C001DF810BD38B5012204460D460020062107
:10978C0002F014F800200521024602F00FF8002028
:10979C000122014602F00AF810F0020FF2D000206C
:1097AC000221024602F002F80020C4F3072102460F
:1097BC0001F0FCFF0020E1B2024601F0F7FF294660
:1097CC000020012201F0F2FF00200521024601F0E9
:1097DC00EDFF00200122014601F0E8FF10F0010F1F
:1097EC00F2D138BD38B50725454305F500650C4663
:1097FC00284609780135FFF7BDFF28466178013509
:10980C00FFF7B8FF2846A1780135FFF7B3FF2846CC
:10981C0021790135FFF7AEFF284661790135FFF755
:10982C00A9FF2846A179FFF7A5FF681CE179FFF78E
:10983C00A1FF38BD37B50725454300200C4602462D
:10984C00032101F0B3FF05F500650020C5F30721E6
:10985C00024601F0ABFF0020E9B2024601F0A6FF80
:10986C0000200146024601F0A1FF8DF80000002007
:10987C000146024601F09AFF8DF8010000200146D6
:10988C00024601F093FF8DF80200002001460246CB
:10989C0001F08CFF8DF8040000200146024601F017
:1098AC0085FF8DF8050000200146024601F07EFF81
:1098BC008DF8060000200122014601F077FF236895
:1098CC00009A23F07F4322F07F429A428DF80700E2
:1098DC0001D0002005E063680198984214BF002075
:1098EC0001203EBD38B5214B1C683BE00020062111
:1098FC00012201F05BFF00200521024601F056FF1A
:10990C0000200122014601F051FF10F0020FF2D0AD
:10991C0000200221024601F049FF0020C4F3072178
:10992C00024601F043FF0020E1B2024601F03EFF87
:10993C00002500203F2D14BF0022012201460135D5
:10994C0001F034FF402DF4D100200521024601F036
:10995C002DFF00200122014601F028FF10F0010F1D
:10996C00F2D14034B4F5804FC0D338BD1000002084
:10997C00194B70B5054618680C46FFF7E3FE174BFC
:10998C001B78834202D1164B1B78BBB1124E0021BF
:10999C003068FFF7EFFEFFF7A5FF124B294618685A
:1099AC002822FFF751FE104B214618687422FFF74E
:1099BC004BFE0A4B30681978FFF7DCFE094B294641
:1099CC0018682822FFF71CFE074B214618687422E2
:1099DC00FFF716FE70BD00BF0C0000200000002039
:1099EC00C1030020900100200400002038B5072599
:1099FC00454300200C460246032101F0D7FE05F535
:109A0C0000650020C5F30721024601F0CFFE0020BF
:109A1C00E9B2024601F0CAFE00200146024601F0FE
:109A2C00C5FE207000200146024601F0BFFE6070AA
:109A3C0000200146024601F0B9FEA070002001464C
:109A4C00024601F0B3FE207100200146024601F0EF
:109A5C00ADFE607100200146024601F0A7FEA07128
:109A6C0000200146012201F0A1FEE07138BD00BFCB
:109A7C00084B9A7852B95B78142B05D8064A1168B2
:109A8C00064A42F8231004E0032200E00422044BAF
:109A9C001A70704758030020BC0300206803002094
:109AAC00B8040020054B01205A7805498242087001
:109ABC0002D15A68034B1A60704700BF580300204C
:109ACC00A404002064040020014B02221A70704789
:109ADC00A4040020074A00231360074A1370074AA6
:109AEC001360074A1360074A1370074A1360074A4A
:109AFC001360704760030020A4040020640400205D
:109B0C00AC04002054030020BC030020F00400200F
:109B1C00014B00221A707047A404002030B5234B6F
:109B2C005B78032B3ED8DFE803F008022F39204B7B
:109B3C0018681E4B5C68002322E01D4A1368092B31
:109B4C0007D81A491B484C68591C40F8234011602F
:109B5C002BE0092227E052F82350591CA5420ED1C4
:109B6C0002EB810204E052F8041C013342F8081C99
:109B7C00411E04328B42F6D30D4B196015E00B4697
:109B8C0083420C4AE7D310E0094A00231360094AC8
:109B9C00002199500433282BF9D106E0064B0A22F8
:109BAC005A6002E00322044B1A7030BD58030020A7
:109BBC00A804002068040020B8040020264A274B83
:109BCC005278092A3BD8DFE802F0050A0F141A2252
:109BDC00282E343720491A6849688A182EE01E4A04
:109BEC00196852688A1A29E01B4A196852684A4354
:109BFC0024E0194A1968526891FBF2F21EE0164AE9
:109C0C001968526891FBF2F002FB101216E012492F
:109C1C001A68496801EA020210E00F491A6849689B
:109C2C0041EA02020AE00C491A68496881EA020218
:109C3C0004E01A68D24301E0074A52681A60074AE6
:109C4C00074B12681AB91A6842F0080202E01A6847
:109C5C0022F008021A60704758030020BC03002051
:109C6C00600300202A4A2B4B52780A2A43D8DFE89B
:109C7C0002F0060B11161C242A30363A3D002649F8
:109C8C001A6809688A1803E0234A196812688A1A44
:109C9C001A6030E0204A196812684A43F8E71E4AF5
:109CAC001968126891FBF2F2F2E71B4A1968126804
:109CBC0091FBF2F002FB1012EAE717491A680968E7
:109CCC0001EA0202E4E714491A68096841EA02024F
:109CDC00DEE711491A68096881EA0202D8E70E4BDF
:109CEC001A68D243D4E71A680B4BD1E70A4A1868B2
:109CFC00116810601960074A084B12681AB91A6883
:109D0C0042F0080202E01A6822F008021A6070475A
:109D1C0058030020BC030020F00400206003002046
:109D2C00134B5B78052B22D8DFE803F003080D12E8
:109D3C00171C104B1A6802F00F0217E00D4B1A6833
:109D4C0022F0100212E00B4B1A6822F020020DE0F8
:109D5C00084B1A6822F0400208E0064B1A6822F001
:109D6C00800203E0034B1A6822F480721A60704779
:109D7C005803002060030020124B1A68124B5B68DA
:109D8C009A4206DD114B196841F0040121F00301E0
:109D9C000CE00E4B05D1196821F0060141F00101D0
:109DAC0004E0196821F0070141F002011960074B2A
:109DBC001AB91A6842F0080202E01A6822F0080286
:109DCC001A607047BC030020580300206003002079
:109DDC0010F0020F0CD111F0100F07D0064B04211C
:109DEC005A68064B1970064B1A6004E00A2200E010
:109DFC000822044B1A70704758030020A40400205A
:109E0C0050030020B8040020014B00221A70704748
:109E1C00A40400200F4B5B78032B1AD8DFE803F067
:109E2C00020413150C4B00E00C4B1A680C4B110A76
:109E3C0093F800C00B4B18780B4B1A7183F807C0C2
:109E4C009871597105E0094B00E0094B1A68064BF3
:109E5C005A6070475803002050030020640400200F
:109E6C00A404002054030020B8040020BC030020EC
:109E7C00F0040020014B02221A707047C00300202E
:109E8C00024B5A68024B1A60704700BF58030020FF
:109E9C0064040020294B5B780C2B4ED8DFE803F0D0
:109EAC00070C11161C21262B30353A3F4400244B4D
:109EBC001B6813F0080F3BE0214B1B6813F0080FD5
:109ECC0008E01F4B1B6813F0010F31E01C4B1B68A3
:109EDC0013F0010F31D12CE0194B1B6813F0040F58
:109EEC0026E0174B1B6813F0050F21E0144B1B6881
:109EFC0013F0020F1CE0124B1B6813F0030F17E05A
:109F0C000F4B1B6813F0100F12E00D4B1B6813F076
:109F1C00200F0DE00A4B1B6813F0400F08E0084BB4
:109F2C001B6813F0800F03E0054B1B6813F4807F54
:109F3C0003D0024B5A68034B1A6070475803002039
:109F4C006003002064040020074970B50B68072BE0
:109F5C0009D8064A064816684068064D5C1C45F848
:109F6C0023600C60106070BDAC0400206404002001
:109F7C005803002044040020054B1A6832B10549EF
:109F8C00013A51F822101A60034B1960704700BF58
:109F9C00AC0400204404002064040020014B002287
:109FAC001A707047A4040020084B9A784AB95A7862
:109FBC00142A04D85968064B43F8221004E00322F3
:109FCC0000E00422034B1A70704700BF58030020B6
:109FDC0068030020B8040020114B9A7852B95A78C3
:109FEC00104B142A04D8104951F822205A6004E06E
:109FFC00032201E00B4B04221A700C4B1B786BB143
:10A00C00084B0B495A680B4B0A601AB91A6842F094
:10A01C00080202E01A6822F008021A60704700BFBA
:10A02C0058030020B8040020680300209C04002082
:10A03C00BC0300206003002010B5094B9A7852B97C
:10A04C005C78142C05D8FAF701FA064B43F8240077
:10A05C0004E0032200E00422034B1A7010BD00BF81
:10A06C005803002068030020B804002038B5284BA2
:10A07C001B788BB9274A284B5268B2F1FF3F04BFBB
:10A08C00264A12680A214A431A6000F05BF9244BF5
:10A09C00012218601E4B1A701E4B5C7814B1012CF7
:10A0AC0035D10EE000F04EF91D4B1A681A4B821A8E
:10A0BC00002A1B68B8BF52429A4224D9144B1C7018
:10A0CC0025E0FFF747FA10F4804507D0154B1049EF
:10A0DC001A68002022F01002087017E00E4C23685A
:10A0EC008BB100F02FF90E4A23681268821A002AED
:10A0FC00B8BF52429A4206D90A4B05491A680D70EC
:10A10C0042F0100202E0084B1A68013A1A6038BD9E
:10A11C005403002058030020F4080020BC03002046
:10A12C0090040020600300206404002070B5104DE2
:10A13C00104E2868104C32787368B0F5006F62705E
:10A14C0063600FD83146FFF74DFB31462868FFF7A7
:10A15C0071FB20B12B6801332B60652300E00723D2
:10A16C00237004E007232370044B00221A7070BD87
:10A17C005003002058030020B8040020A404002041
:10A18C0037B5124C657815B1012D1AD10FE0104B73
:10A19C00042201A91868FFF733FA6168019A0D4B84
:10A1AC00914202D101225A600EE05D600CE0A3786E
:10A1BC002A2B06D1064B211D18680422FFF744FAFE
:10A1CC0002E0044B03221A703EBD00BF580300206E
:10A1DC0008000020B80400202DE9F3411E4B1F4C51
:10A1EC005B681F4A0125B3F5006F1570207027DCE2
:10A1FC0011EA050624D118466946FFF7F7FB9DF8CE
:10A20C0000809DF801709DF802C09DF807009DF834
:10A21C0006109DF805209DF80430267284F8018004
:10A22C00A77084F803C020716171A271E3710B4BAC
:10A23C00E95C1A7A01358A18082D1A72F7D108E0F0
:10A24C000123064A002199540133082BF9D11378C4
:10A25C001372BDE8FC8100BF58030020C40300202A
:10A26C00C003002008B50A4B0A491A6802EA01012A
:10A27C0069B95A6840F2D2439A4208D1064B186821
:10A28C00FFF778FAFFF72EFB0120FFF783F908BDE3
:10A29C005803002000FFFF000C00002008B5034B02
:10A2AC001A68034B5A60FBF7EBFA08BDBC0300209D
:10A2BC005803002008B5044B05201A68034B5A605C
:10A2CC00FBF720FC08BD00BFBC0300205803002096
:10A2DC00154B1A78BAB15968144A01315960116892
:10A2EC00134B01311160134A196812780131012A9C
:10A2FC00196005D1104B1A6812B11A68013A1A602C
:10A30C000022094B00E001221A700A4B1A78012A2C
:10A31C0009D10A4B196831B11968013919601B68E8
:10A32C000BB9074B1A7070471003002088090020E6
:10A33C00800900204E0000209C0900209809002074
:10A34C0094090020014B5868704700BF100300208F
:10A35C0008B5042003F04EFD48F6A04003F05AFD6A
:10A36C00012003F05DFD04480321002204F0F0F904
:10A37C00012003F06BFD08BD9AC3020043F2B60145
:10A38C0002B24A43494903144B434FF0020C99184B
:10A39C0091FBFCF19A1A82B0002992FBFCF201901D
:10A3AC0004DA002A2ADB002B6CDC04E0002A56DAE3
:10A3BC00002B47DC34E003F5E150801A4FF4802188
:10A3CC0090FBF1F000F5617080B200EB6242A1F5F8
:10A3DC00003193FBF1F192B2511A89B2344BB3F8BC
:10A3EC0020C02CF4005C4FEA0C4C4FEA1C4CA3F838
:10A3FC0020C098861A87998702B0704701F5E15002
:10A40C00801A4FF4802390FBF3F000F56170A3F5F4
:10A41C00003380B292FBF3F291FBF3F182182EE041
:10A42C00C3F5E150401880144FF4003200F5617010
:10A43C0091FBF2F180B2411A93FBF2F289B28A18C5
:10A44C0092B2CBE703F5E150801A801400F56170ED
:10A45C004FF4003180B292FBF1F28218B9E701F5AA
:10A46C00E150801A4FF4802390FBF3F000F56170FB
:10A47C00A3F5003380B291FBF3F100EB6242411A79
:10A48C0092B2AAE7C3F5E15040184FF4802290FB3A
:10A49C00F2F000F56170A2F5003291FBF2F180B29E
:10A4AC00411A89B201EB63439AB297E7E0E3FFFFED
:10A4BC00002C0140064B00F5617001F5617102F54D
:10A4CC00617280B289B292B2988619879A87704766
:10A4DC00002C0140F0B57D4B8FB01C78012C07D1BE
:10A4EC002146402003F098FF21464FF4006002E023
:10A4FC0040F60C00012103F08FFF08AC744803F008
:10A50C0017FC204603F00AF84FF000038DF82830B2
:10A51C00ADF820304FF06003ADF822304FF4E1631A
:10A52C0021466B48ADF824304FF48073ADF82630DB
:10A53C0002F09CFE684602F0FBFF4FF07003ADF892
:10A54C0000304FF00103ADF802304FF00403ADF8CA
:10A55C00043040F20553ADF806304FF00203ADF86D
:10A56C0008304FF00803ADF80A304FF480735848A8
:10A57C006946ADF80C304FF40073ADF80E3002F0B4
:10A58C0097FE5348694602F0DBFE0DAC6946504815
:10A59C0002F026FF204604F0C9F94C4B197801292A
:10A5AC0016D14C4804F008FA18238DF837300323E1
:10A5BC0021468DF8363048484FF47C53ADF8343092
:10A5CC0004F06AF944484FF4285104F0D7F915E027
:10A5DC0018238DF837300323404821468DF8363048
:10A5EC004FF4E063ADF8343004F056F94EF200034A
:10A5FC0021463B48ADF8343004F04EF9344C082178
:10A60C00204603F0C5F82046082103F0CBF820467D
:10A61C00082103F0D1F8334B4FF000051B8804A937
:10A62C00ADF816304FF40063ADF810304FF4806382
:10A63C00ADF812304FF400532046ADF81A304FF4F9
:10A64C008043ADF81C30ADF81450ADF8185002F042
:10A65C004DFF2046012103F0A7F901210A462046AF
:10A66C0002F0A2FF2046012103F084F801212046CC
:10A67C0002F07CFF0CAF4FF4A06003F091FF384662
:10A68C0003F0DAFF01261A230BA88DF82C308DF875
:10A69C002D608DF82E508DF82F6003F08BFF192351
:10A6AC0038468DF830308DF832508DF831608DF899
:10A6BC00336003F07FFF2046314602F065FF4FF414
:10A6CC006173A3862387A3870FB0F0BD38020020E7
:10A6DC00002C0140C0001600001801400008014089
:10A6EC00000C014052000020024B1A6801321A6023
:10A6FC00704700BF2C1A00200028B8BF40424043CE
:10A70C004B6EC9694FF0140C48430CFB03FC154B02
:10A71C0070B51A6844F620655C6890FBF5F5BCFBD7
:10A72C00F1F064210132B0FBF1F02D1982421A6074
:10A73C005D6016DB9A680C4C501C90FBF1FC01FB25
:10A74C001C01DE6854F822004FF47A7CB5FBFCF552
:10A75C00361A76190020586044F82250DE60996051
:10A76C00186070BD18030020301A0020014BD86807
:10A77C00704700BF18030020014B1868704700BFDA
:10A78C002C1A0020014B1860704700BF2C1A0020B7
:10A79C0008B5054B1B7C012B05D1044B04491868EB
:10A7AC000422FEF751FF08BD18030020281A0020D0
:10A7BC002C1A002008B5054B042218600449FEF73A
:10A7CC001FFF044B01221A7408BD00BF281A002079
:10A7DC002C1A002018030020014B1868704700BF8A
:10A7EC00C81B0020014B1860704700BFC81B00201D
:10A7FC0008B5074B1B78012B09D1064B0649186885
:10A80C000422FEF721FFFFF79DFD044B186008BDE5
:10A81C002C030020C41B0020C81B0020C01B0020E0
:10A82C0038B50F4B1B78012B18D1FFF78BFD0D4C56
:10A83C004EF65F222368C31A002BB8BF5B429342CB
:10A84C000CDD094B094A1D681068013519460422B4
:10A85C001D60FEF7F9FEFFF775FD206038BD00BFE7
:10A86C002C030020C01B0020C81B0020C41B002090
:10A87C0008B5074B042218600649FEF7C1FEFFF726
:10A88C0061FD054B01221860044B1A7008BD00BF16
:10A89C00C41B0020C81B0020C01B00202C03002060
:10A8AC00014BB3F90000704730030020884203D0FD
:10A8BC00164B4FF000021A800138052822D8DFE829
:10A8CC0000F00717030F0B13012916D0022912E011
:10A8DC00052912D003290EE004290ED001290AE023
:10A8EC0006290AD0052906E0022906D0042902E02F
:10A8FC00032902D0062905D101E0012003E04FF61F
:10A90C00FF7000E0002000B2704700BF3003002051
:10A91C00014B5860704700BF30030020014B586852
:10A92C00704700BF3003002000F13B03762B10B5BD
:10A93C000D4B0BD951430D4AB3F800C0800392FB69
:10A94C00F1F190FBF1F06044188002E04FF000024E
:10A95C001A80054C0649B4F9000042F6AA2201F00F
:10A96C00ABF8208010BD00BF30030020206CFBFF33
:10A97C0056D5FFFF012008B5FDF744F80138C0B2E9
:10A98C00052801D9002002E0024B33F8100000B278
:10A99C0008BD00BF2C00010810B50B4C002220682C
:10A9AC00022102F001FE20684FF448730385002158
:10A9BC0003F046F82068012102F0D8FD206802213E
:10A9CC00012202F0F1FD10BD400000200C4B07B538
:10A9DC001B78012B01D11B3304E00A4B1B78012B94
:10A9EC0002D11D338DF80430002301A88DF80730F7
:10A9FC0003F0E0FD044B186803F09AF90EBD00BF9C
:10AA0C00390200204400002040000020F0B5694BC2
:10AA1C0089B01C780546012C16D12046214603F03E
:10AA2C0009FD2146042006AC03F0F6FC204603F099
:10AA3C007DFF03238DF81A3001338DF81B3021462E
:10AA4C005D484FF0070335E05C4B1E78012E35D185
:10AA5C000420314603F0EEFC594B06AC1F78012F55
:10AA6C001AD13946202003F0D7FC204603F05EFFB4
:10AA7C0003238DF81A30013321468DF81B305148D1
:10AA8C004FF4E043ADF8183003F006FF39464FF4AD
:10AA9C00805003F091FF11E03146082003F0BCFC1C
:10AAAC00204603F043FF482347488DF81B302146CE
:10AABC004FF4E073ADF8183003F0EEFE434C03AEE8
:10AACC00206803F035F9304602F028FD4FF0FF33D3
:10AADC0031462068ADF810304FF00003ADF812305D
:10AAEC0002F0C4FB684602F02DFD4FF00003ADF8F8
:10AAFC0000304FF00203ADF802304FF00B03694603
:10AB0C002068ADF808304FF00303ADF8043003F0C3
:10AB1C00ABF801224FF44871206802F093FD2068D5
:10AB2C0002F060FD0121206802F04CFF40212068FA
:10AB3C0002F096FD0421206802F06AFF01212068D2
:10AB4C0002F032FF012D6E4628D11A4B1B78012BD7
:10AB5C0001D11B3304E0194B1B78012B02D11D339F
:10AB6C008DF81C30194C01250023022607A88DF8FE
:10AB7C001E308DF81D608DF81F5003F01BFD2068F2
:10AB8C0041F65F6102F0C6FF314620682A4602F0AA
:10AB9C000BFD294620682A4602F006FD0B4C0021CD
:10ABAC00206802F04DFF2068012102F0DFFC09B0A3
:10ABBC00F0BD00BF39020020000801404400002015
:10ABCC003802002000140140000C0140400000201D
:10ABDC00014B1880704700BFD01B0020014B186040
:10ABEC00704700BFCC1B002010B504460846FFF789
:10ABFC00EFFF2046FFF7F2FF10BD00BF014B1878A6
:10AC0C00704700BF38030020014B00221A707047B8
:10AC1C0038030020014B1870704700BF8C010020D6
:10AC2C00014B1878704700BF8C010020704700BFA3
:10AC3C00024B80B21B689884704700BF480000200C
:10AC4C00014B5860704700BF38030020014B586817
:10AC5C00704700BF3803002008B5034B0146186845
:10AC6C0002F0EEFE08BD00BF4800002008B5024B04
:10AC7C00186802F041FF08BD4800002008B5084BD9
:10AC8C00186802F039FF074B074A1B68C0EB0040FD
:10AC9C001288B0FBF3F302FB03F080B208BD00BFD7
:10ACAC0048000020CC1B0020D01B0020164B07B501
:10ACBC001B78012B04D107338DF80430143310E0CA
:10ACCC00124B1B78012B04D116338DF8043006334C
:10ACDC0007E00F4B1B78012B14D116338DF8043081
:10ACEC0007338DF8003001A800238DF803308DF860
:10ACFC00073003F05FFC684603F05CFC054B1868FA
:10AD0C0003F016F80EBD00BF3A0200204C000020E4
:10AD1C003B02002048000020F0B5864B8BB01C781D
:10AD2C000746012C0D4618D12046214603F082FB24
:10AD3C002146042008AC03F06FFB204603F0F6FD1F
:10AD4C0048238DF8233021464FF007037A48ADF89D
:10AD5C00203003F0A1FD1C233CE0784B1C78012C27
:10AD6C001CD10220214603F065FB08AE21461020C1
:10AD7C0003F052FB304603F0D9FD482331467048AE
:10AD8C008DF823304FF4E073ADF8203003F084FDE0
:10AD9C0021466C4803F010FE1D231BE06A4B1C7807
:10ADAC00012C19D12146042003F044FB2146082034
:10ADBC0008AC03F031FB204603F0B8FD48238DF8B6
:10ADCC00233021464FF4E0736048ADF8203003F097
:10ADDC0063FD1E238DF824300223002409A88DF86E
:10ADEC002530013B8DF827308DF8264003F0E2FB2F
:10ADFC00574B013F186802F09BFF03A802F08EFB33
:10AE0C00012D18BFADF80E40ADF80C40ADF8124056
:10AE1C004F4C08BF102303A9206808BFADF80E30B3
:10AE2C00ADF8107002F022FA012D01D1002200E0E1
:10AE3C00022203211346206802F026FC684602F029
:10AE4C0081FB434B694618684FF00803ADF8083096
:10AE5C0002F00AFF374B1B78012B02D14FF0040391
:10AE6C000CE0364B1B78012B02D14FF0080305E0A8
:10AE7C00354B1B78012B03D14FF00C03ADF8003090
:10AE8C00334C6946206802F0EFFE0121206802F085
:10AE9C0041FE01210A46206802F086FB20684FF033
:10AEAC0000030121838402F061FB224B1B78012BF0
:10AEBC0005D10020022103F0ADFD04230EE01F4B51
:10AECC001B78012B01D1022003E01F4B18780128BD
:10AEDC0005D1082103F09EFD4FF4807306930023E7
:10AEEC0008248DF81C3006A801338DF81E308DF81F
:10AEFC001D4003F037FE0F4B1B78012B02D18DF850
:10AF0C0024400AE00D4B1B78012B03D00E4B1B7811
:10AF1C00012B02D116338DF824300023012209A80D
:10AF2C008DF826308DF827208DF8253003F042FB64
:10AF3C000BB0F0BD3A020020000801404C0000208C
:10AF4C0000100140000C1A003B020020000C0140D4
:10AF5C0048000020B0F90030B0F9022003FB03F1E7
:10AF6C0002FB021110B50C4CA14214D94FEA116C22
:10AF7C00ACF13A0C09495FFA8CFC31F81CC04FF467
:10AF8C00004102FB0CF203FB0CF392FBF1F293FB7E
:10AF9C00F1F14280018010BD0044FA3A38000108FA
:10AFAC00124B37B5B3F902C0B3F90010B0F9022057
:10AFBC00B0F9000002FB0CF400FB01F500FB0CFCEB
:10AFCC004A434FF4004395FBF3F194FBF3F492FBEB
:10AFDC00F3F264189CFBF3F3D31A0020A2B262F3D1
:10AFEC000F009BB263F31F403EBD00BF4003002027
:10AFFC00A0F50040C0F3891000F44073B3F5807FD6
:10B00C0082B037D001DC23B305E0B3F5007F05D067
:10B01C00B3F5407F0FD00023184639E0C0B21E4B69
:10B02C00420082F4FF7203EB4000D218B0F88C009F
:10B03C00B2F88C302CE0184AC0B202EB400340004E
:10B04C0080F4FF70B3F88C3082185B42B2F88C003D
:10B05C000EE0114BC0B2420082F4FF7203EB4000D1
:10B06C00D218B0F88C00B2F88C3040425B4280B2FF
:10B07C009BB20DE0C0B2084B420082F4FF72D218B2
:10B08C00B2F88C2003EB40035242B3F88C3090B2F0
:10B09C0043EA004002B070473800010830B504465E
:10B0AC0085B00846FFF7A4FFC0F30F43ADF802309C
:10B0BC00ADF80000134A00994FF400431160B4F945
:10B0CC000210B2F90200B4F900C0B2F9002001FB81
:10B0DC0000F50CFB02F40CFB00F04A4394FBF3F478
:10B0EC0095FBF3F192FBF3F2641A90FBF3F3D31894
:10B0FC000020A2B262F30F009BB263F31F4005B0B5
:10B10C0030BD00BF40030020032903D8DFE801F065
:10B11C0004081014002018E00D4B03EB400004E071
:10B12C0040000B4B80F4FF70C018B0F88C000CE0A2
:10B13C00074B03EB400004E04000054B80F4FF702C
:10B14C00C018B0F88C00404280B200B2704700BF0B
:10B15C003800010883B244F6E61100140FFA83FCA0
:10B16C00484301FB0CF14FF4004291FBF2F190FBD0
:10B17C00F2F290B24A42A2EB4002002063F30F00BD
:10B18C0092B284B062F31F4004B0704730B585B002
:10B19C006B4683E80300BDF90410BDF9020040F2D0
:10B1AC00C46202FB01F402FB00FCBDF900506FF01D
:10B1BC00020290FBF2F003236D0091FBF2F10918EF
:10B1CC0095FBF3F540F6B8339CFBF3FC4A1994FB62
:10B1DC00F3F3CCEB030392B2002062F30F009BB2AB
:10B1EC0063F31F4005B030BD30B50C4B0C4C84469E
:10B1FC0022681B689A4201D100200EE02368094A9C
:10B20C005D1C02EB03130FCB8CE80F002560236849
:10B21C00082B01D100232360012030BD601C0020CD
:10B22C00D41B0020E01B0020704700BF7FB52B4BC8
:10B23C002B4A19681268914204D10120002103F0B5
:10B24C00EFFE48E01968274A02EB0111487850B12B
:10B25C001B6802EB0312536804228DF80C200022A9
:10B26C000192029307E01B68029002EB03125368F1
:10B27C008DF80C000193194B1A681A4B03EB02134F
:10B28C009B781BB102238DF80D3001E08DF80D3049
:10B29C00124B00221968134B0901CB5C8DF80E3050
:10B2AC000E4B0DF1180C18680CEB020102EB001C94
:10B2BC000C4801326044007A082A01F8090CEFD1DD
:10B2CC001A6801321A601A68082A01D100221A6021
:10B2DC0001A803F0B3FE07B000BD00BFDC1B0020CB
:10B2EC00D81B0020641C0020F0B5437887B00646BC
:10B2FC00426833B104238DF80C3000230292019381
:10B30C0003E0029301928DF80C30B37803B1022361
:10B31C008DF80D30327800238DF80E20F21801A82C
:10B32C00117AC2180133082BD172F7D103F086FEC3
:10B33C00042818D10D4D0E4B2C681B680134082CB9
:10B34C0008BF00249C4201D100200DE096E80F00BC
:10B35C002F68084E06EB071C8CE80F0001200146F5
:10B36C002C6003F05DFE012007B0F0BDD81B00205F
:10B37C00DC1B0020641C002030B5294D294B2C68A7
:10B38C001B680134082C08BF00249C4287B043D0B2
:10B39C0001A903F02FFF9DF80C20234B042A09D19F
:10B3AC002A68012103EB021251702A6803EB021385
:10B3BC00029A08E02A68002103EB021251702A68F5
:10B3CC0003EB0213019A5A609DF80D30144A022BBC
:10B3DC00154B04D1126803EB0213012203E012682F
:10B3EC0003EB021300229A700D4B9DF80E101A6895
:10B3FC000D4B1201D1540023094A06A9C818116833
:10B40C00094D03EB011110F8090C01334919082BF4
:10B41C000872F1D1146001E003F0D0FE07B030BD2A
:10B42C00601C0020D41B0020E01B002008B501206C
:10B43C00FFF7A2FF08BD00BF08B50020FFF79CFF77
:10B44C0008BD00BF2DE9F0470C238AB08DF81C30E5
:10B45C0003238DF81D30013800238DF81B300C466A
:10B46C00154607281AD8DFE800F01613100D0A1934
:10B47C0007044FF0020313E04FF0040310E04FF009
:10B48C0010030DE04FF014030AE04FF0280307E01F
:10B49C004FF0640304E04FF0C80301E04FF00803E1
:10B4AC00ADF81E3003F0C6FF4FF00070012102F022
:10B4BC00C1FF0120014602F0AFFF0420012102F080
:10B4CC00ABFF0420002102F0C3FF4FF4EA1000216F
:10B4DC0003F072FA0AAE4FF4805326F8043D0323AE
:10B4EC00314667488DF8263015338DF8273003F038
:10B4FC00D3F90423314662488DF827304FF40063AA
:10B50C0000260127ADF824301FFA84F803F0C4F9A3
:10B51C0005A80DF1040A8DF81A608DF814608DF8E9
:10B52C0015708DF816608DF817608DF818708DF801
:10B53C00197003F073FC4FEA4813ADF8083050460D
:10B54C004FF0FF338DF804608DF805608DF80670B0
:10B55C00ADF80A60ADF80C30ADF80E30ADF81060F7
:10B56C008DF81270B14603F0CBFCBDB16B01ADF898
:10B57C00083050464FF0FF338DF80560ADF80A6087
:10B58C008DF812708DF804708DF80670ADF80C30D3
:10B59C00ADF80E30ADF8107003F0B2FC4FEAC803F2
:10B5AC0043F004030DF10408002701260222641362
:10B5BC00ADF80A3040464FF0FF338DF80420ADF85B
:10B5CC0008408DF805708DF80660ADF80C30ADF8BC
:10B5DC000E30ADF810708DF8126003F091FCBD4286
:10B5EC001BDDEB0043F004036D130322ADF80A30AE
:10B5FC0040464FF0FF338DF804208DF80570ADF800
:10B60C0008508DF812608DF80660ADF80C30ADF86E
:10B61C000E30ADF8106003F073FC08AF0124072660
:10B62C000025142338468DF820308DF821608DF8D4
:10B63C0022508DF8234002F0BDFF152338468DF8BB
:10B64C0020308DF821608DF822508DF8234002F0C7
:10B65C00B1FF132338468DF820308DF821608DF81A
:10B66C0022508DF8234002F0A5FF0220214603F062
:10B67C00D7FC2146102003F0D3FC0AB0BDE8F087BC
:10B68C000008014030B52A4B87B01B780546012BCA
:10B69C0003D1012801D1274C00E0274C2046002182
:10B6AC0002F032FC4FF00003ADF804304FF482731B
:10B6BC00ADF806304FF00003ADF808304FF0020340
:10B6CC00ADF80A304FF00103ADF80C304FF40073B5
:10B6DC00ADF80E304FF00003ADF81230ADF8143069
:10B6EC00042D17D8DFE805F00306061609004FF005
:10B6FC00100311E04FF008030EE04FF40063ADF8B7
:10B70C0008304FF01003ADF810304FF00003ADF8D7
:10B71C000A3003E04FF01803ADF8103001A92046B1
:10B72C0002F0B6FB2046012102F0EEFB07B030BD63
:10B73C003C0200200038004000300140F8B5194DA3
:10B74C0004462B780E468342174602D0FFF79AFF29
:10B75C002C7014B1042C23D102E0FCF77DF801E02D
:10B76C00FCF7BAF81048022102F062FC0028F9D06C
:10B77C0031460D4802F000FC0B48012102F058FC48
:10B78C000028F9D047B114B1042C09D102E0FCF720
:10B79C0069F801E0FCF7A2F8034802F0EFFB00E0C7
:10B7AC000020F8BD4403002000300140F8B52A4DBC
:10B7BC0004462B780E468342174602D0FFF762FFF1
:10B7CC002C70042C46D8DFE804F00306090C0F009B
:10B7DC00FCF742F80AE0FCF773F807E0FCF774F8A2
:10B7EC0004E0FCF775F801E0FCF776F81B4B1B78CE
:10B7FC00012B03D1012C01D1194D00E0194D284624
:10B80C00022102F015FC0028F9D03146284602F03E
:10B81C00B3FB2846012102F00BFC0028F9D0A7B19C
:10B82C00042C17D8DFE804F00306090C0F00FCF712
:10B83C0019F80AE0FCF746F807E0FCF747F804E0D3
:10B84C00FCF748F801E0FCF749F8284602F096FBB3
:10B85C00C0B200E00020F8BD440300203C020020F0
:10B86C0000380040003001402DE9F041012186B044
:10B87C004FF4805002F0D0FD0120014605AF02F0DC
:10B88C00CBFD182403264FF0A00348483946ADF8E9
:10B89C0014308DF816608DF8174002F0FDFF4FF054
:10B8AC00400342483946ADF814308DF816608DF8D7
:10B8BC00174002F0F1FF0120002103F07DF84FF05A
:10B8CC000003ADF800304FF48273ADF802304FF046
:10B8DC000003ADF804304FF00203ADF806304FF022
:10B8EC000103ADF808304FF4007331486946ADF8E8
:10B8FC000A304FF00003ADF80E30ADF81030ADF853
:10B90C000C4002F0C5FA0121294802F0FDFA294B3E
:10B91C00E8461D78012D42D14FF48040294602F0B3
:10B92C0089FD4AF2000324483946ADF814308DF8ED
:10B93C0016608DF8174002F0AFFF4FF48043394684
:10B94C001D48ADF814308DF816608DF8174002F0D4
:10B95C00A3FF4FF00003ADF800304FF48273ADF845
:10B96C0002304FF00003ADF804304FF00203ADF895
:10B97C0006304FF4007369461048ADF80A304FF0AA
:10B98C000003ADF80C40ADF80850ADF80E30ADF832
:10B99C00103002F07DFA2946084802F0B5FA084B3F
:10B9AC004FF0FF321A7006B0BDE8F081000801407C
:10B9BC00003001403C020020000C014000380040E7
:10B9CC004403002003464FF6FF70834246DDB3F17B
:10B9DC00807F23DBB3F1805F0FDBB3F1804F07DB9C
:10B9EC00334A934263DC33491A168A5C12020FE025
:10B9FC0030499A158A5CD2010AE0B3F1806F2D4A66
:10BA0C0003DB1915525C920102E09914525C52014D
:10BA1C0093FBF2F101325218521019E0B3F5801F6A
:10BA2C000BDBB3F5800F234A03DB1914525C1201B4
:10BA3C000EE09913525CD2000AE0B3F5802F1D4A38
:10BA4C0003DB1913525C920002E09912525C520013
:10BA5C0093FBF2F1501C401840101BE0FF2B1FDD34
:10BA6C00B3F5805F0ADBB3F5804F124A02DB191283
:10BA7C00505C0EE09911505C40080AE0B3F5806F01
:10BA8C000C4A03DB1911505C800802E09910505CE1
:10BA9C00C008013000FB00F29A4208DD013806E0D4
:10BAAC00002BA9BF034A4FF0FF30D05C0009704750
:10BABC000080FE7FC4020108904203DC8142ACBFCF
:10BACC000A4602461046704770B5044610460E46AC
:10BADC0004F00AF805462946204604F015FA40B948
:10BAEC00304604F001F805462946204604F0EEF9EC
:10BAFC0000B12C46204670BD70B514460E4603F0BE
:10BB0C00F3FF0546204603F0EBFF0446214628468A
:10BB1C0004F0F2F80146284603F030FF05463046A3
:10BB2C0003F0E2FF214604F0E7F80146284603F053
:10BB3C0027FF04F0F3F970BD70B51BB12D2301F88C
:10BB4C00013B40424B1CB0FBF2F402FB140C5D1E9B
:10BB5C00BCF1090F8CBF0CF1570C0CF1300C03F835
:10BB6C0001CC1E4620460133002CECD134702B78CE
:10BB7C000A7805F8012901F8013BA942F7D33046B0
:10BB8C0070BD00BF0A2A08B5844613468E4603D101
:10BB9C00002801DA012303E01A46604671460023AF
:10BBAC00FFF7CAFF08BD00BF642303FB00F292FB42
:10BBBC00F1F29A420BDD47F6122359436FF003035F
:10BBCC00584391FBF0F000F574505C3019E012F121
:10BBDC00640F0BDA47F6122359436FF003035843F3
:10BBEC0091FBF0F0A0F574505C380AE01C224B433A
:10BBFC00424393FBF0F092FBF1F1024B401893FBA4
:10BC0C00F0F0704700410F00002908B502DDFFF786
:10BC1C00CBFF14E006D1002811D0D4BF084843F65E
:10BC2C005C500CE0002805DBFFF7BEFF00F5F4408C
:10BC3C00B83004E0FFF7B8FFA0F5F440B83808BD01
:10BC4C00A4C2FFFF014B1860704700BF405C00406E
:10BC5C00014B186880B27047405C0040014B186083
:10BC6C00704700BF445C0040014B186880B27047BD
:10BC7C00445C0040014B186880B27047485C00403F
:10BC8C00014B1860704700BF4C5C0040014B1868BA
:10BC9C0080B270474C5C00404FF6F873024A00EAE1
:10BCAC0003031360704700BF505C0040014B1868E1
:10BCBC0080B27047505C0040014B43F82010704735
:10BCCC00005C0040024B53F8200080B2704700BF6C
:10BCDC00005C0040054B10B553F8204048F68F121D
:10BCEC0004EA02020A4343F8202010BD005C004025
:10BCFC00024B53F8200000F4C0607047005C004019
:10BD0C000A4B10B553F8202048F6BF7402EA04041D
:10BD1C0011F0100F18BF84F0100411F0200F18BF91
:10BD2C0084F0200443F8204010BD00BF005C0040AC
:10BD3C000A4B10B553F820204BF68F7402EA04041A
:10BD4C0011F4805F18BF84F4805411F4005F18BFA5
:10BD5C0084F4005443F8204010BD00BF005C004048
:10BD6C0038B50D460446FFF7ADFF012D02D120F486
:10BD7C00805003E0022D04D120F01000014B43F859
:10BD8C00240038BD005C0040024B53F8200000F04A
:10BD9C0030007047005C0040024B53F8200000F468
:10BDAC0040507047005C0040054B48F6BF7253F89A
:10BDBC00201001EA020282F0300243F82020704782
:10BDCC00005C0040054B4BF68F7253F8201001EAD3
:10BDDC00020282F4405243F820207047005C00407D
:10BDEC00054B48F68F6253F8201001EA020242F428
:10BDFC00807243F820207047005C0040044B48F6EA
:10BE0C008F6253F8201001EA020243F82020704799
:10BE1C00005C0040044B48F68F6253F8201001EA96
:10BE2C00020243F820207047005C0040054B48F6A6
:10BE3C008F6253F8201001EA020242F4807243F838
:10BE4C0020207047005C0040054B48F68F6253F889
:10BE5C00201001EA020242F4807243F8202070475D
:10BE6C00005C0040044B48F68F6253F8201001EA46
:10BE7C00020243F820207047005C0040044B53F84A
:10BE8C00200000F03000102814BF00200120704763
:10BE9C00005C0040054B53F8200000F44050B0F516
:10BEAC00805F14BF00200120704700BF005C004081
:10BEBC00044B40F68F7253F8201001EA020243F84B
:10BECC0020207047005C0040044B48F60F7253F87A
:10BEDC00201001EA020243F820207047005C004069
:10BEEC00054B48F68F7253F8201001EA020242F417
:10BEFC00804243F820207047005C0040054B48F618
:10BF0C008F7253F8201001EA020242F0400243F80B
:10BF1C0020207047005C0040084B53F8202012F49E
:10BF2C00804F09D053F8201048F68F7201EA0202B4
:10BF3C0042F4804243F82020704700BF005C004070
:10BF4C00084B53F8202012F0400F09D053F8201062
:10BF5C0048F68F7201EA020242F0400243F82020B8
:10BF6C00704700BF005C0040054B10B553F82040F3
:10BF7C0048F68F7204EA02020A4343F8202010BDEF
:10BF8C00005C0040024B53F8200000F00F0070479B
:10BF9C00005C0040064B49081B6849009BB203EB50
:10BFAC00C00303F1005303F540535B001960704765
:10BFBC00505C0040054A064B1268490892B202EBED
:10BFCC00C002D3185B00490019607047505C0040F8
:10BFDC0004300020054B1B689BB203EBC00303F13C
:10BFEC00005303F540535B0018887047505C0040C9
:10BFFC00044A054B126892B202EBC002D3185B00E4
:10C00C0018887047505C004004300020044A054BEF
:10C01C00126892B202EBC002D3185B001960704731
:10C02C00505C0040023000203E2909D94B0911F028
:10C03C001F0F01D1013B9BB29B0243F4004305E06F
:10C04C004B0811F0010F18BF01339B0203607047BE
:10C05C000D4A0E4B126892B2D31803EBC0035B006F
:10C06C003E2909D94A0911F01F0F01D1013A92B2A8
:10C07C00920242F4004205E04A0811F0010F18BF89
:10C08C00013292021A607047505C0040063000206A
:10C09C00054A064B126892B202EBC002D3185B0041
:10C0AC0018688005800D7047505C004002300020FD
:10C0BC00054A064B126892B202EBC002D3185B0021
:10C0CC0018688005800D7047505C004006300020D9
:10C0DC000C4B30B51D681C68C0001FFA85FC8444ED
:10C0EC00A4B2094B00190CF1005CC3180CF5405CB0
:10C0FC00490852084FEA4C0049005B0052000160AD
:10C10C001A6030BD505C004004300020064B4908DA
:10C11C001B6849009BB203EBC00303F1005303F50A
:10C12C0040535B0019607047505C0040054A064B59
:10C13C001268490892B202EBC002D3185B004900A6
:10C14C0019607047505C004004300020054B1B68A0
:10C15C009BB203EBC00303F1005303F540535B00A8
:10C16C0018887047505C0040044A054B126892B224
:10C17C0002EBC002D3185B0018887047505C00407B
:10C18C0004300020012910B524D1254B25491B680A
:10C19C00C0009BB2591809184B003E2A09D9510905
:10C1AC0012F01F0F01D1013989B2890241F400410B
:10C1BC0005E0510812F0010F18BF01318902196016
:10C1CC001749194B096889B2CB18181840003E2A38
:10C1DC001ED913E0022922D1114BC0001C681B6828
:10C1EC00A4B21FFA83FC0F490F4B84440019411869
:10C1FC00634449005B000A601A6010E0530912F0B6
:10C20C001F0F01D1013B9BB29B0243F4004305E09D
:10C21C00530812F0010F18BF01339B02036010BDCD
:10C22C00505C0040023000200630002001291BD158
:10C23C001349144B096889B2CB1803EBC0004000BA
:10C24C003E2A09D9530912F01F0F01D1013B9BB2B1
:10C25C009B0243F4004305E0530812F0010F18BF92
:10C26C0001339B0203600AE0022908D10449054B03
:10C27C00096889B201EBC000C3185B001A607047F3
:10C28C00505C00400230002001291BD11349144B93
:10C29C00096889B2CB1803EBC00040003E2A09D9CB
:10C2AC00530912F01F0F01D1013B9BB29B0243F4C7
:10C2BC00004305E0530812F0010F18BF01339B0235
:10C2CC0003600AE0022908D10449054B096889B2C8
:10C2DC0001EBC000C3185B001A607047505C004053
:10C2EC0006300020054A064B126892B202EBC002DF
:10C2FC00D3185B0018688005800D7047505C0040B7
:10C30C0002300020054A064B126892B202EBC002C2
:10C31C00D3185B0018688005800D7047505C004096
:10C32C00063000200D4BC00019680D4A89B2411827
:10C33C008A185200128812F47C4F01D001200CE0B4
:10C34C001A68084B92B28018C3185B0018888005D5
:10C35C00800D002814BF022000207047505C004064
:10C36C000630002002300020012909D10B4A48F682
:10C37C008F7352F8201001EA030343F040030AE0E4
:10C38C0002290AD1054A48F68F7352F8201001EAA7
:10C39C00030343F4804342F820307047005C0040B4
:10C3AC0041EA0020704700BF030AC0B243EA0020F4
:10C3BC00704700BF01F10051013201F5405110B539
:10C3CC0049005208002308E010F803C06478013AD1
:10C3DC004CEA042C21F813C00233C418002AF3D100
:10C3EC0010BD00BF01F10051013201F5405110B5F3
:10C3FC0049005208002304E031F81340013AC452BA
:10C40C000233002AF8D110BD08B529E047F6FF70B9
:10C41C000860198801F00F018B0003F18043117043
:10C42C0003F5B843196889B211F4004F09D01868A4
:10C43C0040F68F7100EA0101196012780E4B013A37
:10C44C000BE011F0800F0BD0186848F60F7100EA62
:10C45C00010119601278094B013A53F822309847C0
:10C46C000749084B0868084A80B21880188800B23F
:10C47C000028CBDB08BD00BF4001002024010020B8
:10C48C00445C0040A2090020AA090020F8B59AE0FB
:10C49C0047F6FF761E601688564F06F00F06B3005F
:10C4AC0003F1804303F5B8433E70002E64D1276836
:10C4BC002668236807F4405C03EA000080F400500F
:10C4CC002060236806F0300003EA010181F02001AE
:10C4DC0021601388484A13F0100F1080A5F800C093
:10C4EC0004D023689BB213F0800F08D0226848F662
:10C4FC000F7302EA0303236000F0CEFA16E013F484
:10C50C00006F08D0226840F68F7302EA03032360A1
:10C51C0000F062FB0AE013F4004F54D0226840F69E
:10C52C008F7302EA0303236000F0F8F921682A886C
:10C53C004BF68F7301EA030312F4805F18BF83F488
:10C54C00805312F4005F2D4A18BF83F4005313601C
:10C55C00294B11681A8848F6BF7301EA030312F0DD
:10C56C00100F18BF83F0100312F0200F234A18BFCE
:10C57C0083F0200313603BE01C68A4B214F4004F5A
:10C58C000BD0196840F68F7201EA02021A603A78F1
:10C59C001B4B013A53F82230984714F0800F12D0FD
:10C5AC00144948F60F720B789B0003F1804303F596
:10C5BC00B843186800EA02021A600A78114B013A73
:10C5CC0053F822309847104B104A1D680B4C1FFA39
:10C5DC0085FCA2F800C0B2F800C04BF68F700FFAC1
:10C5EC008CFCBCF1000F48F6BF71094DFFF650AF43
:10C5FC00F8BD00BFAA090020E61C0020005C00402A
:10C60C004001002024010020445C0040A2090020CD
:10C61C00E41C0020074A022108B50748117207499B
:10C62C00074B086007490A60074A13601B68984764
:10C63C0008BD00BFB009002060010020CC0900201B
:10C64C0090000020100A0020A409002010B5074C0F
:10C65C0020B922684FF00103138205E0044B1B68DC
:10C66C001B68984720680A3010BD00BF100A0020D4
:10C67C00CC09002010B50A4B0A4A1B685178DA78AD
:10C68C0091420AD3997841B99C8834B99A72064B75
:10C69C001B685B689847204600E0022010BD00BF75
:10C6AC00100A00205C010020CC09002010B5074CBA
:10C6BC0020B922684FF00103138205E0044B1B687C
:10C6CC009B68984720680C3010BD00BF100A0020F2
:10C6DC00CC09002038B50E4C0E4B22681B68D17863
:10C6EC009B695079984723689A7A7AB170B91A790C
:10C6FC0062B99D7855B9084B1B68DB68984723686D
:10C70C0028465979DA78D9721A7300E0022038BDBC
:10C71C00100A0020A4090020CC09002008B502460C
:10C72C00244B20B91B684FF00201198240E0224AC9
:10C73C004FF000011B681180197811F07F0113D1A3
:10C74C005B7A13F0200F03D0117841F002011170C5
:10C75C0013F0400F184B15BF1A781A7822F001020B
:10C76C0042F001021A701EE0012921D0022901D0E9
:10C77C0000221DE0597911F0800F01F00F0306D053
:10C78C000E4951F8233003F03003102B06E00B490F
:10C79C0051F8233003F44053B3F5805F03D1137881
:10C7AC0043F001031370064B1B681B699847024A40
:10C7BC00104608BD100A0020E81C0020005C004058
:10C7CC00CC09002010B51E4B19684A7912F0800F65
:10C7DC0022F0800305D01B4850F8230000F03000F5
:10C7EC0004E0184850F8230000F44050164C94F81C
:10C7FC0000C0634522D24C8804BBF8B1897AE9B1F8
:10C80C0012F0800F09D00F4948F6BF7251F823007F
:10C81C0000EA020282F0100208E00A494BF68F721D
:10C82C0051F8230000EA020282F4805241F82320DE
:10C83C00064B1B689B699847002000E0022010BD46
:10C84C00100A0020005C00405C010020CC09002094
:10C85C0008B5064B1B685A7A42F020025A72044BF8
:10C86C001B68DB699847002008BD00BF100A002038
:10C87C00CC090020054B1A68538A18B98988CB1A41
:10C88C00138201E008681818704700BF100A0020D6
:10C89C0030B50E4B1C78002310E05FFA83FC4FEA96
:10C8AC008C0202F1804202F5B842156848F68F718D
:10C8BC0005EA010141EA0C0111600133A342ECD3FA
:10C8CC00034B40F08000186030BD00BF5C010020BD
:10C8DC004C5C0040704700BF08B50C4B002093F82F
:10C8EC002C10FFF7B5FB0A4B1B68187A082807D1E8
:10C8FC00084B4FF480521A80074B4FF010021A80ED
:10C90C00092814BF0020012008BD00BF90000020A2
:10C91C00100A0020E41C0020E61C002070B52D4BF2
:10C92C001C68237A032B01D0052B46D1A369228ADC
:10C93C00ABB1A2B1A58A954228BF154628469847A7
:10C94C00228A638A521BEB180646228263820020DD
:10C95C00FFF74EFB2A4601463046FFF743FD238A7C
:10C96C005BB11D4B4FF4405200201A800146FFF77B
:10C97C004DFB1A4B4FF030021A80A28A238A9A423E
:10C98C0003D8144B03221B6803E0124A1BB1136833
:10C99C0005221A720DE0126806211172104A1168F4
:10C9AC00104A89B28A18520013600C4B4FF03002B7
:10C9BC001A80084B1B681B7A06E0072B03D10A4B25
:10C9CC001B68DB6898470823024A12681372FFF74A
:10C9DC0083FF70BD100A0020E41C0020E61C002020
:10C9EC00505C004002300020A4090020F8B5244B14
:10C9FC001C68238A267ABBB9042E15D121482249FA
:10CA0C000278012A0BD1214C214A24680370A0B270
:10CA1C008218520013604FF030020A802BE04FF066
:10CA2C0010030B80072626E0A68AA2699E4234BF1B
:10CA3C0035461D462846B34294BF0426022690472D
:10CA4C0007460020FFF7C6FA2A4601463846FFF78C
:10CA5C00B1FC29460020FFF7D9FA638A228AEB1829
:10CA6C006382094B551B4FF0300225821A80094B0B
:10CA7C004FF440521A80024B1B681E72F8BD00BF67
:10CA8C00100A002045030020E61C0020505C0040EA
:10CA9C0002300020E41C002008B5144B1B681A7AE5
:10CAAC00022A01D0042A05D1FFF7A0FF0F4B1B6807
:10CABC001B7A14E0062A11D15A78052A0AD11A7861
:10CACC0012F07F0F06D1D878FFF7E2FE084B1B68F7
:10CADC001B6A9847074B1B689B6898470823034AB7
:10CAEC0012681372FFF7F8FE08BD00BF100A002091
:10CAFC00CC090020A409002038B5324B1B681878EB
:10CB0C0010F07F0004D15A7A22F020025A7258E0B9
:10CB1C00022855D15A88002A52D11A79002A4FD1AD
:10CB2C005A7912F0800F22F0800405D0264951F872
:10CB3C00241001F0300104E0234951F8241001F4D1
:10CB4C0040512248007884423AD2002938D09B7A4E
:10CB5C00002B35D012F0800F0FD01B4B53F8243024
:10CB6C0003F03003102B25D1E4B22046FFF7E8F98F
:10CB7C0020463021FFF7C4F81CE0134D55F8243043
:10CB8C0003F44053B3F5805F14D134B9104B2046F5
:10CB9C0093F82C10FFF75CFA02E02046FFF7BCF983
:10CBAC0055F824204BF68F7302EA030383F44053A9
:10CBBC0045F82430074B1B685B699847002000E060
:10CBCC00022038BD100A0020005C00405C010020EF
:10CBDC0090000020CC090020F7B58D4B8D4E1A68C3
:10CBEC0035688D4B92B2D3182A7A5B00092A1B68E0
:10CBFC001BD09BB203F1005303F540535B001C4662
:10CC0C0014F8012B03F10A072A705B786B70B4F8E7
:10CC1C000300FFF7C9FB6880B4F807003468FFF71E
:10CC2C00C3FBA08033687F88DF807A4C01212368A6
:10CC3C00DA8819725D78002A62D11A7812F07F02B4
:10CC4C002ED1092D02D1FFF715FD3BE0052D0DD19D
:10CC5C0093F90320002A4EDB9A78002A4BD19A884C
:10CC6C00002A48D19B7A002B37D044E0032D0BD1FE
:10CC7C00DA78012A27D19A882ABB5B7A13F0200F25
:10CC8C0021D0FFF7E5FD1DE0012D1CD1DA78012A3A
:10CC9C0019D19A88BAB95B7A13F0200F13D00AE035
:10CCAC00012A04D10B2D0ED1FFF714FD0AE0022A44
:10CCBC0009D1012D02D1FFF71FFF03E0032D02D193
:10CCCC00FFF780FD48B1554B28461B685B699847B8
:10CCDC00032801D109230FE068B94D4A504B126863
:10CCEC004FF0300192B2D3185B0000221A604D4B0A
:10CCFC001980062300E00823464A12681372E3E009
:10CD0C00062D18D11A7812F07F0F40F097809B787F
:10CD1C00012B03D1414B1B68DB696EE0022B03D165
:10CD2C003E4B1B681B6A68E0032B40F087803B4B33
:10CD3C001B685B6A61E0002D3CD1598800297DD1CC
:10CD4C005A6822F47F42B2F5003F77D11A7812F07C
:10CD5C007F0203D19B88002B70D129E0012A0BD1D3
:10CD6C0058792E4B1B689B699847002866D123681D
:10CD7C009B7A002B62D01BE0022A5FD15B7913F007
:10CD8C00800F03F00F0205D0274951F8221001F053
:10CD9C00300104E0244951F8221001F44051234899
:10CDAC00007882424AD213F0700F47D1002945D047
:10CDBC001F4B23E0082D05D11B7813F07F0F3DD1BD
:10CDCC001C4B1BE00A2D39D11A7802F07F02012A84
:10CDDC0034D19A7A002A31D0598800292ED15A6838
:10CDEC0022F47F42B2F5803F28D158790B4B1B6857
:10CDFC009B69984710BB104B00E0FBB1054A4FF004
:10CE0C00000112680020936151829847002020E0B5
:10CE1C00505C0040100A002004300020A4090020BF
:10CE2C0002300020E61C0020005C00405C01002069
:10CE3C0029C7000859C60008B9C60008244C254B60
:10CE4C0022681B6850781B699847032801D1236816
:10CE5C0006E01F4B4FF6FF711B681A8A8A4201D1FC
:10CE6C00092203E0022800D012B908221A722BE022
:10CE7C0093F90010002921DAD98801910198824296
:10CE8C0002D9019A1A8211E08A420FD2114909681B
:10CE9C0091F82C108A4201D2002105E092FBF1F0AE
:10CEAC0001FB102212B901210B4A1170094A1268B8
:10CEBC0092F82C209A82FFF799FD05E003221A7252
:10CECC00064B4FF440521A80FFF706FDFEBD00BF23
:10CEDC00100A0020A409002045030020E41C0020B7
:10CEEC00002383814FF416528380C38003814FF05B
:10CEFC000C030260438170470A8810B54C88B1F866
:10CF0C0004C0038AC98844EA020242EA0C0223F4F0
:10CF1C0070630A431B041B0C92B242EA03030382A4
:10CF2C0010BD00BF0023C380038043808380704703
:10CF3C0021B183899BB243F4005304E0838923F429
:10CF4C0000531B041B0C8381704700BF01F01F03AF
:10CF5C004FF0010CC1F3421161450CFA03F301D1FE
:10CF6C000C3004E0022901D1103000E014301AB169
:10CF7C00026842EA030302E0026822EA0303036048
:10CF8C00704700BF1AB1838A9BB2194303E0838AAE
:10CF9C009BB223EA01018182704700BF038A23F010
:10CFAC000F031B041B0C0382038A9BB241EA03038D
:10CFBC0003827047838923F400631B041B0C838159
:10CFCC0083899BB241EA03038381704721B1838932
:10CFDC009BB243F0020304E0838923F002031B0499
:10CFEC001B0C8381704700BF038A23F020031B04B2
:10CFFC001B0C0382038A9BB241EA03030382704732
:10D00C0021B1038A9BB243F4804304E0038A23F4E6
:10D01C0080431B041B0C0382704700BFC905C90D5C
:10D02C00818070478088C005C00D704783899BB292
:10D03C0043F0010383817047038BDBB20383038BC3
:10D04C009BB243EA01230383704700BF038B03F4B5
:10D05C007F430383038B9BB241EA03030383704733
:10D06C0021B1838A9BB243F0200304E0838A23F02E
:10D07C0020031B041B0C8382704700BF21B1838AE1
:10D08C009BB243F0100304E0838A23F010031B04CB
:10D09C001B0C8382704700BF21B1838A9BB243F083
:10D0AC00080304E0838A23F008031B041B0C83820F
:10D0BC00704700BF838A23F004031B041B0C83827C
:10D0CC00838A9BB241EA03038382704721B1838A2E
:10D0DC009BB243F0020304E0838A23F002031B0497
:10D0EC001B0C8382704700BF038819420CBF0020C1
:10D0FC0001207047C94389B2018070474FF0010C81
:10D10C00C1F3421201F01F0362450CFA03F301D183
:10D11C00828903E0022A0CBF028A828A92B21340EF
:10D12C00028892B20BB9184607E0090A012313FAD8
:10D13C0001F111420CBF002001207047090A0123A4
:10D14C008B40DB439BB20380704700BF038ACA88C5
:10D15C0023F440531B041B0C1343038283898A88DA
:10D16C0030B5044608890D4623F4B053498940EA8A
:10D17C00020223F00C030A431B041B0C92B242EA7A
:10D18C000303A381A38AAA8923F440731B041B0CF9
:10D19C00134387B0A38201A801F0E8F80E4B2A686C
:10D1AC009C420CBF049B039B19215943920064239E
:10D1BC00B1FBF2F1B1FBF3F21201100903FB1011F8
:10D1CC0009013231B1FBF3F303F00F0343EA02021E
:10D1DC0092B2228107B030BD0038014008B5214B16
:10D1EC0098422BD008D8A3F50063984216D003F5CB
:10D1FC008063984234D119E01B4B984226D003F53A
:10D20C00684398422CD101214FF4804001F020F961
:10D21C004FF48040002101F01BF921E04FF4003065
:10D22C00012101F023F94FF4003016E04FF4802077
:10D23C00012101F01BF94FF480200EE04FF4002087
:10D24C00012101F013F94FF4002006E04FF4801097
:10D25C00012101F00BF94FF48010002101F006F9C7
:10D26C0008BD00BF004C004000500040038803F094
:10D27C008F0303800388B1F806C04A889BB243EA47
:10D28C000C0313439BB203808B8883850B88038527
:10D29C00064B984203D003F50063984201D10B7AF8
:10D2AC0003864FF001038382704700BF002C0140BE
:10D2BC00038C2DE9F04123F001031B041B0C0384A8
:10D2CC00038C0A894C8823F002031C4E14431B0464
:10D2DC008288B1F806C0058B1B0CA4B2B04244EA9C
:10D2EC00030392B20C88ADB2A0F834C003D006F59B
:10D2FC000066B04218D18E894F89B1F80E804FF676
:10D30C00F77C03EA0C0C4CEA070748EA06064FF6D2
:10D31C00FB73898847F6FF4C02EA0C0C07EA0303FF
:10D32C00B2B20B4342EA0C024FF68F7105EA0101CF
:10D33C002143828001830384BDE8F081002C0140ED
:10D34C00038C2DE9F04123F010031B041B0C038408
:10D35C00028CB1F808C022F0200212048488120C4E
:10D36C004B8842EA0C1242EA0313A2B21B4C068B06
:10D37C00B1F806C0A0420D88B6B29BB2A0F838C076
:10D38C0003D004F50064A0421BD1B1F80A804FF61B
:10D39C007F748F8903EA040447F2FF3C02EA0C0C09
:10D3AC0044EA0814CA894FF6BF73898804EA030358
:10D3BC004CEA870C43EA01134CEA82023C469BB2CE
:10D3CC0092B248F6FF7106EA010141EA052189B2E1
:10D3DC00828001830384BDE8F08100BF002C0140F2
:10D3EC00038C2DE9F04123F480731B041B0C038484
:10D3FC00028CB1F808C022F4007212048488120C5A
:10D40C004B8842EA0C2242EA0323A2B21A4C868BC6
:10D41C00B1F806C0A0420D88B6B29BB2A0F83CC0D1
:10D42C0003D004F50064A0421BD1B1F80A804FF27E
:10D43C00FF748F8903EA040444F6FF7C02EA0C0CA7
:10D44C0044EA0824CA894FF6FF33898804EA0303A7
:10D45C004CEA071C43EA01234CEA02123C469BB2FD
:10D46C0092B24FF68F7106EA0101294382808183C3
:10D47C000384BDE8F08100BF002C0140038CF0B5A3
:10D48C0023F480531B041B0C0384B1F806C0078CD7
:10D49C000C8882880D89868B4B88A0F840C0DFF8F9
:10D4AC0048C0BFB2604592B2B6B203D00CF5006C66
:10D4BC00604505D192048989920C42EA811292B29C
:10D4CC004DF6FF7C07EA0C0C48F6FF7106EA0101E9
:10D4DC004CEA053C41EA04214CEA033389B29BB285
:10D4EC00828081830384F0BD002C0140B1F802C01E
:10D4FC000B888A884CEA0303B1F806C013430A89E7
:10D50C0043EA0C03B1F80AC013438A8943EA0C03BB
:10D51C0013439BB2A0F84430704700BF00234FF078
:10D52C00FF320372438082800380C380704700BF48
:10D53C000023C381038043808380C38003814381A4
:10D54C008381704700234FF00102038103804380E5
:10D55C008280C380704700BF002383810380438097
:10D56C008380C38003814381704700BF21B103884E
:10D57C009BB243F0010304E0038823F001039B05F5
:10D58C009B0D0380704700BF39B1B0F844306FEA8F
:10D59C0043436FEA53439BB203E0B0F844305B045F
:10D5AC005B0CA0F8443070471AB183899BB21943C5
:10D5BC0003E083899BB223EA01018181704700BF9C
:10D5CC00818270470A43A0F8482070471AB18389BA
:10D5DC009BB2194303E083899BB223EA0101818149
:10D5EC00704700BF038923F007031B041B0C038146
:10D5FC00704700BFB0F808C05FFA8CFC41EA0C0C15
:10D60C0042EA0C0C4CEA032C1FFA8CFCA0F808C064
:10D61C00704700BF10B50446FFF7ECFF23899BB29F
:10D62C0043F48043238110BD10B50446FFF7E2FF9D
:10D63C00238923F077031B041B0C43F0770323810E
:10D64C0010BD00BF01858282704700BF038823F0A4
:10D65C0070039B059B0D41EA03030380704700BFD9
:10D66C00038923F070031B041B0C41EA03030381A1
:10D67C00704700BF10B50446FFF7F2FF23899BB239
:10D68C0043F00703238110BD30B50489B0F818C0EE
:10D69C00058C2CF4407CADB22CF0030C24F0070468
:10D6AC004FEA0C4C25F0220542EA050524044FEA0A
:10D6BC001C4C45EA0315240C4CF4807C21434CF0A3
:10D6CC00010CADB20181A0F818C0058430BD00BFBB
:10D6DC00038B23F070031B041B0C41EA030303832D
:10D6EC00704700BF038B23F4E0431B041B0C43EA7D
:10D6FC0001239BB203837047838B23F070031B04BD
:10D70C001B0C41EA03038383704700BF838B23F414
:10D71C00E0431B041B0C43EA01239BB28383704739
:10D72C0021B103889BB243F0800304E0038823F00B
:10D73C0080039B059B0D0380704700BF21B183883C
:10D74C009BB243F0040304E0838823F004031B041E
:10D75C001B0C8380704700BF21B183889BB243F0C0
:10D76C00080304E0838823F008031B041B0C83804C
:10D77C00704700BF21B183889BB243F0010304E0E2
:10D78C00838823F001031B041B0C8380704700BFAC
:10D79C00038B23F008031B041B0C41EA03030383D4
:10D7AC00704700BF038B23F400631B041B0C43EA7C
:10D7BC0001239BB203837047838B23F008031B0464
:10D7CC001B0C41EA03038383704700BF838B23F454
:10D7DC0000631B041B0C43EA01239BB28383704739
:10D7EC00038B23F004031B041B0C41EA0303038388
:10D7FC00704700BF038B23F480631B041B0C43EAAC
:10D80C0001239BB203837047838B23F004031B0417
:10D81C001B0C41EA03038383704700BF838B23F403
:10D82C0080631B041B0C43EA01239BB28383704768
:10D83C00038B23F080031B041B0C41EA03030383BB
:10D84C00704700BF038B5B045B0C43EA01239BB264
:10D85C0003837047838B23F080031B041B0C41EA6A
:10D86C0003038383704700BF838B5B045B0C43EA29
:10D87C0001239BB283837047038C23F002031B04A8
:10D88C001B0C41EA03030384704700BF038C23F095
:10D89C0008031B041B0C41EA03030384704700BFFD
:10D8AC00038C23F020031B041B0C43EA01139BB2D3
:10D8BC0003847047038C23F080031B041B0C43EA86
:10D8CC0001139BB203847047038C23F400731B0475
:10D8DC001B0C43EA01239BB203847047038C23F493
:10D8EC0000631B041B0C43EA01239BB203847047A7
:10D8FC00038C23F400531B041B0C43EA01339BB22F
:10D90C000384704701238B408A40018C89B221EA41
:10D91C0003030384018C0A4392B20284704700BF54
:10D92C0004238B408A40018C89B221EA03030384CF
:10D93C00018C0A4392B20284704700BF01238B40D2
:10D94C00B0F820C010B51FFA8CFC2CEA030303843A
:10D95C0009B1082909D11830490844584FF68F737A
:10D96C0004EA0303435043580CE004391830C1F364
:10D97C004E01445848F6FF7304EA03034350120265
:10D98C00435892B243EA0202425010BD21B10388BF
:10D99C009BB243F0020304E0038823F002039B05CF
:10D9AC009B0D0380704700BF21B103889BB243F0ED
:10D9BC00040304E0038823F004039B059B0D038000
:10D9CC00704700BF21B183889BB243F0800304E011
:10D9DC00838823F080031B041B0C8380704700BFDB
:10D9EC00038823F008039B059B0D038003889BB2DF
:10D9FC0041EA030303807047838823F070031B0400
:10DA0C001B0C838083889BB241EA0303838070479D
:10DA1C00038923F007031B041B0C038103899BB2AE
:10DA2C0041EA030303817047038923F080031B043D
:10DA3C001B0C038103899BB241EA030303817047EA
:10DA4C008184704781857047818670470187704754
:10DA5C0081877047A0F84010704700BF038B23F0FC
:10DA6C000C031B041B0C0383038B9BB241EA0303C3
:10DA7C0003837047038B23F440631B041B0C038349
:10DA8C00038B9BB243EA01239BB20383704700BF15
:10DA9C00838B23F00C031B041B0C8383838B9BB2A3
:10DAAC0041EA030383837047838B23F440631B0495
:10DABC001B0C8383838B9BB243EA01239BB283832E
:10DACC00704700BF0388DBB2038003889BB241EA36
:10DADC0003030380704700BF808E80B2704700BF85
:10DAEC00008F80B2704700BF808F80B2704700BF3C
:10DAFC00B0F8400080B27047808C80B2704700BF95
:10DB0C00008D80B2704700BF038A19420CBF002001
:10DB1C0001207047C94389B201827047038A828908
:10DB2C0011EA030092B203D011420CBF0020012075
:10DB3C00704700BFC94389B201827047B0F820C05A
:10DB4C0010B52CF0010C4FEA0C4C4FEA1C4CA0F811
:10DB5C0020C0048BB0F820C0A4B21FFA8CFC24F0B7
:10DB6C00F30442EA04042CF0020C44EA03144CF0D3
:10DB7C00010C4CEA010CA4B20483A0F820C010BD27
:10DB8C00B0F820C010B52CF0100C4FEA0C4C4FEA3A
:10DB9C001C4CA0F820C0B0F818C0048C2CF4407CAD
:10DBAC00A4B24FEA0C5C4FEA1C5C24F020044CEA53
:10DBBC00022C44F010044CEA033C44EA01141FFA12
:10DBCC008CFCA4B2A0F818C0048410BD38B50D4666
:10DBDC00602D1146044603D10122FFF7D1FF02E06C
:10DBEC000122FFF7ABFF29462046FFF739FD2389B9
:10DBFC009BB243F00703238138BD00BFF8B50C4638
:10DC0C00A2884988B4F800C0054600290CBF022739
:10DC1C000027012A0CBF022601262389BCF1000F24
:10DC2C0010D1FFF78BFF2846E188FFF717FF284636
:10DC3C00394632462389FFF7A3FF2846E188FFF7D0
:10DC4C0019FF0FE0FFF79CFF2846E188FFF712FF52
:10DC5C002846394632462389FFF770FF2846E1886B
:10DC6C00FFF7FCFEF8BD00BF38B50B880C46054627
:10DC7C004BB94988A2882389FFF760FF2846E188C1
:10DC8C00FFF7ECFE53E0042B09D14988A2882389C5
:10DC9C00FFF776FF2846E188FFF7ECFE47E0082BFC
:10DCAC00B1F802C0B1F804E0098920D1028C22F449
:10DCBC0080721204120C0284838B028C9BB292B27F
:10DCCC0023F0F30322F4007243EA011142EA0C2C14
:10DCDC0089B21FFA8CFC41EA0E0E4CF4807CA0F841
:10DCEC001CE0A0F820C0E188FFF7D2FE1FE0028CF8
:10DCFC0022F480521204120C0284838B028C23F4C3
:10DD0C00407392B21B051B0D22F4005243EA0E2302
:10DD1C0042EA0C3C43EA01331FFA8CFC9BB24CF4F4
:10DD2C00805C8383A0F820C0E188FFF7BDFE38BD7E
:10DD3C0008B52D4B984237D00BD8A3F50063984209
:10DD4C0026D003F58063984228D0B0F1804F4AD199
:10DD5C0018E0264B984233D004D8A3F58063984240
:10DD6C0041D127E0224B984204D003F5006398423E
:10DD7C0039D12EE04FF40060012100F069FB4FF423
:10DD8C0000602DE00120014600F070FB01201CE03A
:10DD9C000220012100F06AFB022016E00420012180
:10DDAC0000F064FB042010E00820012100F05EFB71
:10DDBC0008200AE01020012100F058FB102004E09C
:10DDCC002020012100F052FB2020002100F04EFB0E
:10DDDC0009E04FF40050012100F03AFB4FF40050E1
:10DDEC00002100F035FB08BD000C00400014004081
:10DDFC00002C0140042804D1054B1A6842F004029F
:10DE0C0003E0034B1A6822F004021A60704700BF4B
:10DE1C0010E000E0014B5860704700BF10E000E0DC
:10DE2C00012804D1084B1A6842F0010206E010F1F7
:10DE3C00020F05D1044B1A6822F001021A6002E0AD
:10DE4C00014B00229A60704710E000E020B1054BB6
:10DE5C001A6842F0020203E0024B1A6822F0020236
:10DE6C001A60704710E000E0014B9868704700BFE3
:10DE7C0010E000E0C308022B0BBF044B034B1B68E4
:10DE8C00DB6833FA00F000F00100704710E000E0AE
:10DE9C000B884A88B1F804C01A43CB8842EA0C02BA
:10DEAC00B1F808C01A434B8930B542EA0C028D898F
:10DEBC00B0F800C0CC891A432A4322430CF44153D6
:10DECC0013439BB20380838B23F400631B041B0C52
:10DEDC0083830B8A038230BD00234FF00702C3817A
:10DEEC000282038043808380C380038143818381CA
:10DEFC00704700BF00234381038043808380C3802D
:10DF0C004FF002030381704721B103889BB243F0A9
:10DF1C00400304E0038823F040031B041B0C038024
:10DF2C00704700BF21B1838B9BB243F4806304E044
:10DF3C00838B23F480631B041B0C8383704700BF0B
:10DF4C000909012313FA01F189B21AB183889BB232
:10DF5C00194303E083889BB223EA01018180704757
:10DF6C001AB183889BB2194303E083889BB223EADE
:10DF7C0001018180704700BF81817047808980B228
:10DF8C00704700BF4FF6FF63994205D003889BB2E0
:10DF9C0043F48073038002E00388194001807047CA
:10DFAC0021B183889BB243F0040304E0838823F0FF
:10DFBC0004031B041B0C8380704700BF038823F4ED
:10DFCC0000631B041B0C038003889BB241EA030310
:10DFDC000380704703889BB243F4805303807047DF
:10DFEC0021B103889BB243F4005304E0038823F46B
:10DFFC0000531B041B0C0380704700BF012914BF86
:10E00C00008B808A80B27047008A80B2704700BF54
:10E01C00B1F5804F04D103889BB243F4804304E0F4
:10E02C00038823F480431B041B0C0380704700BF40
:10E03C00038919420CBF002001207047202906D10A
:10E04C00038903889BB243F04003038008E0402916
:10E05C0001D0082901D1038902E0C94389B20181A9
:10E06C00704700BF012301F00F0213FA02F2B0F85F
:10E07C0004C000891FFA8CFC80B2104006D009093C
:10E08C008B401CEA030F0CBF00200120704700BF1F
:10E09C00552906D1038903889BB243F040030380C2
:10E0AC000DE0562901D0532901D1038907E001F075
:10E0BC000F01012313FA01F1C94389B201817047A1
:10E0CC00838BF0B523F47A6323F01F031B041B0C22
:10E0DC0083834FF0020303840B89868B022B87B05A
:10E0EC0004460D46B6B201D1002225E001A88F8866
:10E0FC0000F03CF9EB88002F0CBF01270227B3F589
:10E10C00007F2989019A06D1A3F5FB7353430902B9
:10E11C00B3FBF1F305E00A2349015A434F43B2FB29
:10E12C00F7F305330A229BB2B3FBF2F303F00102BF
:10E13C001202C3F34F0392B2991E89B2FE2928BF73
:10E14C00002228BF0223E98842EA03030B439BB257
:10E15C0023842B886A8846EA0303A98843F4006366
:10E16C0013436A890B4313439BB2A38307B0F0BDDF
:10E17C0008B5154B98421BD003F57443984204D054
:10E18C00A3F5784398421DD10AE001214FF4805049
:10E19C0000F05EF94FF48050002100F059F911E0C5
:10E1AC004FF48040012100F061F94FF4804006E00B
:10E1BC004FF40040012100F059F94FF400400021C8
:10E1CC0000F054F908BD00BF003C00400D4B0E4A56
:10E1DC00196841F001011960596801EA02025A609C
:10E1EC001A6822F0847222F480321A601A6822F4BF
:10E1FC0080221A605A6822F4FE025A6000229A6049
:10E20C00704700BF001002400000FFF80C4BB0F547
:10E21C00803F1A6822F480321A601A6822F4802235
:10E22C001A6003D0B0F5802F08D103E01A6842F4CD
:10E23C00803202E01A6842F4A0221A60704700BFD4
:10E24C0000100240034B1A6822F0F80242EAC002A6
:10E25C001A60704700100240014B1860704700BFF5
:10E26C0000004242044B5A6822F47C1240EA02023B
:10E27C000A435A60704700BF00100240014B1860FF
:10E28C00704700BF60004242034B5A6822F0030201
:10E29C0040EA02025A60704700100240024B586874
:10E2AC0000F00C00704700BF00100240034B5A688E
:10E2BC0022F0F00240EA02025A607047001002405D
:10E2CC00034B5A6822F4E06240EA02025A6070473B
:10E2DC0000100240034B5A6822F4605242EAC0021A
:10E2EC005A6070470010024019B1054B1A78104360
:10E2FC0003E0034B1A7822EA00001870704700BF45
:10E30C0009100240014B1860704700BFD800424210
:10E31C00034B5A6822F4404240EA02025A607047AA
:10E32C0000100240064B002201281A701A7002D00D
:10E33C00042804D101E0187001E005221A7070471E
:10E34C0020100240014B1860704700BF800442420D
:10E35C00024B1A6A40EA02021A627047001002402D
:10E36C00014B1860704700BF3C0442421F4B10B574
:10E37C005A6802F00C02042A13D0082A11D15A68E8
:10E38C005968C2F38342023211F4803F03D05B68B8
:10E39C0013F4003F01D0164B00E0164B5A430260B9
:10E3AC0001E0144B0360114A134B51680468C1F32C
:10E3BC000311595C34FA01F141605468C4F3022C26
:10E3CC0013F80C4031FA04F484605468C4F3C22C82
:10E3DC0013F80CC021FA0CF1C1605268C2F38132FF
:10E3EC009B181B7CB1FBF3F1016110BD00100240C6
:10E3FC0000093D0000127A00C403010819B1054B55
:10E40C005A69104303E0034B5A6922EA0000586131
:10E41C00704700BF0010024019B1054B9A691043B8
:10E42C0003E0034B9A6922EA00009861704700BF31
:10E43C000010024019B1054BDA69104303E0034B9D
:10E44C00DA6922EA0000D861704700BF0010024070
:10E45C0019B1054BDA68104303E0034BDA6822EA82
:10E46C000000D860704700BF0010024019B1054B86
:10E47C001A69104303E0034B1A6922EA0000186181
:10E48C00704700BF00100240014B1860704700BF7E
:10E49C0040044242014B1860704700BF4C0042429E
:10E4AC00014B1870704700BF071002404309012B45
:10E4BC0002D1084B1B6805E0022B0BBF054B054B2B
:10E4CC001B6A5B6A00F01F0033FA00F000F00100D9
:10E4DC00704700BF0010024008B53120FFF7E6FF7F
:10E4EC00094B18705A6801325A601A7822B95A6866
:10E4FC0040F2FF139A42F0D13120FFF7D7FF0038DA
:10E50C0018BF012008BD00BF48030020024B5A6A07
:10E51C0042F080725A62704700100240034B9B68B5
:10E52C0018420CBF00200120704700BF00100240B1
:10E53C00014B1870704700BF0A1002400B4B4FF094
:10E54C00FF316FF07042C3F88010C3F88420C3F819
:10E55C008011C3F88421002303F1C001034A013365
:10E56C0000200F2B42F82100F6D1704700E100E0AB
:10E57C00094B4FF020605860084800224FF0FF31E3
:10E58C009A60D8601A615A619A61DA611A625A62A9
:10E59C009962D9621963704700ED00E00000FA053A
:10E5AC0040F0BE60024B40F42020D860704700BFA2
:10E5BC0000ED00E030B5C27803787AB31C4A41789C
:10E5CC00D2684FF00F0CD243C2F302222CFA02FC99
:10E5DC00C2F104029140807803F003020CEA000CB3
:10E5EC004CEA010CD2004FEA0C1CFF2090400CFAB4
:10E5FC0002FC012403F01F02944099080D4AC0311B
:10E60C0052F821500CEA000C25EA00004CEA0000FC
:10E61C005B0942F8210042F8234008E003F01F0296
:10E62C00012191405B09034A203342F8231030BD8D
:10E63C0000ED00E000E100E00023C37003704370C4
:10E64C0083707047024B5868C0F30930704700BFA5
:10E65C0000ED00E0012200F01F0312FA03F3400961
:10E66C00044A403052F820001840984214BF002051
:10E67C000120704700E100E0014B1860704700BFBB
:10E68C0000EF00E000F01F0301229A404009024B0A
:10E69C00603043F82020704700E100E0024B5868DE
:10E6AC008005800D704700BF00ED00E0012200F0F6
:10E6BC001F0312FA03F34009044A803052F8200079
:10E6CC001840984214BF00200120704700E100E080
:10E6DC00014B1868704700BF00ED00E021F060416D
:10E6EC0021F07F01014B01439960704700ED00E080
:10E6FC00014A024BDA6070470400FA0500ED00E0B5
:10E70C00014A024BDA6070470100FA0500ED00E0A7
:10E71C0019B1054B1A69104303E0034B1A6922EA3D
:10E72C0000001861704700BF00ED00E000F01F0012
:10E73C00012313FA00F019B1044B5A6A104303E099
:10E74C00024B5A6A22EA00005862704700ED00E062
:10E75C00144B70B5DC684FF0FF0CE443C4F3022497
:10E76C002CFA04F5C4F1040411FA04F4C0F30126E4
:10E77C00F6000CFA06FC02EA050545EA040424013D
:10E78C0014FA06F6C0F38110063053F8202022EA62
:10E79C000C0243F8202053F82020164343F8206045
:10E7AC0070BD00BF00ED00E0C0F383200123834067
:10E7BC00044A506A03EA0000984214BF002001206A
:10E7CC00704700BF00ED00E000F01F000122824006
:10E7DC00024B59680A435A60704700BF00ED00E0D5
:10E7EC0000F01F020123013A13FA02F2024B59689E
:10E7FC000A435A60704700BF00ED00E0C0F383305D
:10E80C0001238340044A506A03EA0000984214BF73
:10E81C0000200120704700BF00ED00E0C0F38143F1
:10E82C0013B90A4BD86A10E0012B0CD1074AC0F37C
:10E83C000153906ADA00D040022B14BF00F00F0095
:10E84C0000F0FF0001E0014B186B704700ED00E099
:10E85C0010F4800F0BBF024B014B586B986B704739
:10E86C0000ED00E008B5F5F77BFC08BD08B500012C
:10E87C00F5F773FC08BD00BF08B5F5F76CFC08BDD7
:10E88C0008B5F5F766FC08BD08B5F5F760FC08BDE2
:10E89C0008B5F5F75AFC08BDCB78F0B513F0100F9E
:10E8AC0018BF8A78098803F00F0C18BF4CEA020CC9
:10E8BC0011F0FF0F1AD0046800220126964006EAD8
:10E8CC000105B5420ED196000F27B7400CFA06F69B
:10E8DC0024EA07043443282B01D1456102E0482B7C
:10E8EC0008BF05610132082AE7D10460FF291CD951
:10E8FC004468002202F108050126AE4006EA010533
:10E90C00B5420ED196000F27B7400CFA06F624EA52
:10E91C0007043443282B01D1456102E0482B08BF82
:10E92C0005610132082AE5D14460F0BD0423C370AF
:10E93C00022383704FF0FF330380704783681942C2
:10E94C000CBF002001207047806880B2704700BF68
:10E95C00C36819420CBF002001207047C06880B208
:10E96C00704700BF01617047416170470AB1016196
:10E97C0000E04161704700BFC160704741F48033D3
:10E98C00836181618361836983697047064A10B52D
:10E99C0014684FF6807341EA001104EA030341EA5C
:10E9AC000303136010BD00BF00000140014B186051
:10E9BC00704700BF1C0020420304154A00F4401CA1
:10E9CC001B0CBCF5401F30B5546806D1556824F0BB
:10E9DC00706425F07065556011E010F4801F06D04E
:10E9EC00C0F303424FF0030C0CFA02F203E0420DA9
:10E9FC00120113FA02F224EA020444F0706419B111
:10EA0C00400D000183401C43014B5C6030BD00BFD6
:10EA1C000000014001F003039B000F229A4010FA02
:10EA2C0003F310B58908074C023154F8210020EA91
:10EA3C00020244F8212054F82120134344F82130D9
:10EA4C0010BD00BF000001400120014608B5FFF7D2
:10EA5C00FFFC01200021FFF7FBFC08BD08B5264B8D
:10EA6C0098422BD00CD8A3F5006398421AD003F52A
:10EA7C00806398421CD0A3F5006398423AD10BE016
:10EA8C001E4B984226D003F58063984228D0A3F5FC
:10EA9C00006398422ED117E004200121FFF7D8FC27
:10EAAC00042024E008200121FFF7D2FC08201EE0FE
:10EABC0010200121FFF7CCFC102018E020200121B0
:10EACC00FFF7C6FC202012E040200121FFF7C0FC1C
:10EADC0040200CE080200121FFF7BAFC802006E0EA
:10EAEC004FF480700121FFF7B3FC4FF480700021CC
:10EAFC00FFF7AEFC08BD00BF00140140001C014034
:10EB0C00044B1A6802F038021A601A6840EA0202D2
:10EB1C001A60704700200240044B1A6822F0080269
:10EB2C001A601A6840EA02021A607047002002401C
:10EB3C00044B1A6822F010021A601A6840EA0202AA
:10EB4C001A60704700200240044B00221A605A6081
:10EB5C009A60DA60024A5A61704700BF00040140B3
:10EB6C00FFFF0700837930B5016802794BB3184B6E
:10EB7C00CC431D6890F805C004EA05051D605D686E
:10EB8C002C405C60D45844EA0101D150026898686A
:10EB9C00D14301EA00009860D8680140BCF1100F25
:10EBAC00D96007D1996811439960D96841EA02028A
:10EBBC00DA600BE05CF8031041EA02024CF8032027
:10EBCC0004E0034BD05820EA0101D15030BD00BF06
:10EBDC000004014000230C22837142710360037115
:10EBEC00704700BF024B1A6940EA02021A61704773
:10EBFC0000040140034B5B6918420CBF002001204C
:10EC0C00704700BF00040140014B5861704700BFC2
:10EC1C0000040140054B1A685B69034001D118469A
:10EC2C0003E010420CBF002001207047000401409B
:10EC3C00014B5861704700BF00040140026800237B
:10EC4C0022F001020260036043608360C3602D4BBD
:10EC5C00984233D011D83C3B984229D006D8283B57
:10EC6C00984221D0143398424BD11FE0264B984246
:10EC7C0020D01433984244D11EE0244B98422CD01F
:10EC8C0008D8A3F5677398421DD003F562739842B8
:10EC9C0037D11DE01E4B984229D0143398422BD00B
:10ECAC00283B98422DD11DE01A4B12E0194B15E070
:10ECBC00184B18E0174B1BE0164B1EE0154B5A680F
:10ECCC0042F470021CE0134B5A6842F0706217E079
:10ECDC00114B5A6842F00F0212E00F4B5A6842F087
:10ECEC00F0020DE00C4B5A6842F4706208E00A4BDB
:10ECFC005A6842F4704203E0074B5A6842F470229F
:10ED0C005A6070476C000240440002401C040240F0
:10ED1C004404024000000240000402408A6870B5BE
:10ED2C000C6A0B6944EA02024C691A438B69224350
:10ED3C00CC6905684E6A42EA030323438C6A334369
:10ED4C0025F4FE4C23432CF0F00C43EA0C03036037
:10ED5C00CB6843600B6883604B68C36070BD00BFB9
:10ED6C0000238362036043608360C360036143617B
:10ED7C008361C36103624362704700BF19B10368CA
:10ED8C0043F0010302E0036823F0010303607047C2
:10ED9C0012B10368194302E0036823EA0101016020
:10EDAC00704700BF406880B2704700BF10F0805FB2
:10EDBC0014BF044B044B1B6803420CBF0020012002
:10EDCC00704700BF000402400000024010F0805F5A
:10EDDC0014BF024B024B5860704700BF0004024046
:10EDEC000000024010F0805F14BF044B044B1B6802
:10EDFC0003420CBF00200120704700BF00040240FA
:10EE0C000000024010F0805F14BF024B024B5860B0
:10EE1C00704700BF0004024000000240374B012243
:10EE2C001A605A6812F0010201D1104664E00278AF
:10EE3C00012A0BBF1A681A6842F0800222F0800285
:10EE4C001A604378012B04D12C4B1A6842F0400213
:10EE5C0003E02A4B1A6822F040021A608378012BD7
:10EE6C0004D1264B1A6842F0200203E0234B1A68A7
:10EE7C0022F020021A60C378012B04D11F4B1A68B0
:10EE8C0042F0100203E01D4B1A6822F010021A60C7
:10EE9C000379012B04D1194B1A6842F0080203E0E4
:10EEAC00164B1A6822F008021A604379012B04D120
:10EEBC00124B1A6842F0040203E0104B1A6822F05D
:10EECC0004021A608279C37990F808C0920742EA6A
:10EEDC0003624189437A42EA0C4242EA0352013905
:10EEEC00064B0A43DA611A6822F001021A6058686C
:10EEFC0080F0010000F00100704700BF006400408A
:10EF0C0090F800C0012202FA0CF23B4B2DE9F045BF
:10EF1C00D3F8004292B244F00104C3F80042D3F893
:10EF2C001C42D14301EA0404C3F81C428478A4B9FE
:10EF3C000CF1480CD3F80C72B0F80AA0C688B0F8E3
:10EF4C00088085884FEACC0404F1804446EA0A46DE
:10EF5C0045EA084501EA070715E0012C1AD10CF126
:10EF6C00480CD3F80C72B0F804A0C688B0F808802E
:10EF7C0045894FEACC0404F1804446EA0A4645EA46
:10EF8C00084542EA070704F5C844C3F80C7243F875
:10EF9C003C60656043782BB9174BD3F8044201EA07
:10EFAC00040404E0144BD3F8044242EA0404C3F80A
:10EFBC000442838923B9104BD3F81442214006E054
:10EFCC00012B06D10C4BD3F8141242EA0101C3F801
:10EFDC001412837B012B05D1074BD3F81C120A4367
:10EFEC00C3F81C22044BD3F8002222F00102C3F810
:10EFFC000022BDE8F08500BF0064004003220272CD
:10F00C00013A002342724FF00102C3714281037036
:10F01C0043708370C370037143718371704700BF79
:10F02C0019B1054B5A69104303E0034B5A6922EAA4
:10F03C0000005861704700BF00640040364B70B54B
:10F04C009968024611F0806F01D000200CE099689D
:10F05C0011F0006F01D0012006E09B6813F0805F77
:10F06C0001D1042056E002202B4B00F118010901BC
:10F07C00CC5804F00104CC50157A92F809C035B97B
:10F08C00146864051460CD584CEA050C07E054680C
:10F09C0045EA0C0CE4005460CE584CEA060C4CEAE1
:10F0AC000404CC50947A00F1180C4FEA0C1C04F0B8
:10F0BC000F040CF18043947203F5C8435D680101A1
:10F0CC0025F00F055D605D6801F180412C435C60AB
:10F0DC00537B947BD57A1B0443EA0463147B2B4348
:10F0EC0043EA042301F5C841C1F88831557C937C6F
:10F0FC00D47B2D0445EA0365137C45EA040242EAFD
:10F10C000322054BC1F88C215CF8032042F001026C
:10F11C004CF8032070BD00BF00640040012810D0E3
:10F12C0002D302282CD11AE0164A9168936892688F
:10F13C0001F0010103F0020343EA8103C2F3806290
:10F14C001AE0104A9368916803F48073926801F492
:10F15C0000719B0943EA1123C2F3C0620CE0094A17
:10F16C009368916803F48033926801F400319B0B2F
:10F17C0043EA1143C2F300721343034AD05C704755
:10F18C000023FAE700640040D8030108012808D0E6
:10F19C0002D302280FD109E0074B9A6842F0800293
:10F1AC0008E0054B9A6842F4004203E0024B9A686F
:10F1BC0042F400029A6070470064004018B9044B96
:10F1CC002022DA6002E0024B20221A61704700BF55
:10F1DC000064004010B9064BD86805E0012801D046
:10F1EC00002003E0024B186900F00300704700BFD9
:10F1FC0000640040254B00F11B02120110B5D458DD
:10F20C0004F004040C721CB9D3585B0D0B6002E0C3
:10F21C00D358DB084B6000F11B021C4B1201D35876
:10F22C0002F1804203F002034B7202F5C8425468AB
:10F23C00030104F00F0C81F80AC0526803F18043FB
:10F24C00120ACA7403F5C843D3F8B821CA72D3F8AA
:10F25C00B821120A0A73D3F8B821120C4A73D3F8E6
:10F26C00B821120E8A73D3F8BC21CA73D3F8BC210F
:10F27C00120A0A74D3F8BC21120C4A74D3F8BC31AC
:10F28C001B0E8B74FFF79AFF10BD00BF006400408B
:10F29C00044B1A6842F002021A601868C0F340006E
:10F2AC00704700BF00640040054B1A6822F0020250
:10F2BC001A60186880F00200C0F34000704700BF6D
:10F2CC0000640040034B9B6918420CBF00200120D6
:10F2DC00704700BF00640040024B9A6922EA0002AA
:10F2EC009A61704700640040202831D00CD8062861
:10F2FC0020D004D8042825D0052844D118E00728AC
:10F30C001DD008283FD11FE0B0F5007F2BD005D8C9
:10F31C0040281FD0B0F5807F35D11FE0B0F5803F7D
:10F32C002CD0B0F5003F2BD0B0F5806F2BD11FE067
:10F33C00012201E04FF48072134B9A6023E04FF4EA
:10F34C008032F9E7082200E010220F4BDA601AE055
:10F35C00082200E010220C4B1A6114E00A4B9A6947
:10F36C0022F0010208E0084B9A6922F0020203E045
:10F37C00054B9A6922F004029A6104E0082200E02D
:10F38C001022014B5A6070470064004001420CBFD0
:10F39C0000200120704700BF202808B532D00CD8BF
:10F3AC00062821D004D8042826D0052818D119E025
:10F3BC0007281ED0082813D120E0B0F5007F29D0F3
:10F3CC0005D8402820D0B0F5807F09D120E0B0F5D9
:10F3DC00803F27D0B0F5003F22D0B0F5806F1BD016
:10F3EC00002024E0012101E04FF48071104B98685B
:10F3FC001BE04FF48031F9E7082100E010210C4BA1
:10F40C00D86812E0082100E01021094B18690CE0C3
:10F41C00012102E0022100E00421054B986904E07F
:10F42C00102100E00821024B5868FFF7AFFF08BD20
:10F43C0000640040012108B54FF00070FFF716F88A
:10F44C004FF000700021FFF711F808BD436830B58C
:10F45C0023F470230C680A7923F48073234343EA62
:10F46C000223436082688D68CC680A4B45EA040C21
:10F47C0002EA03034A794CEA030343EA420383603A
:10F48C000B7CC26A013B22F47002DBB242EA0353EA
:10F49C00C36230BDFDF7F1FF002301220274C3608B
:10F4AC000360037143718360704700BF19B18368B7
:10F4BC0043F0010302E0836823F00103836070478B
:10F4CC0019B1836843F4807302E0836823F480737A
:10F4DC0083607047C9B212B14368194302E04368B4
:10F4EC0023EA010141607047836843F0080383609D
:10F4FC00704700BF8068C0F3C0007047836843F05A
:10F50C0004038360704700BF8068C0F380007047BD
:10F51C0019B1836843F4A00302E0836823F4A003C9
:10F52C00836070478068C0F380507047436801392E
:10F53C0023F4604343EA41334360704719B1436895
:10F54C0043F4006302E0436823F4006343607047B4
:10F55C00092930B511D94FF0030C0CFB01FC072520
:10F56C00ACF11E0C05FA0CF503FA0CFCC46824EA89
:10F57C00050343EA0C03C3600EE04FF0030C0CFBD5
:10F58C0001FC072505FA0CF503FA0CFC046924EAC6
:10F59C00050343EA0C030361062A0DD80523013A3F
:10F5AC005A434FF01F0C0CFA02FC9140436B23EAB8
:10F5BC000C020A4342631CE00C2A0DD805235A4363
:10F5CC004FF01F0C233A0CFA02FC9140036B23EA18
:10F5DC000C020A4302630CE005235A434FF01F0C44
:10F5EC00413A0CFA02FC9140C36A23EA0C020A432A
:10F5FC00C26230BD19B1836843F4801302E08368A2
:10F60C0023F4801383607047C06C80B2704700BFD6
:10F61C00014B1868704700BF4C24014019B1436876
:10F62C0043F4806302E0436823F4806343607047D3
:10F63C0019B1436843F4805302E0436823F48053C8
:10F64C0043607047836823F4E04341EA030383601B
:10F65C00704700BF19B1836843F4004302E083682C
:10F66C0023F400438360704719B1836843F4021399
:10F67C0002E0836823F40213836070478068C0F350
:10F68C0040507047092930B511D94FF0030C0CFBD1
:10F69C0001FC0725ACF11E0C05FA0CF503FA0CFC69
:10F6AC00C46824EA050343EA0C03C3600EE04FF080
:10F6BC00030C0CFB01FC072505FA0CF503FA0CFCFA
:10F6CC00046924EA050343EA0C030361836BC3F367
:10F6DC00015CCCEB020202324FF0050CD2B20CFBF7
:10F6EC0002F20CF11A0C0CFA02FC914023EA0C0306
:10F6FC000B43836330BD00BF836B013923F440138C
:10F70C0043EA0153836370470A50704728304058CE
:10F71C0080B27047436823F4400323F4007341EA3A
:10F72C0003034360704700BF41628262704700BFB1
:10F73C00436823F01F0341EA03034360704700BF93
:10F74C0020B1054B9A6842F4000203E0024B9A6820
:10F75C0022F400029A6070470024014003681942A9
:10F76C000CBF002001207047C9430160704700BFE7
:10F77C004368006810EA112004D0C9B219420CBFCA
:10F78C0000200120704700BF6FEA11210160704713
:10F79C0008B5134B98420FD003F5A053984213D0E1
:10F7AC00A3F5C053984219D14FF400700121FEF714
:10F7BC004FFE4FF400700EE04FF480600121FEF715
:10F7CC0047FE4FF4806006E04FF400400121FEF745
:10F7DC003FFE4FF400400021FEF73AFE08BD00BF8B
:10F7EC0000280140032A2DE9F0070BD83AB1002379
:10F7FC0011F803C000F803C001339342F8D1BDE8FF
:10F80C00F007704782180C46034603E014F8011CFD
:10F81C0003F8011C03F003061946A4460133013416
:10F82C00002EF3D11CF00304634608BFC1EB020C9D
:10F83C0068D06542C4F1040A0CEB050733464FEA65
:10F84C00CA0A5CF805604FEAC408551A08E057F874
:10F85C00044F264604FA0AF449EA0404CC50043353
:10F86C005C18032D26FA08F9A5F104050CEB030628
:10F87C00EDDC002302E0F15CE154013319199142F3
:10F88C00F9D3BCE753F8404C41F8404C53F83C4C8E
:10F89C0041F83C4C53F8384C41F8384C53F8344C44
:10F8AC0041F8344C53F8304C41F8304C53F82C4C54
:10F8BC0041F82C4C53F8284C41F8284C53F8244C64
:10F8CC0041F8244C53F8204C41F8204C53F81C4C74
:10F8DC0041F81C4C53F8184C41F8184C53F8144C84
:10F8EC0041F8144C53F8104C41F8104C53F80C4C94
:10F8FC0041F80C4C53F8084C41F8084C53F8044CA4
:10F90C0041F8044C1C460D4640334031BCF13F0FCE
:10F91C00ACF1400CB6DC21462B46541B0FE051F8E1
:10F92C00105C43F8105C51F80C5C43F80C5C51F81B
:10F93C00085C43F8085C51F8045C43F8045C0F2C39
:10F94C000D469C4601F1100103F11003A4F11004C3
:10F95C00E5DCCCEB0201002303E0EC584CF803404F
:10F96C0004335E19032903EB0C04A1F10401F4DC4C
:10F97C007FE700BF80F0004002E000BF81F0004153
:10F98C0042001FBF5FEA410392EA030F7FEA226C39
:10F99C007FEA236C6AD04FEA1262D2EB1363C1BFC9
:10F9AC00D218414048404140B8BF5B42192B88BF38
:10F9BC00704710F0004F40F4000020F07F4018BF5B
:10F9CC00404211F0004F41F4000121F07F4118BF7B
:10F9DC00494292EA030F3FD0A2F1010241FA03FC23
:10F9EC0010EB0C00C3F1200301FA03F100F000430B
:10F9FC0002D5494260EB4000B0F5000F13D3B0F1D3
:10FA0C00807F06D340084FEA310102F10102FE2A41
:10FA1C0051D2B1F1004F40EBC25008BF20F00100B1
:10FA2C0040EA03007047490040EB000010F4000F5F
:10FA3C00A2F10102EDD1B0FA80FCACF1080CB2EBF2
:10FA4C000C0200FA0CF0AABF00EBC2505242184351
:10FA5C00BCBFD0401843704792F0000F81F40001F6
:10FA6C0006BF80F400000132013BB5E74FEA4103C9
:10FA7C007FEA226C18BF7FEA236C21D092EA030F35
:10FA8C0004D092F0000F08BF0846704790EA010FAF
:10FA9C001CBF0020704712F07F4F04D1400028BFDC
:10FAAC0040F00040704712F100723CBF00F50000BE
:10FABC00704700F0004343F0FE4040F400007047F4
:10FACC007FEA226216BF08467FEA236301464202A0
:10FADC0006BF5FEA412390EA010F40F480007047B3
:10FAEC004FF0000304E000BF10F0004348BF404259
:10FAFC005FEA000C08BF704743F0964301464FF095
:10FB0C0000001CE050EA010208BF70474FF00003F0
:10FB1C000AE000BF50EA010208BF704711F0004331
:10FB2C0002D5404261EB41015FEA010C02BF844601
:10FB3C000146002043F0B64308BFA3F18053A3F560
:10FB4C000003BCFA8CF2083AA3EBC25310DB01FAA7
:10FB5C0002FC634400FA02FCC2F12002BCF1004F2B
:10FB6C0020FA02F243EB020008BF20F001007047BC
:10FB7C0002F1200201FA02FCC2F1200250EA4C0010
:10FB8C0021FA02F243EB020008BF20EADC70704756
:10FB9C004FF0FF0C1CEAD0521EBF1CEAD15392EA64
:10FBAC000C0F93EA0C0F6FD01A4480EA010C400240
:10FBBC0018BF5FEA41211ED04FF0006343EA50109A
:10FBCC0043EA5111A0FB01310CF00040B1F5000FDC
:10FBDC003EBF490041EAD3715B0040EA010062F18B
:10FBEC007F02FD2A1DD8B3F1004F40EBC25008BF75
:10FBFC0020F00100704790F0000F0CF0004C08BF93
:10FC0C0049024CEA502040EA51207F3AC2BFD2F15F
:10FC1C00FF0340EAC250704740F400004FF000036D
:10FC2C00013A5DDC12F1190FDCBF00F000407047A7
:10FC3C00C2F10002410021FA02F1C2F1200200FAE5
:10FC4C0002FC5FEA310040F1000053EA4C0308BFAC
:10FC5C0020EADC70704792F0000F00F0004C02BFFD
:10FC6C00400010F4000F013AF9D040EA0C0093F078
:10FC7C00000F01F0004C02BF490011F4000F013BD2
:10FC8C00F9D041EA0C018FE70CEAD15392EA0C0F40
:10FC9C0018BF93EA0C0F0AD030F0004C18BF31F0AB
:10FCAC00004CD8D180EA010000F00040704790F081
:10FCBC00000F17BF90F0004F084691F0000F91F025
:10FCCC00004F14D092EA0C0F01D142020FD193EAEB
:10FCDC000C0F03D14B0218BF084608D180EA010073
:10FCEC0000F0004040F0FE4040F40000704740F04F
:10FCFC00FE4040F4400070474FF0FF0C1CEAD0521D
:10FD0C001EBF1CEAD15392EA0C0F93EA0C0F69D078
:10FD1C00A2EB030280EA010C49024FEA402037D0E3
:10FD2C004FF0805343EA111143EA10130CF00040DA
:10FD3C008B4238BF5B0042F17D024FF4000C8B42CA
:10FD4C0024BF5B1A40EA0C00B3EB510F24BFA3EBAA
:10FD5C00510340EA5C00B3EB910F24BFA3EB91037A
:10FD6C0040EA9C00B3EBD10F24BFA3EBD10340EAD4
:10FD7C00DC001B0118BF5FEA1C1CE0D1FD2A3FF61A
:10FD8C0050AF8B4240EBC25008BF20F001007047CF
:10FD9C000CF0004C4CEA50207F32C2BFD2F1FF0372
:10FDAC0040EAC250704740F400004FF00003013AA3
:10FDBC0037E792F0000F00F0004C02BF400010F447
:10FDCC00000F013AF9D040EA0C0093F0000F01F05B
:10FDDC00004C02BF490011F4000F013BF9D041EA7D
:10FDEC000C0195E70CEAD15392EA0C0F08D14202B0
:10FDFC007FF47DAF93EA0C0F7FF470AF084676E783
:10FE0C0093EA0C0F04D14B023FF44CAF08466EE75B
:10FE1C0030F0004C18BF31F0004CCAD130F0004229
:10FE2C007FF45CAF31F000437FF43CAF5FE700BF81
:10FE3C004FF0FF3C06E000BF4FF0010C02E000BFAA
:10FE4C004FF0010C4DF804CD4FEA40024FEA41034C
:10FE5C007FEA226C18BF7FEA236C11D001B052EA02
:10FE6C00530C18BF90EA010F58BFB2EB030088BFC8
:10FE7C00C81738BF6FEAE17018BF40F00100704737
:10FE8C007FEA226C02D15FEA402C05D17FEA236C19
:10FE9C00E4D15FEA412CE1D05DF8040B704700BF60
:10FEAC00844608466146FFE70FB5FFF7C9FF0028F7
:10FEBC0048BF10F1000F0FBD4DF808EDFFF7F4FF30
:10FECC000CBF012000205DF808FB00BF4DF808EDC9
:10FEDC00FFF7EAFF34BF012000205DF808FB00BFEC
:10FEEC004DF808EDFFF7E0FF94BF012000205DF80E
:10FEFC0008FB00BF4DF808EDFFF7D2FF94BF0120BF
:10FF0C0000205DF808FB00BF4DF808EDFFF7C8FFB7
:10FF1C0034BF012000205DF808FB00BF4FEA40020F
:10FF2C00B2F1FE4F0FD34FF09E03B3EB12620DD91B
:10FF3C004FEA002343F0004310F0004F23FA02F085
:10FF4C0018BF404270474FF00000704712F1610F2C
:10FF5C0001D1420205D110F0004008BF6FF0004003
:10FF6C0070474FF00000704754004D0043004D00A7
:10FF7C002D003100360033003000200028007600C0
:10FF8C00690072007400750061006C002000430071
:10FF9C004F004D002900200054004D0043004D003F
:10FFAC0031003600330000000000000000000000AB
:10FFBC0009024300020100C03209040000010202E0
:10FFCC000100052400100105240100010424020293
:10FFDC000524060001070582030800FF090401003F
:10FFEC00020A000000070503024000000705810219
:04FFFC0040000000C1
:020000040801F1
:100000000403090426035400720069006E006100B5
:100010006D00690063004D006F00740069006F009F
:100020006E002000430074006C0000005515AC6A9F
:10003000004001C0ABEA57956B7FD87EB87DA07CAD
:100040008F7B857A827985780878147726763D7556
:1000500059747B73A172367264719670CC6F076F9E
:10006000456EE66D2A6D726CBE6B0D6B5F6AB5698D
:100070006169BB6819687967DC664266AB65606573
:10008000CC643B64AD63206396620F62CB614761D1
:10009000C4604460C65F495FCE5E925E1A5EA45D36
:1000A0002F5DBD5C4B5CDC5BA55B385BCC5A625A58
:1000B000F95992592C59F95895583358D1577157C5
:1000C0001257B4560000C90092015B022403ED03ED
:1000D000B6047F0548061107D907A2086A09330A42
:1000E000FB0AC40B8C0C540D1C0EE30EAB0F7210EC
:1000F0003A110112C8128F1355141C15E215A816D7
:100100006E173318F918BE19821A471B0B1CCF1C27
:10011000931D571E1A1FDD1F9F2061212322E522F8
:10012000A62367242825E825A82667272628E5286A
:10013000A329612A1F2BDC2B992C552D112ECC2E97
:10014000872F4130FB30B5316E322633DF339634A2
:100150004D350436BA366F372438D9388C39403AA1
:10016000F23AA53B563C073DB83D683E173FC53FB8
:1001700073402141CE417A422543D0437A442445FD
:10018000CD4575461C47C34769480F49B449584A8D
:10019000FB4A9D4B3F4CE04C814D204EBF4E5D4F86
:1001A000FB4F97503351CE51685202539B533254F8
:1001B000C9546055F5558A561D57B0574258D35803
:1001C0006459F359825A0F5B9C5B285CB35C3E5DBB
:1001D000C75D4F5ED75E5D5FE35F6860EB606E6139
:1001E000F0617162F1627063EE636C64E864636590
:1001F000DD655666CF664667BC673268A6681969D2
:100200008B69FD696D6ADC6A4A6BB76B236C8E6C17
:10021000F86C616DC96D306E966EFB6E5E6FC16F6E
:1002200022708370E27040719D71F9715472AE72E8
:1002300007735E73B5730A745F74B2740475557591
:10024000A575F37541768D76D87622776B77B3777F
:10025000FA773F788478C77809794A798979C879B3
:10026000057A417A7C7AB67AEE7A267B5C7B917B42
:10027000C57BF87B297C597C887CB67CE37C0E7D31
:10028000397D627D897DB07DD57DFA7D1D7E3E7E86
:100290005F7E7E7E9C7EB97ED57EEF7E097F217F4C
:1002A000377F4D7F617F747F867F977FA67FB47F86
:1002B000C17FCD7FD87FE17FE97FF07FF57FF97F38
:1002C000FD7FFE7F0010161B2023272A2D3032359C
:1002D00037393B3D4041434547494B4C4E505153C4
:1002E000545657595A5B5D5E606162636566676824
:1002F0006A6B6C6D6E707172737475767778797ADB
:100300007B7C7D7E80808182838485868788898AC4
:100310008B8C8D8E8F9090919293949596969798C2
:10032000999A9B9B9C9D9E9FA0A0A1A2A3A3A4A5DC
:10033000A6A7A7A8A9AAAAABACADADAEAFB0B0B105
:10034000B2B2B3B4B5B5B6B7B7B8B9B9BABBBBBC3E
:10035000BDBDBEBFC0C0C1C1C2C3C3C4C5C5C6C781
:10036000C7C8C9C9CACBCBCCCCCDCECECFD0D0D1CB
:10037000D1D2D3D3D4D4D5D6D6D7D7D8D9D9DADA1F
:10038000DBDBDCDDDDDEDEDFE0E0E1E1E2E2E3E37A
:10039000E4E5E5E6E6E7E7E8E8E9EAEAEBEBECECDA
:1003A000EDEDEEEEEFF0F0F1F1F2F2F3F3F4F4F53F
:1003B000F5F6F6F7F7F8F8F9F9FAFAFBFBFCFCFDAD
:1003C000FDFEFEFF00000000010203040102030421
:1003D00006070809020406080200000000000001E8
:0C03E0003136333056323035000000005A
:1003EC00DC00000040000000FB070000FF070000DD
:1003FC0000080000140000000100000005000000CF
:10040C0006000000E00301080B0C0D0A0E080900A1
:10041C0001000000020000000300000004000000C6
:10042C00000800400100000000040040010101012F
:10043C0001010100A000000000C201000000080042
:10044C000000010804000000040001082600000060
:10045C00D400002032000000080100201A00000027
:10046C00BCFF000843000000C00000201200000088
:10047C003592000839900008858E0008998E000886
:10048C009D8E0008FD8E0008218F00082990000821
:10049C0019900008F58F00080000000040000000D3
:1004AC001201100102000040D016000002050102EA
:1004BC0003010000320354004D0043004D002D0099
:1004CC003000300030003000200028007600690039
:1004DC0072007400750061006C00200043004F0036
:1004EC004D002900200000001A0354004D00430069
:1004FC004D003000300030003000000000000000E3
:10050C0000000000858D0008E1C80008E1C8000863
:10051C00E1C80008E1C80008E1C80008E1C800080B
:10052C00E1C80008E1C8000889910008E1C800088A
:10053C00E1C80008E1C80008E1C800080401000097
:10054C00E1C80008618E0008E1C80008E1C8000895
:10055C00E1C80008E1C80008E1C80008E1C80008CB
:10056C00798E00080100000001000000010000006D
:040000050800410CA2
:00000001FF
